 luafar3

 Timestamp is 5685d19c (Fri Jan 01 04:08:44 2016)

 Preferred load address is 10000000

 Start         Length     Name                   Class
 0001:00000000 00000350H .idata$5                CODE
 0001:00000350 00000004H .CRT$XCA                CODE
 0001:00000354 00000004H .CRT$XCZ                CODE
 0001:00000358 00000004H .CRT$XIA                CODE
 0001:0000035c 00000010H .CRT$XIC                CODE
 0001:0000036c 00000004H .CRT$XIZ                CODE
 0001:00000370 00000004H .CRT$XPA                CODE
 0001:00000374 00000008H .CRT$XPX                CODE
 0001:0000037c 00000004H .CRT$XPXA               CODE
 0001:00000380 00000004H .CRT$XPZ                CODE
 0001:00000384 00000004H .CRT$XTA                CODE
 0001:00000388 00000004H .CRT$XTZ                CODE
 0001:00000390 00010d48H .rdata                  CODE
 0001:000110e0 0000000cH .rdata$sxdata           CODE
 0001:000110ec 00000004H .rtc$IAA                CODE
 0001:000110f0 00000004H .rtc$IZZ                CODE
 0001:000110f4 00000004H .rtc$TAA                CODE
 0001:000110f8 00000004H .rtc$TZZ                CODE
 0001:00011100 0002fa7eH .text                   CODE
 0001:00040b80 0000068cH .xdata$x                CODE
 0001:0004120c 00000064H .idata$2                CODE
 0001:00041270 00000014H .idata$3                CODE
 0001:00041284 00000350H .idata$4                CODE
 0001:000415d4 00000e66H .idata$6                CODE
 0001:00042440 00000482H .edata                  CODE
 0002:00000000 00008ee0H .data                   DATA
 0002:00008ee0 00001e44H .bss                    DATA
 0003:00000000 00000058H .rsrc$01                DATA
 0003:00000060 00000358H .rsrc$02                DATA

  Address         Publics by Value              Rva+Base       Lib:Object

 0000:00000000       __except_list              00000000     <absolute>
 0000:00000003       ___safe_se_handler_count   00000003     <absolute>
 0000:00000000       ___ImageBase               10000000     <linker-defined>
 0001:00000000       __imp__RegEnumKeyExW@32    10001000     advapi32:ADVAPI32.dll
 0001:00000004       __imp__RegDeleteValueW@8   10001004     advapi32:ADVAPI32.dll
 0001:00000008       __imp__RegQueryValueExW@24 10001008     advapi32:ADVAPI32.dll
 0001:0000000c       __imp__RegSetValueExW@24   1000100c     advapi32:ADVAPI32.dll
 0001:00000010       __imp__RegCloseKey@4       10001010     advapi32:ADVAPI32.dll
 0001:00000014       __imp__RegOpenKeyExW@20    10001014     advapi32:ADVAPI32.dll
 0001:00000018       __imp__RegCreateKeyExW@36  10001018     advapi32:ADVAPI32.dll
 0001:0000001c       __imp__RegDeleteKeyW@8     1000101c     advapi32:ADVAPI32.dll
 0001:00000020       __imp__RegEnumValueW@32    10001020     advapi32:ADVAPI32.dll
 0001:00000024       \177ADVAPI32_NULL_THUNK_DATA 10001024     advapi32:ADVAPI32.dll
 0001:00000028       __imp__GetModuleFileNameW@12 10001028     kernel32:KERNEL32.dll
 0001:0000002c       __imp__FreeLibrary@4       1000102c     kernel32:KERNEL32.dll
 0001:00000030       __imp__LoadLibraryW@4      10001030     kernel32:KERNEL32.dll
 0001:00000034       __imp__MultiByteToWideChar@24 10001034     kernel32:KERNEL32.dll
 0001:00000038       __imp__WideCharToMultiByte@32 10001038     kernel32:KERNEL32.dll
 0001:0000003c       __imp__GetACP@0            1000103c     kernel32:KERNEL32.dll
 0001:00000040       __imp__GetOEMCP@0          10001040     kernel32:KERNEL32.dll
 0001:00000044       __imp__GetDriveTypeW@4     10001044     kernel32:KERNEL32.dll
 0001:00000048       __imp__SearchPathW@24      10001048     kernel32:KERNEL32.dll
 0001:0000004c       __imp__OutputDebugStringW@4 1000104c     kernel32:KERNEL32.dll
 0001:00000050       __imp__FormatMessageW@28   10001050     kernel32:KERNEL32.dll
 0001:00000054       __imp__GetLastError@0      10001054     kernel32:KERNEL32.dll
 0001:00000058       __imp__EnumSystemCodePagesW@8 10001058     kernel32:KERNEL32.dll
 0001:0000005c       __imp__GetCPInfoExW@12     1000105c     kernel32:KERNEL32.dll
 0001:00000060       __imp__GetLogicalDriveStringsW@8 10001060     kernel32:KERNEL32.dll
 0001:00000064       __imp__GlobalMemoryStatusEx@4 10001064     kernel32:KERNEL32.dll
 0001:00000068       __imp__GetEnvironmentVariableW@12 10001068     kernel32:KERNEL32.dll
 0001:0000006c       __imp__GetCurrentDirectoryW@8 1000106c     kernel32:KERNEL32.dll
 0001:00000070       __imp__SetCurrentDirectoryW@4 10001070     kernel32:KERNEL32.dll
 0001:00000074       __imp__SetEnvironmentVariableW@8 10001074     kernel32:KERNEL32.dll
 0001:00000078       __imp__ReadConsoleInputW@16 10001078     kernel32:KERNEL32.dll
 0001:0000007c       __imp__PeekConsoleInputW@16 1000107c     kernel32:KERNEL32.dll
 0001:00000080       __imp__FindClose@4         10001080     kernel32:KERNEL32.dll
 0001:00000084       __imp__FindFirstFileW@8    10001084     kernel32:KERNEL32.dll
 0001:00000088       __imp__FileTimeToSystemTime@8 10001088     kernel32:KERNEL32.dll
 0001:0000008c       __imp__SystemTimeToFileTime@8 1000108c     kernel32:KERNEL32.dll
 0001:00000090       __imp__FileTimeToLocalFileTime@8 10001090     kernel32:KERNEL32.dll
 0001:00000094       __imp__CompareStringW@24   10001094     kernel32:KERNEL32.dll
 0001:00000098       __imp__CopyFileW@12        10001098     kernel32:KERNEL32.dll
 0001:0000009c       __imp__MoveFileExW@12      1000109c     kernel32:KERNEL32.dll
 0001:000000a0       __imp__DeleteFileW@4       100010a0     kernel32:KERNEL32.dll
 0001:000000a4       __imp__RemoveDirectoryW@4  100010a4     kernel32:KERNEL32.dll
 0001:000000a8       __imp__CreateDirectoryW@8  100010a8     kernel32:KERNEL32.dll
 0001:000000ac       __imp__GetFileAttributesW@4 100010ac     kernel32:KERNEL32.dll
 0001:000000b0       __imp__SwitchToThread@0    100010b0     kernel32:KERNEL32.dll
 0001:000000b4       __imp__CreateThread@24     100010b4     kernel32:KERNEL32.dll
 0001:000000b8       __imp__GetSystemTimeAsFileTime@4 100010b8     kernel32:KERNEL32.dll
 0001:000000bc       __imp__Sleep@4             100010bc     kernel32:KERNEL32.dll
 0001:000000c0       __imp__GetStdHandle@4      100010c0     kernel32:KERNEL32.dll
 0001:000000c4       __imp__GetConsoleScreenBufferInfo@8 100010c4     kernel32:KERNEL32.dll
 0001:000000c8       __imp__GetModuleHandleA@4  100010c8     kernel32:KERNEL32.dll
 0001:000000cc       __imp__SetFileAttributesW@8 100010cc     kernel32:KERNEL32.dll
 0001:000000d0       __imp__GetProcAddress@8    100010d0     kernel32:KERNEL32.dll
 0001:000000d4       __imp__HeapSize@12         100010d4     kernel32:KERNEL32.dll
 0001:000000d8       __imp__WriteConsoleW@20    100010d8     kernel32:KERNEL32.dll
 0001:000000dc       __imp__GetProcessHeap@0    100010dc     kernel32:KERNEL32.dll
 0001:000000e0       __imp__SetEndOfFile@4      100010e0     kernel32:KERNEL32.dll
 0001:000000e4       __imp__LCMapStringW@24     100010e4     kernel32:KERNEL32.dll
 0001:000000e8       __imp__HeapReAlloc@16      100010e8     kernel32:KERNEL32.dll
 0001:000000ec       __imp__CreateFileW@28      100010ec     kernel32:KERNEL32.dll
 0001:000000f0       __imp__SetStdHandle@8      100010f0     kernel32:KERNEL32.dll
 0001:000000f4       __imp__GetTickCount@0      100010f4     kernel32:KERNEL32.dll
 0001:000000f8       __imp__QueryPerformanceCounter@4 100010f8     kernel32:KERNEL32.dll
 0001:000000fc       __imp__GetModuleFileNameA@12 100010fc     kernel32:KERNEL32.dll
 0001:00000100       __imp__GetEnvironmentStringsW@0 10001100     kernel32:KERNEL32.dll
 0001:00000104       __imp__FreeEnvironmentStringsW@4 10001104     kernel32:KERNEL32.dll
 0001:00000108       __imp__FlushFileBuffers@4  10001108     kernel32:KERNEL32.dll
 0001:0000010c       __imp__GetConsoleMode@8    1000110c     kernel32:KERNEL32.dll
 0001:00000110       __imp__GetConsoleCP@0      10001110     kernel32:KERNEL32.dll
 0001:00000114       __imp__CreateFileA@28      10001114     kernel32:KERNEL32.dll
 0001:00000118       __imp__GetCurrentProcessId@0 10001118     kernel32:KERNEL32.dll
 0001:0000011c       __imp__WaitForSingleObject@8 1000111c     kernel32:KERNEL32.dll
 0001:00000120       __imp__GetExitCodeProcess@8 10001120     kernel32:KERNEL32.dll
 0001:00000124       __imp__CreatePipe@16       10001124     kernel32:KERNEL32.dll
 0001:00000128       __imp__IsValidCodePage@4   10001128     kernel32:KERNEL32.dll
 0001:0000012c       __imp__GetCPInfo@8         1000112c     kernel32:KERNEL32.dll
 0001:00000130       __imp__DeleteCriticalSection@4 10001130     kernel32:KERNEL32.dll
 0001:00000134       __imp__GetStartupInfoW@4   10001134     kernel32:KERNEL32.dll
 0001:00000138       __imp__GetFileType@4       10001138     kernel32:KERNEL32.dll
 0001:0000013c       __imp__SetHandleCount@4    1000113c     kernel32:KERNEL32.dll
 0001:00000140       __imp__SetFilePointer@16   10001140     kernel32:KERNEL32.dll
 0001:00000144       __imp__InterlockedDecrement@4 10001144     kernel32:KERNEL32.dll
 0001:00000148       __imp__SetLastError@4      10001148     kernel32:KERNEL32.dll
 0001:0000014c       __imp__InterlockedIncrement@4 1000114c     kernel32:KERNEL32.dll
 0001:00000150       __imp__TlsFree@4           10001150     kernel32:KERNEL32.dll
 0001:00000154       __imp__TlsSetValue@8       10001154     kernel32:KERNEL32.dll
 0001:00000158       __imp__TlsGetValue@4       10001158     kernel32:KERNEL32.dll
 0001:0000015c       __imp__TlsAlloc@0          1000115c     kernel32:KERNEL32.dll
 0001:00000160       __imp__ReadFile@20         10001160     kernel32:KERNEL32.dll
 0001:00000164       __imp__RtlUnwind@16        10001164     kernel32:KERNEL32.dll
 0001:00000168       __imp__InitializeCriticalSectionAndSpinCount@8 10001168     kernel32:KERNEL32.dll
 0001:0000016c       __imp__WriteFile@20        1000116c     kernel32:KERNEL32.dll
 0001:00000170       __imp__ExitProcess@4       10001170     kernel32:KERNEL32.dll
 0001:00000174       __imp__GetModuleHandleW@4  10001174     kernel32:KERNEL32.dll
 0001:00000178       __imp__HeapDestroy@4       10001178     kernel32:KERNEL32.dll
 0001:0000017c       __imp__HeapCreate@12       1000117c     kernel32:KERNEL32.dll
 0001:00000180       __imp__TerminateProcess@8  10001180     kernel32:KERNEL32.dll
 0001:00000184       __imp__IsDebuggerPresent@0 10001184     kernel32:KERNEL32.dll
 0001:00000188       __imp__SetUnhandledExceptionFilter@4 10001188     kernel32:KERNEL32.dll
 0001:0000018c       __imp__UnhandledExceptionFilter@4 1000118c     kernel32:KERNEL32.dll
 0001:00000190       __imp__IsProcessorFeaturePresent@4 10001190     kernel32:KERNEL32.dll
 0001:00000194       __imp__EncodePointer@4     10001194     kernel32:KERNEL32.dll
 0001:00000198       __imp__GetCommandLineA@0   10001198     kernel32:KERNEL32.dll
 0001:0000019c       __imp__DecodePointer@4     1000119c     kernel32:KERNEL32.dll
 0001:000001a0       __imp__GetCurrentThreadId@0 100011a0     kernel32:KERNEL32.dll
 0001:000001a4       __imp__CreateProcessW@40   100011a4     kernel32:KERNEL32.dll
 0001:000001a8       __imp__GetCurrentProcess@0 100011a8     kernel32:KERNEL32.dll
 0001:000001ac       __imp__DuplicateHandle@28  100011ac     kernel32:KERNEL32.dll
 0001:000001b0       __imp__CloseHandle@4       100011b0     kernel32:KERNEL32.dll
 0001:000001b4       __imp__GetStringTypeW@16   100011b4     kernel32:KERNEL32.dll
 0001:000001b8       __imp__LeaveCriticalSection@4 100011b8     kernel32:KERNEL32.dll
 0001:000001bc       __imp__EnterCriticalSection@4 100011bc     kernel32:KERNEL32.dll
 0001:000001c0       __imp__HeapAlloc@12        100011c0     kernel32:KERNEL32.dll
 0001:000001c4       __imp__HeapFree@12         100011c4     kernel32:KERNEL32.dll
 0001:000001c8       \177KERNEL32_NULL_THUNK_DATA 100011c8     kernel32:KERNEL32.dll
 0001:000001cc       __imp__UuidCreate@4        100011cc     rpcrt4:RPCRT4.dll
 0001:000001d0       __imp__RpcStringFreeA@4    100011d0     rpcrt4:RPCRT4.dll
 0001:000001d4       __imp__UuidToStringA@8     100011d4     rpcrt4:RPCRT4.dll
 0001:000001d8       __imp__UuidFromStringA@8   100011d8     rpcrt4:RPCRT4.dll
 0001:000001dc       \177RPCRT4_NULL_THUNK_DATA 100011dc     rpcrt4:RPCRT4.dll
 0001:000001e0       __imp__ShellExecuteW@24    100011e0     shell32:SHELL32.dll
 0001:000001e4       __imp__SHGetFolderPathW@20 100011e4     shell32:SHELL32.dll
 0001:000001e8       \177SHELL32_NULL_THUNK_DATA 100011e8     shell32:SHELL32.dll
 0001:000001ec       __imp__luaL_prepbuffer     100011ec     lua51:lua51.dll
 0001:000001f0       __imp__luaL_checkstack     100011f0     lua51:lua51.dll
 0001:000001f4       __imp__lua_dump            100011f4     lua51:lua51.dll
 0001:000001f8       __imp__lua_typename        100011f8     lua51:lua51.dll
 0001:000001fc       __imp__lua_tocfunction     100011fc     lua51:lua51.dll
 0001:00000200       __imp__luaL_checkoption    10001200     lua51:lua51.dll
 0001:00000204       __imp__luaL_gsub           10001204     lua51:lua51.dll
 0001:00000208       __imp__lua_iscfunction     10001208     lua51:lua51.dll
 0001:0000020c       __imp__luaL_findtable      1000120c     lua51:lua51.dll
 0001:00000210       __imp__lua_isuserdata      10001210     lua51:lua51.dll
 0001:00000214       __imp__lua_setallocf       10001214     lua51:lua51.dll
 0001:00000218       __imp__luaL_checknumber    10001218     lua51:lua51.dll
 0001:0000021c       __imp__lua_getfenv         1000121c     lua51:lua51.dll
 0001:00000220       __imp__lua_setfenv         10001220     lua51:lua51.dll
 0001:00000224       __imp__lua_settable        10001224     lua51:lua51.dll
 0001:00000228       __imp__lua_rawset          10001228     lua51:lua51.dll
 0001:0000022c       __imp__lua_getallocf       1000122c     lua51:lua51.dll
 0001:00000230       __imp__lua_next            10001230     lua51:lua51.dll
 0001:00000234       __imp__luaL_typerror       10001234     lua51:lua51.dll
 0001:00000238       __imp__luaopen_base        10001238     lua51:lua51.dll
 0001:0000023c       __imp__luaopen_table       1000123c     lua51:lua51.dll
 0001:00000240       __imp__luaopen_os          10001240     lua51:lua51.dll
 0001:00000244       __imp__luaopen_string      10001244     lua51:lua51.dll
 0001:00000248       __imp__luaopen_math        10001248     lua51:lua51.dll
 0001:0000024c       __imp__luaopen_debug       1000124c     lua51:lua51.dll
 0001:00000250       __imp__luaL_checktype      10001250     lua51:lua51.dll
 0001:00000254       __imp__lua_getstack        10001254     lua51:lua51.dll
 0001:00000258       __imp__lua_getinfo         10001258     lua51:lua51.dll
 0001:0000025c       __imp__luaL_addvalue       1000125c     lua51:lua51.dll
 0001:00000260       __imp__lua_checkstack      10001260     lua51:lua51.dll
 0001:00000264       __imp__luaL_error          10001264     lua51:lua51.dll
 0001:00000268       __imp__luaL_checklstring   10001268     lua51:lua51.dll
 0001:0000026c       __imp__luaL_optlstring     1000126c     lua51:lua51.dll
 0001:00000270       __imp__lua_replace         10001270     lua51:lua51.dll
 0001:00000274       __imp__luaL_checkudata     10001274     lua51:lua51.dll
 0001:00000278       __imp__luaL_buffinit       10001278     lua51:lua51.dll
 0001:0000027c       __imp__luaL_addlstring     1000127c     lua51:lua51.dll
 0001:00000280       __imp__luaL_pushresult     10001280     lua51:lua51.dll
 0001:00000284       __imp__luaL_checkany       10001284     lua51:lua51.dll
 0001:00000288       __imp__lua_concat          10001288     lua51:lua51.dll
 0001:0000028c       __imp__lua_load            1000128c     lua51:lua51.dll
 0001:00000290       __imp__lua_pushfstring     10001290     lua51:lua51.dll
 0001:00000294       __imp__luaL_loadstring     10001294     lua51:lua51.dll
 0001:00000298       __imp__lua_pushlstring     10001298     lua51:lua51.dll
 0001:0000029c       __imp__lua_pushlightuserdata 1000129c     lua51:lua51.dll
 0001:000002a0       __imp__lua_isnumber        100012a0     lua51:lua51.dll
 0001:000002a4       __imp__lua_tointeger       100012a4     lua51:lua51.dll
 0001:000002a8       __imp__lua_toboolean       100012a8     lua51:lua51.dll
 0001:000002ac       __imp__luaL_ref            100012ac     lua51:lua51.dll
 0001:000002b0       __imp__luaL_unref          100012b0     lua51:lua51.dll
 0001:000002b4       __imp__lua_gettable        100012b4     lua51:lua51.dll
 0001:000002b8       __imp__lua_isstring        100012b8     lua51:lua51.dll
 0001:000002bc       __imp__lua_objlen          100012bc     lua51:lua51.dll
 0001:000002c0       __imp__lua_rawseti         100012c0     lua51:lua51.dll
 0001:000002c4       __imp__lua_createtable     100012c4     lua51:lua51.dll
 0001:000002c8       __imp__lua_setfield        100012c8     lua51:lua51.dll
 0001:000002cc       __imp__lua_rawgeti         100012cc     lua51:lua51.dll
 0001:000002d0       __imp__lua_pushcclosure    100012d0     lua51:lua51.dll
 0001:000002d4       __imp__lua_insert          100012d4     lua51:lua51.dll
 0001:000002d8       __imp__lua_pcall           100012d8     lua51:lua51.dll
 0001:000002dc       __imp__lua_remove          100012dc     lua51:lua51.dll
 0001:000002e0       __imp__lua_gc              100012e0     lua51:lua51.dll
 0001:000002e4       __imp__lua_pushvalue       100012e4     lua51:lua51.dll
 0001:000002e8       __imp__lua_pushinteger     100012e8     lua51:lua51.dll
 0001:000002ec       __imp__lua_call            100012ec     lua51:lua51.dll
 0001:000002f0       __imp__luaL_newmetatable   100012f0     lua51:lua51.dll
 0001:000002f4       __imp__luaL_register       100012f4     lua51:lua51.dll
 0001:000002f8       __imp__lua_pushboolean     100012f8     lua51:lua51.dll
 0001:000002fc       __imp__lua_pushstring      100012fc     lua51:lua51.dll
 0001:00000300       __imp__lua_tolstring       10001300     lua51:lua51.dll
 0001:00000304       __imp__lua_pushnil         10001304     lua51:lua51.dll
 0001:00000308       __imp__luaL_checkinteger   10001308     lua51:lua51.dll
 0001:0000030c       __imp__lua_gettop          1000130c     lua51:lua51.dll
 0001:00000310       __imp__lua_tonumber        10001310     lua51:lua51.dll
 0001:00000314       __imp__luaL_argerror       10001314     lua51:lua51.dll
 0001:00000318       __imp__lua_type            10001318     lua51:lua51.dll
 0001:0000031c       __imp__lua_getmetatable    1000131c     lua51:lua51.dll
 0001:00000320       __imp__lua_rawequal        10001320     lua51:lua51.dll
 0001:00000324       __imp__lua_settop          10001324     lua51:lua51.dll
 0001:00000328       __imp__lua_touserdata      10001328     lua51:lua51.dll
 0001:0000032c       __imp__lua_pushnumber      1000132c     lua51:lua51.dll
 0001:00000330       __imp__lua_newuserdata     10001330     lua51:lua51.dll
 0001:00000334       __imp__lua_getfield        10001334     lua51:lua51.dll
 0001:00000338       __imp__lua_setmetatable    10001338     lua51:lua51.dll
 0001:0000033c       __imp__lua_rawget          1000133c     lua51:lua51.dll
 0001:00000340       __imp__lua_error           10001340     lua51:lua51.dll
 0001:00000344       __imp__luaL_optnumber      10001344     lua51:lua51.dll
 0001:00000348       __imp__luaL_optinteger     10001348     lua51:lua51.dll
 0001:0000034c       \177lua51_NULL_THUNK_DATA  1000134c     lua51:lua51.dll
 0001:00000350       ___xc_a                    10001350     LIBCMT:crt0init.obj
 0001:00000354       ___xc_z                    10001354     LIBCMT:crt0init.obj
 0001:00000358       ___xi_a                    10001358     LIBCMT:crt0init.obj
 0001:0000036c       ___xi_z                    1000136c     LIBCMT:crt0init.obj
 0001:00000370       ___xp_a                    10001370     LIBCMT:crt0init.obj
 0001:00000380       ___xp_z                    10001380     LIBCMT:crt0init.obj
 0001:00000384       ___xt_a                    10001384     LIBCMT:crt0init.obj
 0001:00000388       ___xt_z                    10001388     LIBCMT:crt0init.obj
 0001:00000390       ??_C@_0L@HDFPAPPH@__tostring?$AA@ 10001390     bit64.obj
 0001:0000039c       ??_C@_04EJLHOCKK@__le?$AA@ 1000139c     bit64.obj
 0001:000003a4       ??_C@_04BKGOMBLK@__lt?$AA@ 100013a4     bit64.obj
 0001:000003ac       ??_C@_04GIMIAOHA@__eq?$AA@ 100013ac     bit64.obj
 0001:000003b4       ??_C@_05MHFNBPAK@__unm?$AA@ 100013b4     bit64.obj
 0001:000003bc       ??_C@_05ICPALBAE@__mod?$AA@ 100013bc     bit64.obj
 0001:000003c4       ??_C@_05IDIBPCOP@__div?$AA@ 100013c4     bit64.obj
 0001:000003cc       ??_C@_05FLJIBNKK@__mul?$AA@ 100013cc     bit64.obj
 0001:000003d4       ??_C@_05HFNNBAII@__sub?$AA@ 100013d4     bit64.obj
 0001:000003dc       ??_C@_05MEHDOBFN@__add?$AA@ 100013dc     bit64.obj
 0001:000003e4       ??_C@_04GPMDFGEJ@type?$AA@ 100013e4     bit64.obj
 0001:000003ec       ??_C@_02FJPJILEL@le?$AA@   100013ec     bit64.obj
 0001:000003f0       ??_C@_02KCAKIFL@lt?$AA@    100013f0     bit64.obj
 0001:000003f4       ??_C@_02HIIGGHJB@eq?$AA@   100013f4     bit64.obj
 0001:000003f8       ??_C@_03FFONCNID@mod?$AA@  100013f8     bit64.obj
 0001:000003fc       ??_C@_03FEJMGOGI@div?$AA@  100013fc     bit64.obj
 0001:00000400       ??_C@_03IMIFIBCN@mul?$AA@  10001400     bit64.obj
 0001:00000404       ??_C@_03KCMAIMAP@sub?$AA@  10001404     bit64.obj
 0001:00000408       ??_C@_03BDGOHNNK@add?$AA@  10001408     bit64.obj
 0001:0000040c       ??_C@_03CLCAEGCJ@new?$AA@  1000140c     bit64.obj
 0001:00000410       ??_C@_07JILILBLL@arshift?$AA@ 10001410     bit64.obj
 0001:00000418       ??_C@_06HMLHBBIJ@rshift?$AA@ 10001418     bit64.obj
 0001:00000420       ??_C@_06ELFGPGBK@lshift?$AA@ 10001420     bit64.obj
 0001:00000428       ??_C@_04CKCGDDNF@bxor?$AA@ 10001428     bit64.obj
 0001:00000430       ??_C@_03BBBGIIAC@bor?$AA@  10001430     bit64.obj
 0001:00000434       ??_C@_04BKGNPECA@band?$AA@ 10001434     bit64.obj
 0001:0000043c       ??_C@_04JAOJMBA@bnot?$AA@  1000143c     bit64.obj
 0001:00000448       _metatable_name            10001448     bit64.obj
 0001:00000540       ??_C@_09GPALILFO@bad?5int64?$AA@ 10001540     bit64.obj
 0001:00000550       __real@433fffffffffffff    10001550     bit64.obj
 0001:00000558       ??_C@_05LLAMLEHD@?$CFI64d?$AA@ 10001558     bit64.obj
 0001:00000560       ??_C@_05OALCLICP@bit64?$AA@ 10001560     bit64.obj
 0001:00000d90       _COLLECTOR_FD              10001d90     exported.obj
 0001:00000da4       _COLLECTOR_OPI             10001da4     exported.obj
 0001:00000dbc       _COLLECTOR_PI              10001dbc     exported.obj
 0001:00000dd4       _KEY_OBJECT                10001dd4     exported.obj
 0001:00000ddc       ??_C@_09GPFEECNC@traceback?$AA@ 10001ddc     exported.obj
 0001:00000de8       ??_C@_05GFCDIDHO@debug?$AA@ 10001de8     exported.obj
 0001:00000df0       ??_C@_06NKNNMLDJ@export?$AA@ 10001df0     exported.obj
 0001:00000df8       ??_C@_07PCNKBAGB@OnError?$AA@ 10001df8     exported.obj
 0001:00000e00       ??_C@_08JNHPECBG@UserData?$AA@ 10001e00     exported.obj
 0001:00000e0c       ??_C@_01LOCGONAA@?$AA?$AA@ 10001e0c     service.obj
 0001:00000e0c       ??_C@_11LOCGONAA@?$AA?$AA@ 10001e0c     exported.obj
 0001:00000e10       ??_C@_0BB@OKGMKOG@CustomColumnData?$AA@ 10001e10     exported.obj
 0001:00000e24       ??_C@_05HDCNEILF@Owner?$AA@ 10001e24     exported.obj
 0001:00000e2c       ??_C@_0M@OHKMKKDH@Description?$AA@ 10001e2c     exported.obj
 0001:00000e38       ??_C@_0BC@COCBGKAE@AlternateFileName?$AA@ 10001e38     exported.obj
 0001:00000e4c       ??_C@_08FDCJCDOL@FileName?$AA@ 10001e4c     exported.obj
 0001:00000e58       ??_C@_05MHNOECFO@CRC32?$AA@ 10001e58     exported.obj
 0001:00000e60       ??_C@_0O@DLGJHFNH@NumberOfLinks?$AA@ 10001e60     exported.obj
 0001:00000e70       ??_C@_05BOOEKJH@Flags?$AA@ 10001e70     exported.obj
 0001:00000e78       ??_C@_0P@JBACEJLL@AllocationSize?$AA@ 10001e78     exported.obj
 0001:00000e88       ??_C@_08BHIEONMC@FileSize?$AA@ 10001e88     exported.obj
 0001:00000e94       ??_C@_0L@FCILKIIG@ChangeTime?$AA@ 10001e94     exported.obj
 0001:00000ea0       ??_C@_0O@FCFNCAHK@LastWriteTime?$AA@ 10001ea0     exported.obj
 0001:00000eb0       ??_C@_0P@MFHPCDDH@LastAccessTime?$AA@ 10001eb0     exported.obj
 0001:00000ec0       ??_C@_0N@NJMIGDDL@CreationTime?$AA@ 10001ec0     exported.obj
 0001:00000ed0       ??_C@_0M@DFMHDHBL@GetFindData?$AA@ 10001ed0     exported.obj
 0001:00000edc       ??_C@_08CJLOJPNI@selected?$AA@ 10001edc     exported.obj
 0001:00000ee8       ??_C@_0BC@IECOKJFL@GetFiles?4DestPath?$AA@ 10001ee8     exported.obj
 0001:00000efc       ??_C@_08FFPEEIHA@GetFiles?$AA@ 10001efc     exported.obj
 0001:00000f08       ??_C@_1DC@PABHCCON@?$AAD?$AAe?$AAf?$AAa?$AAu?$AAl?$AAt?$AA?5?$AAs?$AAc?$AAr?$AAi?$AAp?$AAt?$AA?5?$AAn?$AAo?$AAt?$AA?5?$AAf?$AAo?$AAu?$AAn?$AAd?$AA?$AA@ 10001f08     exported.obj
 0001:00000f3c       ??_C@_13BPINEIPE@?$AAr?$AA?$AA@ 10001f3c     exported.obj
 0001:00000f40       ??_C@_19BCNABNAK@?$AA?4?$AAl?$AAu?$AAa?$AA?$AA@ 10001f40     exported.obj
 0001:00000f4c       ??_C@_05LFOKGKBN@?$DMboot?$AA@ 10001f4c     exported.obj
 0001:00000f54       ??_C@_07GCEAJMEA@preload?$AA@ 10001f54     exported.obj
 0001:00000f5c       ??_C@_07KNEGBPNO@package?$AA@ 10001f5c     exported.obj
 0001:00000f64       ??_C@_15CBMDENPJ@?$AA?4?$AA?9?$AA?$AA@ 10001f64     exported.obj
 0001:00000f6c       ??_C@_0BE@HCPAIELH@ReloadDefaultScript?$AA@ 10001f6c     exported.obj
 0001:00000f80       ??_C@_03JEOKDCFP@far?$AA@  10001f80     exported.obj
 0001:00000f84       ??_C@_06EPIAKPGD@OpMode?$AA@ 10001f84     exported.obj
 0001:00000f8c       ??_C@_06LBMCOACO@Buffer?$AA@ 10001f8c     exported.obj
 0001:00000f94       ??_C@_0L@OCPPMCCK@StructSize?$AA@ 10001f94     exported.obj
 0001:00000fa0       ??_C@_07GDADDFBD@Analyse?$AA@ 10001fa0     exported.obj
 0001:00000fa8       ??_C@_0N@IHDKLODA@ShortcutData?$AA@ 10001fa8     exported.obj
 0001:00000fb8       ??_C@_08DGDJEKCP@LongText?$AA@ 10001fb8     exported.obj
 0001:00000fc4       ??_C@_0BA@MFFHAKP@ControlKeyState?$AA@ 10001fc4     exported.obj
 0001:00000fd4       ??_C@_0P@PKDBPEJI@VirtualKeyCode?$AA@ 10001fd4     exported.obj
 0001:00000fe4       ??_C@_06ONGFDHIA@KeyBar?$AA@ 10001fe4     exported.obj
 0001:00000fec       ??_C@_0P@KMACBLNK@StartSortOrder?$AA@ 10001fec     exported.obj
 0001:00000ffc       ??_C@_0O@NIFKFGBJ@StartSortMode?$AA@ 10001ffc     exported.obj
 0001:0000100c       ??_C@_0P@BEEDPJDK@StartPanelMode?$AA@ 1000200c     exported.obj
 0001:0000101c       ??_C@_0N@EHCEJHEE@ColumnTitles?$AA@ 1000201c     exported.obj
 0001:0000102c       ??_C@_0BD@DNDIPKDK@StatusColumnWidths?$AA@ 1000202c     exported.obj
 0001:00001040       ??_C@_0BC@KELOOKNK@StatusColumnTypes?$AA@ 10002040     exported.obj
 0001:00001054       ??_C@_0N@ILFJPGHI@ColumnWidths?$AA@ 10002054     exported.obj
 0001:00001064       ??_C@_0M@KDJPJFOF@ColumnTypes?$AA@ 10002064     exported.obj
 0001:00001070       ??_C@_0BB@LFNABPEF@PanelModesNumber?$AA@ 10002070     exported.obj
 0001:00001084       ??_C@_0BA@BBOGKOKF@PanelModesArray?$AA@ 10002084     exported.obj
 0001:00001094       ??_C@_0L@FPEHOFAI@DescrFiles?$AA@ 10002094     exported.obj
 0001:000010a0       ??_C@_04DICKPMGH@Data?$AA@ 100020a0     exported.obj
 0001:000010a8       ??_C@_04OJAHODMC@Text?$AA@ 100020a8     exported.obj
 0001:000010b0       ??_C@_0BA@BLCGOCOG@InfoLinesNumber?$AA@ 100020b0     exported.obj
 0001:000010c0       ??_C@_09PMEOAIAA@InfoLines?$AA@ 100020c0     exported.obj
 0001:000010cc       ??_C@_0L@CMHIOLLB@PanelTitle?$AA@ 100020cc     exported.obj
 0001:000010d8       ??_C@_06PEPCFMNJ@Format?$AA@ 100020d8     exported.obj
 0001:000010e0       ??_C@_06IBPEEEAJ@CurDir?$AA@ 100020e0     exported.obj
 0001:000010e8       ??_C@_08PAJOMFPO@HostFile?$AA@ 100020e8     exported.obj
 0001:000010f4       ??_C@_08KDMNIFGM@FreeSize?$AA@ 100020f4     exported.obj
 0001:00001100       ??_C@_1EO@OOOCECGK@?$AAG?$AAe?$AAt?$AAO?$AAp?$AAe?$AAn?$AAP?$AAa?$AAn?$AAe?$AAl?$AAI?$AAn?$AAf?$AAo?$AA?5?$AAs?$AAh?$AAo?$AAu?$AAl?$AAd?$AA?5?$AAr?$AAe?$AAt?$AAu?$AAr?$AAn?$AA?5?$AAa@ 10002100     exported.obj
 0001:00001150       ??_C@_05ELNJBDOO@reuse?$AA@ 10002150     exported.obj
 0001:00001158       ??_C@_0BB@CKIGBGLB@GetOpenPanelInfo?$AA@ 10002158     exported.obj
 0001:0000116c       ??_C@_05HIFJDKLD@array?$AA@ 1000216c     exported.obj
 0001:00001174       ??_C@_01EFFIKLCJ@n?$AA@    10002174     exported.obj
 0001:00001176       ??_C@_00CNPNBAHC@?$AA@     10002176     exported.obj
 0001:00001178       __real@bff0000000000000    10002178     exported.obj
 0001:00001180       ??_C@_05LNOAKADA@panel?$AA@ 10002180     exported.obj
 0001:00001188       ??_C@_06BNNOMDLO@Handle?$AA@ 10002188     exported.obj
 0001:00001190       ??_C@_04OPJIDECA@hDlg?$AA@ 10002190     exported.obj
 0001:00001198       ??_C@_04DNCDCIAE@Open?$AA@ 10002198     exported.obj
 0001:000011a0       ??_C@_0L@JMPDJFBN@ClosePanel?$AA@ 100021a0     exported.obj
 0001:000011ac       ??_C@_07MBOMJGGF@Compare?$AA@ 100021ac     exported.obj
 0001:000011b4       ??_C@_09NANCCILE@Configure?$AA@ 100021b4     exported.obj
 0001:000011c0       ??_C@_0M@MMKKMEFA@DeleteFiles?$AA@ 100021c0     exported.obj
 0001:000011cc       ??_C@_0BD@PJNONGDB@MakeDirectory?4Name?$AA@ 100021cc     exported.obj
 0001:000011e0       ??_C@_0O@GLLEDHJA@MakeDirectory?$AA@ 100021e0     exported.obj
 0001:000011f0       ??_C@_0BC@COPMJGBI@ProcessPanelEvent?$AA@ 100021f0     exported.obj
 0001:00001204       ??_C@_0BA@DPJAKFGC@ProcessHostFile?$AA@ 10002204     exported.obj
 0001:00001214       ??_C@_0BC@HOBKGBBM@ProcessPanelInput?$AA@ 10002214     exported.obj
 0001:00001228       ??_C@_08OBOOFGOD@PutFiles?$AA@ 10002228     exported.obj
 0001:00001234       ??_C@_0N@KCFEBPAO@SetDirectory?$AA@ 10002234     exported.obj
 0001:00001244       ??_C@_0M@PNOHHCCH@SetFindList?$AA@ 10002244     exported.obj
 0001:00001250       ??_C@_07EACELFAO@ExitFAR?$AA@ 10002250     exported.obj
 0001:00001258       ??_C@_0BE@GAFPNGIP@PluginConfigStrings?$AA@ 10002258     exported.obj
 0001:0000126c       ??_C@_0BC@ILBHAHCH@PluginConfigGuids?$AA@ 1000226c     exported.obj
 0001:00001280       ??_C@_0BC@DJMJFBJC@PluginMenuStrings?$AA@ 10002280     exported.obj
 0001:00001294       ??_C@_0BA@FOMPNLJF@PluginMenuGuids?$AA@ 10002294     exported.obj
 0001:000012a4       ??_C@_0BA@NLBDFPEO@DiskMenuStrings?$AA@ 100022a4     exported.obj
 0001:000012b4       ??_C@_0O@PHBKMNMJ@DiskMenuGuids?$AA@ 100022b4     exported.obj
 0001:000012c4       ??_C@_0O@GDMHGAFH@CommandPrefix?$AA@ 100022c4     exported.obj
 0001:000012d4       ??_C@_0O@OBCKADMD@GetPluginInfo?$AA@ 100022d4     exported.obj
 0001:000012e4       ??_C@_0BD@DECJPBBK@ProcessEditorInput?$AA@ 100022e4     exported.obj
 0001:000012f8       ??_C@_08DOHJINHB@CodePage?$AA@ 100022f8     exported.obj
 0001:00001304       ??_C@_07MOCFLHCN@FileEOL?$AA@ 10002304     exported.obj
 0001:0000130c       ??_C@_0N@EKPHGDMI@StringNumber?$AA@ 1000230c     exported.obj
 0001:0000131c       ??_C@_04KOACHJEN@Type?$AA@ 1000231c     exported.obj
 0001:00001324       ??_C@_0BD@GEMPAGBO@ProcessEditorEvent?$AA@ 10002324     exported.obj
 0001:00001338       ??_C@_0BD@GGKMLEJG@ProcessViewerEvent?$AA@ 10002338     exported.obj
 0001:0000134c       ??_C@_03MLMOILGK@Msg?$AA@  1000234c     exported.obj
 0001:00001350       ??_C@_06EDEGJMB@Param1?$AA@ 10002350     exported.obj
 0001:00001358       ??_C@_06CPBJDKAC@Param2?$AA@ 10002358     exported.obj
 0001:00001360       ??_C@_0BD@FNHBEIC@ProcessDialogEvent?$AA@ 10002360     exported.obj
 0001:00001374       ??_C@_0BE@LHJGGGHN@ProcessSynchroEvent?$AA@ 10002374     exported.obj
 0001:00001388       ??_C@_0BB@PHIEFGHD@GetContentFields?$AA@ 10002388     exported.obj
 0001:0000139c       ??_C@_0P@DPJDPMPI@GetContentData?$AA@ 1000239c     exported.obj
 0001:000013ac       ??_C@_06HHECMMLE@Author?$AA@ 100023ac     exported.obj
 0001:000013b4       ??_C@_05PABKJLOM@Title?$AA@ 100023b4     exported.obj
 0001:000013bc       ??_C@_04MJHIICBJ@Guid?$AA@ 100023bc     exported.obj
 0001:000013c4       ??_C@_07NGFJPNPN@Version?$AA@ 100023c4     exported.obj
 0001:000013cc       ??_C@_0O@CALOEOI@MinFarVersion?$AA@ 100023cc     exported.obj
 0001:000013dc       ??_C@_0O@GJMOPLGM@GetGlobalInfo?$AA@ 100023dc     exported.obj
 0001:000013ec       ??_C@_1CA@IBKDMBNJ@?$AA_?$AAg?$AAl?$AAo?$AAb?$AAa?$AAl?$AAi?$AAn?$AAf?$AAo?$AA?4?$AAl?$AAu?$AAa?$AA?$AA@ 100023ec     exported.obj
 0001:0000140c       ??_C@_0N@DDJEHLKE@?$DM_globalinfo?$AA@ 1000240c     exported.obj
 0001:0000141c       ??_C@_0BE@DONMOPMJ@ProcessConsoleInput?$AA@ 1000241c     exported.obj
 0001:00001430       ??_C@_0O@GABDOPO@MOUSE_WHEELED?$AA@ 10002430     flags.obj
 0001:00001440       ??_C@_0N@EDCKBGJE@DOUBLE_CLICK?$AA@ 10002440     flags.obj
 0001:00001450       ??_C@_0M@KKBDEELB@MOUSE_MOVED?$AA@ 10002450     flags.obj
 0001:0000145c       ??_C@_0BN@CNMHAAPD@FROM_LEFT_4TH_BUTTON_PRESSED?$AA@ 1000245c     flags.obj
 0001:0000147c       ??_C@_0BN@PMJNFPGM@FROM_LEFT_3RD_BUTTON_PRESSED?$AA@ 1000247c     flags.obj
 0001:0000149c       ??_C@_0BN@BJCFPKCG@FROM_LEFT_2ND_BUTTON_PRESSED?$AA@ 1000249c     flags.obj
 0001:000014bc       ??_C@_0BJ@JECFAJNJ@RIGHTMOST_BUTTON_PRESSED?$AA@ 100024bc     flags.obj
 0001:000014d8       ??_C@_0BN@HACKHGAB@FROM_LEFT_1ST_BUTTON_PRESSED?$AA@ 100024d8     flags.obj
 0001:000014f8       ??_C@_0O@LAHFNPLG@SCROLLLOCK_ON?$AA@ 100024f8     flags.obj
 0001:00001508       ??_C@_0L@IMGKKBIM@NUMLOCK_ON?$AA@ 10002508     flags.obj
 0001:00001514       ??_C@_0O@OGDFJMBK@SHIFT_PRESSED?$AA@ 10002514     flags.obj
 0001:00001524       ??_C@_0BC@FDNOAAAE@LEFT_CTRL_PRESSED?$AA@ 10002524     flags.obj
 0001:00001538       ??_C@_0BD@NEHHNAHO@RIGHT_CTRL_PRESSED?$AA@ 10002538     flags.obj
 0001:0000154c       ??_C@_0BB@MCADLJJO@LEFT_ALT_PRESSED?$AA@ 1000254c     flags.obj
 0001:00001560       ??_C@_0BC@GDHABBAP@RIGHT_ALT_PRESSED?$AA@ 10002560     flags.obj
 0001:00001574       ??_C@_0N@EMEOEKDA@ENHANCED_KEY?$AA@ 10002574     flags.obj
 0001:00001584       ??_C@_0M@MKBGBFGO@CAPSLOCK_ON?$AA@ 10002584     flags.obj
 0001:00001590       ??_C@_0M@LNGHCCGJ@FOCUS_EVENT?$AA@ 10002590     flags.obj
 0001:0000159c       ??_C@_0L@MPODFLFH@MENU_EVENT?$AA@ 1000259c     flags.obj
 0001:000015a8       ??_C@_0BJ@OHDOHJKG@WINDOW_BUFFER_SIZE_EVENT?$AA@ 100025a8     flags.obj
 0001:000015c4       ??_C@_0M@CPILDGOO@MOUSE_EVENT?$AA@ 100025c4     flags.obj
 0001:000015d0       ??_C@_09JBABGNAE@KEY_EVENT?$AA@ 100025d0     flags.obj
 0001:000015dc       ??_C@_0BK@CDKLKCHJ@ENABLE_WRAP_AT_EOL_OUTPUT?$AA@ 100025dc     flags.obj
 0001:000015f8       ??_C@_0BI@MHKNPIFM@ENABLE_PROCESSED_OUTPUT?$AA@ 100025f8     flags.obj
 0001:00001610       ??_C@_0BF@PEBFEBKN@ENABLE_AUTO_POSITION?$AA@ 10002610     flags.obj
 0001:00001628       ??_C@_0BG@CBCHHIEH@ENABLE_EXTENDED_FLAGS?$AA@ 10002628     flags.obj
 0001:00001640       ??_C@_0BH@BJKMFKAO@ENABLE_QUICK_EDIT_MODE?$AA@ 10002640     flags.obj
 0001:00001658       ??_C@_0BD@KJBPOMPN@ENABLE_INSERT_MODE?$AA@ 10002658     flags.obj
 0001:0000166c       ??_C@_0BD@BJECBJPO@ENABLE_MOUSE_INPUT?$AA@ 1000266c     flags.obj
 0001:00001680       ??_C@_0BE@BLAHACNB@ENABLE_WINDOW_INPUT?$AA@ 10002680     flags.obj
 0001:00001694       ??_C@_0BH@EHINFMOF@ENABLE_PROCESSED_INPUT?$AA@ 10002694     flags.obj
 0001:000016ac       ??_C@_0BC@JPFKLHOC@ENABLE_ECHO_INPUT?$AA@ 100026ac     flags.obj
 0001:000016c0       ??_C@_0BC@BBOPHMOM@ENABLE_LINE_INPUT?$AA@ 100026c0     flags.obj
 0001:000016d4       ??_C@_0BE@BCNEFGKM@CTRL_SHUTDOWN_EVENT?$AA@ 100026d4     flags.obj
 0001:000016e8       ??_C@_0BC@MCKCEPAL@CTRL_LOGOFF_EVENT?$AA@ 100026e8     flags.obj
 0001:000016fc       ??_C@_0BB@KMPDMOKK@CTRL_CLOSE_EVENT?$AA@ 100026fc     flags.obj
 0001:00001710       ??_C@_0BB@ELEIIFAE@CTRL_BREAK_EVENT?$AA@ 10002710     flags.obj
 0001:00001724       ??_C@_0N@FEFOEFHG@CTRL_C_EVENT?$AA@ 10002724     flags.obj
 0001:00001734       ??_C@_0BF@NIGKKPCF@BACKGROUND_INTENSITY?$AA@ 10002734     flags.obj
 0001:0000174c       ??_C@_0P@DANALJMC@BACKGROUND_RED?$AA@ 1000274c     flags.obj
 0001:0000175c       ??_C@_0BB@GKLNBMEL@BACKGROUND_GREEN?$AA@ 1000275c     flags.obj
 0001:00001770       ??_C@_0BA@PIFINJCK@BACKGROUND_BLUE?$AA@ 10002770     flags.obj
 0001:00001780       ??_C@_0BF@OOGEJCC@FOREGROUND_INTENSITY?$AA@ 10002780     flags.obj
 0001:00001798       ??_C@_0P@PBJHCFGA@FOREGROUND_RED?$AA@ 10002798     flags.obj
 0001:000017a8       ??_C@_0BB@PDFNMAI@FOREGROUND_GREEN?$AA@ 100027a8     flags.obj
 0001:000017bc       ??_C@_0BA@MAEBFMHC@FOREGROUND_BLUE?$AA@ 100027bc     flags.obj
 0001:000017cc       ??_C@_09HNBBLIGN@PCIF_NONE?$AA@ 100027cc     flags.obj
 0001:000017d8       ??_C@_0O@PLFENGLI@PCIF_FROMMAIN?$AA@ 100027d8     flags.obj
 0001:000017e8       ??_C@_09FMOOJHDF@FOSF_NONE?$AA@ 100027e8     flags.obj
 0001:000017f4       ??_C@_0M@MIGJPBPE@FOSF_ACTIVE?$AA@ 100027f4     flags.obj
 0001:00001800       ??_C@_08EGEBMPBD@OPM_NONE?$AA@ 10002800     flags.obj
 0001:0000180c       ??_C@_0N@HKCLLJDG@OPM_COMMANDS?$AA@ 1000280c     flags.obj
 0001:0000181c       ??_C@_08LCEGJCAC@OPM_PGDN?$AA@ 1000281c     flags.obj
 0001:00001828       ??_C@_0O@OPDAGBBE@OPM_QUICKVIEW?$AA@ 10002828     flags.obj
 0001:00001838       ??_C@_09EBKAPHPA@OPM_DESCR?$AA@ 10002838     flags.obj
 0001:00001844       ??_C@_0N@NDGKAFDM@OPM_TOPLEVEL?$AA@ 10002844     flags.obj
 0001:00001854       ??_C@_08LAAGEMJG@OPM_EDIT?$AA@ 10002854     flags.obj
 0001:00001860       ??_C@_08EHBLNDLO@OPM_VIEW?$AA@ 10002860     flags.obj
 0001:0000186c       ??_C@_08EKEBOKEP@OPM_FIND?$AA@ 1000286c     flags.obj
 0001:00001878       ??_C@_0L@GEHHKNBL@OPM_SILENT?$AA@ 10002878     flags.obj
 0001:00001884       ??_C@_09DOPJBMLM@OPIF_NONE?$AA@ 10002884     flags.obj
 0001:00001890       ??_C@_0O@FJPLJDBC@OPIF_SHORTCUT?$AA@ 10002890     flags.obj
 0001:000018a0       ??_C@_0BB@PFDFAFHG@OPIF_USEFREESIZE?$AA@ 100028a0     flags.obj
 0001:000018b4       ??_C@_0O@JHHHMHIG@OPIF_USECRC32?$AA@ 100028b4     flags.obj
 0001:000018c4       ??_C@_0BJ@CALDMPLF@OPIF_USEATTRHIGHLIGHTING?$AA@ 100028c4     flags.obj
 0001:000018e0       ??_C@_0BD@JIMJPFEP@OPIF_EXTERNALMKDIR?$AA@ 100028e0     flags.obj
 0001:000018f4       ??_C@_0BE@LKEMICNM@OPIF_EXTERNALDELETE?$AA@ 100028f4     flags.obj
 0001:00001908       ??_C@_0BB@CFFPNDFK@OPIF_EXTERNALPUT?$AA@ 10002908     flags.obj
 0001:0000191c       ??_C@_0BB@PELHBPAM@OPIF_EXTERNALGET?$AA@ 1000291c     flags.obj
 0001:00001930       ??_C@_0BE@GJEJHNKJ@OPIF_COMPAREFATTIME?$AA@ 10002930     flags.obj
 0001:00001944       ??_C@_0BG@HGPMKHIE@OPIF_SHOWPRESERVECASE?$AA@ 10002944     flags.obj
 0001:0000195c       ??_C@_0BJ@NMIFAPJD@OPIF_SHOWRIGHTALIGNNAMES?$AA@ 1000295c     flags.obj
 0001:00001978       ??_C@_0BD@FPGMNAPD@OPIF_SHOWNAMESONLY?$AA@ 10002978     flags.obj
 0001:0000198c       ??_C@_0P@OFEDJCO@OPIF_REALNAMES?$AA@ 1000298c     flags.obj
 0001:0000199c       ??_C@_0BC@HOFHNJIG@OPIF_RAWSELECTION?$AA@ 1000299c     flags.obj
 0001:000019b0       ??_C@_0N@JANKJMLP@OPIF_ADDDOTS?$AA@ 100029b0     flags.obj
 0001:000019c0       ??_C@_0BJ@NGLIANCL@OPIF_DISABLEHIGHLIGHTING?$AA@ 100029c0     flags.obj
 0001:000019dc       ??_C@_0BH@FHBKALPD@OPIF_DISABLESORTGROUPS?$AA@ 100029dc     flags.obj
 0001:000019f4       ??_C@_0BD@PBMGDJEM@OPIF_DISABLEFILTER?$AA@ 100029f4     flags.obj
 0001:00001a08       ??_C@_0BH@KOFCBJBO@PMFLAGS_CASECONVERSION?$AA@ 10002a08     flags.obj
 0001:00001a20       ??_C@_0BI@BMHIBDMH@PMFLAGS_ALIGNEXTENSIONS?$AA@ 10002a20     flags.obj
 0001:00001a38       ??_C@_0BH@GDAAKEMH@PMFLAGS_DETAILEDSTATUS?$AA@ 10002a38     flags.obj
 0001:00001a50       ??_C@_0BD@KGHJOBGM@PMFLAGS_FULLSCREEN?$AA@ 10002a50     flags.obj
 0001:00001a64       ??_C@_0BD@EGELEIIG@IPLFLAGS_SEPARATOR?$AA@ 10002a64     flags.obj
 0001:00001a78       ??_C@_07MGEGJMPI@PF_NONE?$AA@ 10002a78     flags.obj
 0001:00001a80       ??_C@_09GMFDAFKL@PF_DIALOG?$AA@ 10002a80     flags.obj
 0001:00001a8c       ??_C@_0P@MBLBBCNK@PF_FULLCMDLINE?$AA@ 10002a8c     flags.obj
 0001:00001a9c       ??_C@_09NEKIJNNA@PF_VIEWER?$AA@ 10002a9c     flags.obj
 0001:00001aa8       ??_C@_09OENCMPGE@PF_EDITOR?$AA@ 10002aa8     flags.obj
 0001:00001ab4       ??_C@_0BB@GCINAIGN@PF_DISABLEPANELS?$AA@ 10002ab4     flags.obj
 0001:00001ac8       ??_C@_0L@NHEJGKCF@PF_PRELOAD?$AA@ 10002ac8     flags.obj
 0001:00001ad4       ??_C@_0BH@PEGBPJKE@FFFS_MINSIZEINDEX_MASK?$AA@ 10002ad4     flags.obj
 0001:00001aec       ??_C@_0BC@LLLANJJO@FFFS_MINSIZEINDEX?$AA@ 10002aec     flags.obj
 0001:00001b00       ??_C@_0O@HFIGPFIH@FFFS_THOUSAND?$AA@ 10002b00     flags.obj
 0001:00001b10       ??_C@_0O@FPIOAIMC@FFFS_ECONOMIC?$AA@ 10002b10     flags.obj
 0001:00001b20       ??_C@_0BE@NPKCCEJ@FFFS_SHOWBYTESINDEX?$AA@ 10002b20     flags.obj
 0001:00001b34       ??_C@_0P@JPMLNBKL@FFFS_FLOATSIZE?$AA@ 10002b34     flags.obj
 0001:00001b44       ??_C@_0M@JDMKDBDH@FFFS_COMMAS?$AA@ 10002b44     flags.obj
 0001:00001b50       ??_C@_08EBKEJHAL@MLF_NONE?$AA@ 10002b50     flags.obj
 0001:00001b5c       ??_C@_0P@EPFBLPAE@MLF_HOLDTARGET?$AA@ 10002b5c     flags.obj
 0001:00001b6c       ??_C@_0BF@LMAGFLHF@MLF_DONOTUPDATEPANEL?$AA@ 10002b6c     flags.obj
 0001:00001b84       ??_C@_0P@LJPBHEIE@MLF_SHOWERRMSG?$AA@ 10002b84     flags.obj
 0001:00001b94       ??_C@_0BA@JCPHOEAE@FRS_SCANSYMLINK?$AA@ 10002b94     flags.obj
 0001:00001ba4       ??_C@_09GHEPLOHO@FRS_RECUR?$AA@ 10002ba4     flags.obj
 0001:00001bb0       ??_C@_0N@PJEDCNNJ@FRS_RETUPDIR?$AA@ 10002bb0     flags.obj
 0001:00001bc0       ??_C@_09JCNLKBBK@XLAT_NONE?$AA@ 10002bc0     flags.obj
 0001:00001bcc       ??_C@_0BH@IANKLOAC@XLAT_CONVERTALLCMDLINE?$AA@ 10002bcc     flags.obj
 0001:00001be4       ??_C@_0BH@KBFAFPNA@XLAT_USEKEYBLAYOUTNAME?$AA@ 10002be4     flags.obj
 0001:00001bfc       ??_C@_0BE@KOIJDNLA@XLAT_SWITCHKEYBBEEP?$AA@ 10002bfc     flags.obj
 0001:00001c10       ??_C@_0BG@GOMJDMCK@XLAT_SWITCHKEYBLAYOUT?$AA@ 10002c10     flags.obj
 0001:00001c28       ??_C@_0BE@OPDBOAAE@PN_SHOWERRORMESSAGE?$AA@ 10002c28     flags.obj
 0001:00001c3c       ??_C@_0M@NOOLKEBH@PN_SKIPPATH?$AA@ 10002c3c     flags.obj
 0001:00001c48       ??_C@_0N@FEGPCCPJ@PN_CHECKMASK?$AA@ 10002c48     flags.obj
 0001:00001c58       ??_C@_0BA@BJCCEIOI@PN_GENERATENAME?$AA@ 10002c58     flags.obj
 0001:00001c68       ??_C@_0P@KDEENAHJ@PN_CMPNAMELIST?$AA@ 10002c68     flags.obj
 0001:00001c78       ??_C@_0L@HODJIPGA@PN_CMPNAME?$AA@ 10002c78     flags.obj
 0001:00001c84       ??_C@_08OIOFCNLC@FPF_NONE?$AA@ 10002c84     flags.obj
 0001:00001c90       ??_C@_08GKECKCCJ@FPF_ANSI?$AA@ 10002c90     flags.obj
 0001:00001c9c       ??_C@_0L@NMBLFMBN@FPF_LOADED?$AA@ 10002c9c     flags.obj
 0001:00001ca8       ??_C@_08HPFOCDKB@FIB_NONE?$AA@ 10002ca8     flags.obj
 0001:00001cb4       ??_C@_0BB@DCODFLEL@FIB_EDITPATHEXEC?$AA@ 10002cb4     flags.obj
 0001:00001cc8       ??_C@_0N@LBOCEEGH@FIB_EDITPATH?$AA@ 10002cc8     flags.obj
 0001:00001cd8       ??_C@_0BA@COBBDHNL@FIB_NOAMPERSAND?$AA@ 10002cd8     flags.obj
 0001:00001ce8       ??_C@_0M@KJOJJDIM@FIB_BUTTONS?$AA@ 10002ce8     flags.obj
 0001:00001cf4       ??_C@_0BF@CEMIHIOK@FIB_NOUSELASTHISTORY?$AA@ 10002cf4     flags.obj
 0001:00001d0c       ??_C@_0O@DOHEGELC@FIB_EXPANDENV?$AA@ 10002d0c     flags.obj
 0001:00001d1c       ??_C@_0N@DLDJCGJI@FIB_PASSWORD?$AA@ 10002d1c     flags.obj
 0001:00001d2c       ??_C@_0BA@KNNLMGCA@FIB_ENABLEEMPTY?$AA@ 10002d2c     flags.obj
 0001:00001d3c       ??_C@_0P@BAFEMBAJ@ECF_AUTODELETE?$AA@ 10002d3c     flags.obj
 0001:00001d4c       ??_C@_0BD@DKGCCJNG@ECF_TABMARKCURRENT?$AA@ 10002d4c     flags.obj
 0001:00001d60       ??_C@_0BB@EDGIEBDF@ECF_TABMARKFIRST?$AA@ 10002d60     flags.obj
 0001:00001d74       ??_C@_0N@GHBDMLON@VMF_WORDWRAP?$AA@ 10002d74     flags.obj
 0001:00001d84       ??_C@_08FAPBJAKB@VMF_WRAP?$AA@ 10002d84     flags.obj
 0001:00001d90       ??_C@_0BA@JKDMJLJG@VSP_NORETNEWPOS?$AA@ 10002d90     flags.obj
 0001:00001da0       ??_C@_0N@JGGGCNIP@VSP_RELATIVE?$AA@ 10002da0     flags.obj
 0001:00001db0       ??_C@_0M@LHNGMHFO@VSP_PERCENT?$AA@ 10002db0     flags.obj
 0001:00001dbc       ??_C@_0N@GHEHKHJN@VSP_NOREDRAW?$AA@ 10002dbc     flags.obj
 0001:00001dcc       ??_C@_0N@ILNDJNNO@VSMFL_REDRAW?$AA@ 10002dcc     flags.obj
 0001:00001ddc       ??_C@_09FIOJMNJ@VOPT_NONE?$AA@ 10002ddc     flags.obj
 0001:00001de8       ??_C@_0BI@NCAHLEBN@VOPT_AUTODETECTCODEPAGE?$AA@ 10002de8     flags.obj
 0001:00001e00       ??_C@_0BG@JMJAOELH@VOPT_SAVEFILEPOSITION?$AA@ 10002e00     flags.obj
 0001:00001e18       ??_C@_09FPGEBDGO@WIF_MODAL?$AA@ 10002e18     flags.obj
 0001:00001e24       ??_C@_0M@ICPAPCOF@WIF_CURRENT?$AA@ 10002e24     flags.obj
 0001:00001e30       ??_C@_0N@MLMCEKPH@WIF_MODIFIED?$AA@ 10002e30     flags.obj
 0001:00001e40       ??_C@_0N@LCOHPDHN@FSETCLR_NONE?$AA@ 10002e40     flags.obj
 0001:00001e50       ??_C@_0P@LMBMJIMF@FSETCLR_REDRAW?$AA@ 10002e50     flags.obj
 0001:00001e60       ??_C@_0O@GKOLBMFK@AKMFLAGS_NONE?$AA@ 10002e60     flags.obj
 0001:00001e70       ??_C@_0N@GIJCDFJI@KMFLAGS_NONE?$AA@ 10002e70     flags.obj
 0001:00001e80       ??_C@_0BD@JHNPMIGP@KMFLAGS_MOONSCRIPT?$AA@ 10002e80     flags.obj
 0001:00001e94       ??_C@_0M@HFBACHCP@KMFLAGS_LUA?$AA@ 10002e94     flags.obj
 0001:00001ea0       ??_C@_0BB@NCECNBPK@KMFLAGS_LANGMASK?$AA@ 10002ea0     flags.obj
 0001:00001eb4       ??_C@_0BF@PHHPAAOK@KMFLAGS_ENABLEOUTPUT?$AA@ 10002eb4     flags.obj
 0001:00001ecc       ??_C@_0BM@BBOPLPKC@KMFLAGS_NOSENDKEYSTOPLUGINS?$AA@ 10002ecc     flags.obj
 0001:00001ee8       ??_C@_0BE@GEGKIINM@KMFLAGS_SILENTCHECK?$AA@ 10002ee8     flags.obj
 0001:00001efc       ??_C@_0L@MAGMKNFN@FHELP_NONE?$AA@ 10002efc     flags.obj
 0001:00001f08       ??_C@_0BC@PNPOIHMG@FHELP_USECONTENTS?$AA@ 10002f08     flags.obj
 0001:00001f1c       ??_C@_0L@OOIMFPBD@FHELP_GUID?$AA@ 10002f1c     flags.obj
 0001:00001f28       ??_C@_0BB@IHFFPJJA@FHELP_CUSTOMPATH?$AA@ 10002f28     flags.obj
 0001:00001f3c       ??_C@_0BB@KNKDPNI@FHELP_CUSTOMFILE?$AA@ 10002f3c     flags.obj
 0001:00001f50       ??_C@_0O@FLGGLFLC@FHELP_FARHELP?$AA@ 10002f50     flags.obj
 0001:00001f60       ??_C@_0P@GANNLHEJ@FHELP_SELFHELP?$AA@ 10002f60     flags.obj
 0001:00001f70       ??_C@_0BC@HHNGCBAM@FHELP_NOSHOWERROR?$AA@ 10002f70     flags.obj
 0001:00001f84       ??_C@_07MBPCONNA@EN_NONE?$AA@ 10002f84     flags.obj
 0001:00001f8c       ??_C@_0BJ@MOLGCBMH@EF_OPENMODE_RELOADIFOPEN?$AA@ 10002f8c     flags.obj
 0001:00001fa8       ??_C@_0BI@EJBKKDJ@EF_OPENMODE_BREAKIFOPEN?$AA@ 10002fa8     flags.obj
 0001:00001fc0       ??_C@_0BI@KGOKGPEI@EF_OPENMODE_USEEXISTING?$AA@ 10002fc0     flags.obj
 0001:00001fd8       ??_C@_0BG@BFKJJBAG@EF_OPENMODE_NEWIFOPEN?$AA@ 10002fd8     flags.obj
 0001:00001ff0       ??_C@_0BC@GAIDEJIA@EF_OPENMODE_QUERY?$AA@ 10002ff0     flags.obj
 0001:00002004       ??_C@_0BB@NILAHAFO@EF_OPENMODE_MASK?$AA@ 10003004     flags.obj
 0001:00002018       ??_C@_0BC@GFHJGKD@EF_DISABLESAVEPOS?$AA@ 10003018     flags.obj
 0001:0000202c       ??_C@_09IJMPFPLB@EF_LOCKED?$AA@ 1000302c     flags.obj
 0001:00002038       ??_C@_0BJ@ILCPOFKL@EF_DELETEONLYFILEONCLOSE?$AA@ 10003038     flags.obj
 0001:00002054       ??_C@_0BD@IHIGHGPL@EF_IMMEDIATERETURN?$AA@ 10003054     flags.obj
 0001:00002068       ??_C@_0BB@KGPIDKFC@EF_DELETEONCLOSE?$AA@ 10003068     flags.obj
 0001:0000207c       ??_C@_0BC@PPEPEFFI@EF_DISABLEHISTORY?$AA@ 1000307c     flags.obj
 0001:00002090       ??_C@_0N@LKLNHALI@EF_ENABLE_F6?$AA@ 10003090     flags.obj
 0001:000020a0       ??_C@_0N@DBHFPBEO@EF_CREATENEW?$AA@ 100030a0     flags.obj
 0001:000020b0       ??_C@_0M@PIFGAPFH@EF_NONMODAL?$AA@ 100030b0     flags.obj
 0001:000020bc       ??_C@_07CJJFHP@VF_NONE?$AA@ 100030bc     flags.obj
 0001:000020c4       ??_C@_0BJ@OGNFHEJG@VF_DELETEONLYFILEONCLOSE?$AA@ 100030c4     flags.obj
 0001:000020e0       ??_C@_0BD@DHJCMLFI@VF_IMMEDIATERETURN?$AA@ 100030e0     flags.obj
 0001:000020f4       ??_C@_0BC@DLGKMECC@VF_DISABLEHISTORY?$AA@ 100030f4     flags.obj
 0001:00002108       ??_C@_0N@LDHALKKM@VF_ENABLE_F6?$AA@ 10003108     flags.obj
 0001:00002118       ??_C@_0BB@OCDDPIKL@VF_DELETEONCLOSE?$AA@ 10003118     flags.obj
 0001:0000212c       ??_C@_0M@IDNADAFL@VF_NONMODAL?$AA@ 1000312c     flags.obj
 0001:00002138       ??_C@_0M@NEMAHHGP@PFLAGS_NONE?$AA@ 10003138     flags.obj
 0001:00002144       ??_C@_0BA@GHMDCHHI@PFLAGS_SHORTCUT?$AA@ 10003144     flags.obj
 0001:00002154       ??_C@_0BI@EOCCAHFA@PFLAGS_ALTERNATIVENAMES?$AA@ 10003154     flags.obj
 0001:0000216c       ??_C@_0N@EOFAELOJ@PFLAGS_FOCUS?$AA@ 1000316c     flags.obj
 0001:0000217c       ??_C@_0P@MLDEBNPK@PFLAGS_VISIBLE?$AA@ 1000317c     flags.obj
 0001:0000218c       ??_C@_0O@DBPJGING@PFLAGS_PLUGIN?$AA@ 1000318c     flags.obj
 0001:0000219c       ??_C@_0BJ@HJFOABKG@PFLAGS_CASESENSITIVESORT?$AA@ 1000319c     flags.obj
 0001:000021b8       ??_C@_0BA@KJEPHDOM@PFLAGS_USECRC32?$AA@ 100031b8     flags.obj
 0001:000021c8       ??_C@_0BI@EHHAJLOH@PFLAGS_DIRECTORIESFIRST?$AA@ 100031c8     flags.obj
 0001:000021e0       ??_C@_0BB@ILEHDKFJ@PFLAGS_PANELLEFT?$AA@ 100031e0     flags.obj
 0001:000021f4       ??_C@_0BD@MOODMDAB@PFLAGS_NUMERICSORT?$AA@ 100031f4     flags.obj
 0001:00002208       ??_C@_0BB@KDANIJNM@PFLAGS_REALNAMES?$AA@ 10003208     flags.obj
 0001:0000221c       ??_C@_0BF@LBBAIOCD@PFLAGS_SELECTEDFIRST?$AA@ 1000321c     flags.obj
 0001:00002234       ??_C@_0BF@KJNCJPKN@PFLAGS_USESORTGROUPS?$AA@ 10003234     flags.obj
 0001:0000224c       ??_C@_0BI@BFAFODJ@PFLAGS_REVERSESORTORDER?$AA@ 1000324c     flags.obj
 0001:00002264       ??_C@_0BB@BCAJEJEH@PFLAGS_HIGHLIGHT?$AA@ 10003264     flags.obj
 0001:00002278       ??_C@_0BC@BONLDOOD@PFLAGS_SHOWHIDDEN?$AA@ 10003278     flags.obj
 0001:0000228c       ??_C@_09OIFMMGNJ@PPIF_NONE?$AA@ 1000328c     flags.obj
 0001:00002298       ??_C@_0BC@LPBDBIOM@PPIF_PROCESSDESCR?$AA@ 10003298     flags.obj
 0001:000022ac       ??_C@_0O@JEAJLDHC@PPIF_SELECTED?$AA@ 100032ac     flags.obj
 0001:000022bc       ??_C@_0L@DGFIEOMD@FMENU_NONE?$AA@ 100032bc     flags.obj
 0001:000022c8       ??_C@_0BJ@FCEONOJC@FMENU_CHANGECONSOLETITLE?$AA@ 100032c8     flags.obj
 0001:000022e4       ??_C@_0BL@OKAIKPMN@FMENU_REVERSEAUTOHIGHLIGHT?$AA@ 100032e4     flags.obj
 0001:00002300       ??_C@_0BE@IDAMFDEA@FMENU_AUTOHIGHLIGHT?$AA@ 10003300     flags.obj
 0001:00002314       ??_C@_0P@HICDNKDJ@FMENU_WRAPMODE?$AA@ 10003314     flags.obj
 0001:00002324       ??_C@_0BE@FALMPPJK@FMENU_SHOWAMPERSAND?$AA@ 10003324     flags.obj
 0001:00002338       ??_C@_08JEEJJGP@MIF_NONE?$AA@ 10003338     flags.obj
 0001:00002344       ??_C@_0L@DEJINBIP@MIF_HIDDEN?$AA@ 10003344     flags.obj
 0001:00002350       ??_C@_0L@DLLNLLIG@MIF_GRAYED?$AA@ 10003350     flags.obj
 0001:0000235c       ??_C@_0M@OPPCPJOL@MIF_DISABLE?$AA@ 1000335c     flags.obj
 0001:00002368       ??_C@_0O@DEIKOCPA@MIF_SEPARATOR?$AA@ 10003368     flags.obj
 0001:00002378       ??_C@_0M@IHMNAMOE@MIF_CHECKED?$AA@ 10003378     flags.obj
 0001:00002384       ??_C@_0N@JOOGIBAO@MIF_SELECTED?$AA@ 10003384     flags.obj
 0001:00002394       ??_C@_09NNFHCBNL@FDLG_NONE?$AA@ 10003394     flags.obj
 0001:000023a0       ??_C@_0BG@GHNOOENB@FDLG_KEEPCONSOLETITLE?$AA@ 100033a0     flags.obj
 0001:000023b8       ??_C@_0BB@NPLEEAKK@FDLG_NODRAWPANEL?$AA@ 100033b8     flags.obj
 0001:000023cc       ??_C@_0BC@ONGLDAJN@FDLG_NODRAWSHADOW?$AA@ 100033cc     flags.obj
 0001:000023e0       ??_C@_0BB@DKMEBDJJ@FDLG_SMALLDIALOG?$AA@ 100033e0     flags.obj
 0001:000023f4       ??_C@_0N@OLGDMHKL@FDLG_WARNING?$AA@ 100033f4     flags.obj
 0001:00002404       ??_C@_0L@EPACPANF@LINFO_NONE?$AA@ 10003404     flags.obj
 0001:00002410       ??_C@_0BE@OHJCOKAE@LINFO_SHOWAMPERSAND?$AA@ 10003410     flags.obj
 0001:00002424       ??_C@_0P@KLBMHNCG@LINFO_WRAPMODE?$AA@ 10003424     flags.obj
 0001:00002434       ??_C@_0BH@BADLEILJ@LINFO_REVERSEHIGHLIGHT?$AA@ 10003434     flags.obj
 0001:0000244c       ??_C@_0BE@DECCEGNO@LINFO_AUTOHIGHLIGHT?$AA@ 1000344c     flags.obj
 0001:00002460       ??_C@_0BA@OOIEKCFB@LINFO_SHOWNOBOX?$AA@ 10003460     flags.obj
 0001:00002470       ??_C@_0M@FPOGKIGO@LIFIND_NONE?$AA@ 10003470     flags.obj
 0001:0000247c       ??_C@_0BC@BGAENNBJ@LIFIND_EXACTMATCH?$AA@ 1000347c     flags.obj
 0001:00002490       ??_C@_08BODPINCM@LIF_NONE?$AA@ 10003490     flags.obj
 0001:0000249c       ??_C@_0BD@HEPCOIEH@LIF_DELETEUSERDATA?$AA@ 1000349c     flags.obj
 0001:000024b0       ??_C@_0L@PFBGAOEP@LIF_HIDDEN?$AA@ 100034b0     flags.obj
 0001:000024bc       ??_C@_0L@PKDDGEEG@LIF_GRAYED?$AA@ 100034bc     flags.obj
 0001:000024c8       ??_C@_0M@HEFHLFIE@LIF_DISABLE?$AA@ 100034c8     flags.obj
 0001:000024d4       ??_C@_0O@KJIFADIG@LIF_SEPARATOR?$AA@ 100034d4     flags.obj
 0001:000024e4       ??_C@_0M@BMGIEAIL@LIF_CHECKED?$AA@ 100034e4     flags.obj
 0001:000024f0       ??_C@_0N@EDHAFIIL@LIF_SELECTED?$AA@ 100034f0     flags.obj
 0001:00002500       ??_C@_08KFOHCPDE@DIF_NONE?$AA@ 10003500     flags.obj
 0001:0000250c       ??_C@_0N@LAEOODAD@DIF_WORDWRAP?$AA@ 1000350c     flags.obj
 0001:0000251c       ??_C@_0O@KJADCBBN@DIF_RIGHTTEXT?$AA@ 1000351c     flags.obj
 0001:0000252c       ??_C@_09LCJIOEMN@DIF_FOCUS?$AA@ 1000352c     flags.obj
 0001:00002538       ??_C@_0BC@CHAAKEJO@DIF_DEFAULTBUTTON?$AA@ 10003538     flags.obj
 0001:0000254c       ??_C@_0M@HCFLMDHK@DIF_DISABLE?$AA@ 1000354c     flags.obj
 0001:00002558       ??_C@_0M@NLLDINIM@DIF_NOFOCUS?$AA@ 10003558     flags.obj
 0001:00002564       ??_C@_0N@KOGKCAKJ@DIF_READONLY?$AA@ 10003564     flags.obj
 0001:00002574       ??_C@_0L@EPNFOPAK@DIF_HIDDEN?$AA@ 10003574     flags.obj
 0001:00002580       ??_C@_0BB@GMKDKOOP@DIF_EDITPATHEXEC?$AA@ 10003580     flags.obj
 0001:00002594       ??_C@_0BA@JNOKLHOL@DIF_LISTNOCLOSE?$AA@ 10003594     flags.obj
 0001:000025a4       ??_C@_0BG@MONEJILE@DIF_LISTAUTOHIGHLIGHT?$AA@ 100035a4     flags.obj
 0001:000025bc       ??_C@_0BD@MFOKKGGF@DIF_NOAUTOCOMPLETE?$AA@ 100035bc     flags.obj
 0001:000025d0       ??_C@_0BB@NPNALIGO@DIF_LISTWRAPMODE?$AA@ 100035d0     flags.obj
 0001:000025e4       ??_C@_0N@GBGHICKO@DIF_EDITPATH?$AA@ 100035e4     flags.obj
 0001:000025f4       ??_C@_0L@KKNJDNBK@DIF_3STATE?$AA@ 100035f4     flags.obj
 0001:00002600       ??_C@_0BC@JNLDMGBD@DIF_SELECTONENTRY?$AA@ 10003600     flags.obj
 0001:00002614       ??_C@_0BK@LEFIBDOA@DIF_LISTTRACKMOUSEINFOCUS?$AA@ 10003614     flags.obj
 0001:00002630       ??_C@_0BD@LPDHCLJI@DIF_LISTTRACKMOUSE?$AA@ 10003630     flags.obj
 0001:00002644       ??_C@_0N@MOCGNIKC@DIF_MASKEDIT?$AA@ 10003644     flags.obj
 0001:00002654       ??_C@_0BD@MNGIOLFF@DIF_USELASTHISTORY?$AA@ 10003654     flags.obj
 0001:00002668       ??_C@_0BB@EIMEKEFP@DIF_DROPDOWNLIST?$AA@ 10003668     flags.obj
 0001:0000267c       ??_C@_0P@EEJEDBLH@DIF_EDITEXPAND?$AA@ 1000367c     flags.obj
 0001:0000268c       ??_C@_0O@IKJBMPOF@DIF_SETSHIELD?$AA@ 1000368c     flags.obj
 0001:0000269c       ??_C@_0BC@ODEMBOPK@DIF_SEPARATORUSER?$AA@ 1000369c     flags.obj
 0001:000026b0       ??_C@_0P@KOJCCCGB@DIF_CENTERTEXT?$AA@ 100036b0     flags.obj
 0001:000026c0       ??_C@_0P@EGFAEEDC@DIF_BTNNOCLOSE?$AA@ 100036c0     flags.obj
 0001:000026d0       ??_C@_0M@IPFBMFDN@DIF_HISTORY?$AA@ 100036d0     flags.obj
 0001:000026dc       ??_C@_0O@FFJNBMAD@DIF_LISTNOBOX?$AA@ 100036dc     flags.obj
 0001:000026ec       ??_C@_0BE@PFICAGJF@DIF_LISTNOAMPERSAND?$AA@ 100036ec     flags.obj
 0001:00002700       ??_C@_0L@NBPFNGLB@DIF_EDITOR?$AA@ 10003700     flags.obj
 0001:0000270c       ??_C@_0P@CGILDLOA@DIF_SEPARATOR2?$AA@ 1000370c     flags.obj
 0001:0000271c       ??_C@_0O@JKNMBNLA@DIF_SEPARATOR?$AA@ 1000371c     flags.obj
 0001:0000272c       ??_C@_0BF@JBCDBJCL@DIF_MANUALADDHISTORY?$AA@ 1000372c     flags.obj
 0001:00002744       ??_C@_0P@MKFBJPOB@DIF_NOBRACKETS?$AA@ 10003744     flags.obj
 0001:00002754       ??_C@_0BA@BLCOKAAO@DIF_CENTERGROUP?$AA@ 10003754     flags.obj
 0001:00002764       ??_C@_0BC@PDKFKKEI@DIF_SHOWAMPERSAND?$AA@ 10003764     flags.obj
 0001:00002778       ??_C@_0P@BGPBEDHH@DIF_MOVESELECT?$AA@ 10003778     flags.obj
 0001:00002788       ??_C@_0N@GCKJNBCM@DIF_LEFTTEXT?$AA@ 10003788     flags.obj
 0001:00002798       ??_C@_09IAEPIICA@DIF_GROUP?$AA@ 10003798     flags.obj
 0001:000027a4       ??_C@_0N@DHJCDIKM@DIF_BOXCOLOR?$AA@ 100037a4     flags.obj
 0001:000027b4       ??_C@_09NEGPLEAH@FMSG_NONE?$AA@ 100037b4     flags.obj
 0001:000027c0       ??_C@_0BE@OCLAIENB@FMSG_MB_RETRYCANCEL?$AA@ 100037c0     flags.obj
 0001:000027d4       ??_C@_0BE@IBNOLCGP@FMSG_MB_YESNOCANCEL?$AA@ 100037d4     flags.obj
 0001:000027e8       ??_C@_0O@GPCAPHCL@FMSG_MB_YESNO?$AA@ 100037e8     flags.obj
 0001:000027f8       ??_C@_0BJ@BKJADAHA@FMSG_MB_ABORTRETRYIGNORE?$AA@ 100037f8     flags.obj
 0001:00002814       ??_C@_0BB@JGAPGIEP@FMSG_MB_OKCANCEL?$AA@ 10003814     flags.obj
 0001:00002828       ??_C@_0L@BGALGPOK@FMSG_MB_OK?$AA@ 10003828     flags.obj
 0001:00002834       ??_C@_0O@FOIOKDHJ@FMSG_ALLINONE?$AA@ 10003834     flags.obj
 0001:00002844       ??_C@_0P@KBEMNNEP@FMSG_LEFTALIGN?$AA@ 10003844     flags.obj
 0001:00002854       ??_C@_0BE@FHOOILPH@FMSG_KEEPBACKGROUND?$AA@ 10003854     flags.obj
 0001:00002868       ??_C@_0P@HHIGLJAP@FMSG_ERRORTYPE?$AA@ 10003868     flags.obj
 0001:00002878       ??_C@_0N@ELMEMNDH@FMSG_WARNING?$AA@ 10003878     flags.obj
 0001:00002888       ??_C@_08FKIDFHCM@CDF_NONE?$AA@ 10003888     flags.obj
 0001:00002894       ??_C@_08BKNBBLHK@FCF_NONE?$AA@ 10003894     flags.obj
 0001:000028a0       ??_C@_0O@LGBGBIGB@FCF_STYLEMASK?$AA@ 100038a0     flags.obj
 0001:000028b0       ??_C@_0BB@NPEFGEGA@FCF_FG_UNDERLINE?$AA@ 100038b0     flags.obj
 0001:000028c4       ??_C@_0O@FAPDECBF@FCF_FG_ITALIC?$AA@ 100038c4     flags.obj
 0001:000028d4       ??_C@_0M@LFMGCKHG@FCF_FG_BOLD?$AA@ 100038d4     flags.obj
 0001:000028e0       ??_C@_0BC@NKBLNNIA@FCF_EXTENDEDFLAGS?$AA@ 100038e0     flags.obj
 0001:000028f4       ??_C@_0BB@PJFLJJLD@FCF_RAWATTR_MASK?$AA@ 100038f4     flags.obj
 0001:00002908       ??_C@_0N@HMKJBHOA@FCF_4BITMASK?$AA@ 10003908     flags.obj
 0001:00002918       ??_C@_0M@PJHNDJIE@FCF_BG_4BIT?$AA@ 10003918     flags.obj
 0001:00002924       ??_C@_0M@HNDHDHHO@FCF_FG_4BIT?$AA@ 10003924     flags.obj
 0001:00002930       ??_C@_0BE@PONEECEM@FE_CHANGESORTPARAMS?$AA@ 10003930     flags.obj
 0001:00002944       ??_C@_0N@DGHFKMFL@FE_KILLFOCUS?$AA@ 10003944     flags.obj
 0001:00002954       ??_C@_0M@FIECADDF@FE_GOTFOCUS?$AA@ 10003954     flags.obj
 0001:00002960       ??_C@_0L@LELAIPLL@FE_COMMAND?$AA@ 10003960     flags.obj
 0001:0000296c       ??_C@_08MOMCCKPB@FE_BREAK?$AA@ 1000396c     flags.obj
 0001:00002978       ??_C@_08DENCGKED@FE_CLOSE?$AA@ 10003978     flags.obj
 0001:00002984       ??_C@_07CLNPDBLG@FE_IDLE?$AA@ 10003984     flags.obj
 0001:0000298c       ??_C@_09DENIDBMJ@FE_REDRAW?$AA@ 1000398c     flags.obj
 0001:00002998       ??_C@_0BC@PNCKAHJO@FE_CHANGEVIEWMODE?$AA@ 10003998     flags.obj
 0001:000029ac       ??_C@_0BA@GEAFHJNF@MPRT_HASNOMACRO?$AA@ 100039ac     flags.obj
 0001:000029bc       ??_C@_0O@IEMNLPAB@MPRT_USERMENU?$AA@ 100039bc     flags.obj
 0001:000029cc       ??_C@_0BD@HHINMPPI@MPRT_PLUGINCOMMAND?$AA@ 100039cc     flags.obj
 0001:000029e0       ??_C@_0BC@LEDOPMKI@MPRT_PLUGINCONFIG?$AA@ 100039e0     flags.obj
 0001:000029f4       ??_C@_0BA@EJFFOAMM@MPRT_PLUGINMENU?$AA@ 100039f4     flags.obj
 0001:00002a04       ??_C@_0BA@OBIDLEIM@MPRT_PLUGINCALL?$AA@ 10003a04     flags.obj
 0001:00002a14       ??_C@_0L@GEHHCKFA@MPRT_PRINT?$AA@ 10003a14     flags.obj
 0001:00002a20       ??_C@_09EJDAADCN@MPRT_KEYS?$AA@ 10003a20     flags.obj
 0001:00002a2c       ??_C@_0BA@BCBAEEOI@MPRT_ERRORPARSE?$AA@ 10003a2c     flags.obj
 0001:00002a3c       ??_C@_0BB@PMCBIGCA@MPRT_ERRORFINISH?$AA@ 10003a3c     flags.obj
 0001:00002a50       ??_C@_0BC@IOECJI@MPRT_NORMALFINISH?$AA@ 10003a50     flags.obj
 0001:00002a64       ??_C@_0N@BHFJFHA@MCT_KEYMACRO?$AA@ 10003a64     flags.obj
 0001:00002a74       ??_C@_0N@FOPIOCHO@MCT_ADDMACRO?$AA@ 10003a74     flags.obj
 0001:00002a84       ??_C@_0BH@PKKJIOHM@MCT_GETCUSTOMSORTMODES?$AA@ 10003a84     flags.obj
 0001:00002a9c       ??_C@_0O@CDBDPKIC@MCT_PANELSORT?$AA@ 10003a9c     flags.obj
 0001:00002aac       ??_C@_0P@HOMHAEFB@MCT_EXECSTRING?$AA@ 10003aac     flags.obj
 0001:00002abc       ??_C@_0BC@NALHIHJ@MCT_RUNSTARTMACRO?$AA@ 10003abc     flags.obj
 0001:00002ad0       ??_C@_0N@OLCKOJMI@MCT_DELMACRO?$AA@ 10003ad0     flags.obj
 0001:00002ae0       ??_C@_0BC@NFGGBILF@MCT_RECORDEDMACRO?$AA@ 10003ae0     flags.obj
 0001:00002af4       ??_C@_0N@IGJGAHKE@MCT_GETMACRO?$AA@ 10003af4     flags.obj
 0001:00002b04       ??_C@_0BA@MOCJHMJK@MCT_WRITEMACROS?$AA@ 10003b04     flags.obj
 0001:00002b14       ??_C@_0P@HMDDACMI@MCT_ENUMMACROS?$AA@ 10003b14     flags.obj
 0001:00002b24       ??_C@_0P@GNPFPCF@MCT_LOADMACROS?$AA@ 10003b24     flags.obj
 0001:00002b34       ??_C@_0P@GBMLNMMI@MCT_MACROPARSE?$AA@ 10003b34     flags.obj
 0001:00002b44       ??_C@_0O@NEDDJIHC@OPEN_LUAMACRO?$AA@ 10003b44     flags.obj
 0001:00002b54       ??_C@_0P@FOKOAMLC@OPEN_FROMMACRO?$AA@ 10003b54     flags.obj
 0001:00002b64       ??_C@_0BD@NFNGGFHI@OPEN_RIGHTDISKMENU?$AA@ 10003b64     flags.obj
 0001:00002b78       ??_C@_0N@CBHPGAKB@OPEN_ANALYSE?$AA@ 10003b78     flags.obj
 0001:00002b88       ??_C@_0M@LEBKLGKD@OPEN_DIALOG?$AA@ 10003b88     flags.obj
 0001:00002b94       ??_C@_0P@LCDNLGDE@OPEN_FILEPANEL?$AA@ 10003b94     flags.obj
 0001:00002ba4       ??_C@_0M@MOBCONI@OPEN_VIEWER?$AA@ 10003ba4     flags.obj
 0001:00002bb0       ??_C@_0M@DMJLHMGM@OPEN_EDITOR?$AA@ 10003bb0     flags.obj
 0001:00002bbc       ??_C@_0BB@JHCCMIPF@OPEN_COMMANDLINE?$AA@ 10003bbc     flags.obj
 0001:00002bd0       ??_C@_0O@OGDCDPNG@OPEN_SHORTCUT?$AA@ 10003bd0     flags.obj
 0001:00002be0       ??_C@_0O@IEJHJCNB@OPEN_FINDLIST?$AA@ 10003be0     flags.obj
 0001:00002bf0       ??_C@_0BB@CEFDHHLF@OPEN_PLUGINSMENU?$AA@ 10003bf0     flags.obj
 0001:00002c04       ??_C@_0BC@OOKLINPG@OPEN_LEFTDISKMENU?$AA@ 10003c04     flags.obj
 0001:00002c18       ??_C@_05MMFLPJEB@VS_RC?$AA@ 10003c18     flags.obj
 0001:00002c20       ??_C@_07OKFPMINB@VS_BETA?$AA@ 10003c20     flags.obj
 0001:00002c28       ??_C@_08BDGLHPMJ@VS_ALPHA?$AA@ 10003c28     flags.obj
 0001:00002c34       ??_C@_0L@NCFOENCC@VS_RELEASE?$AA@ 10003c34     flags.obj
 0001:00002c40       ??_C@_0L@NPJNPCJM@CPM_NATIVE?$AA@ 10003c40     flags.obj
 0001:00002c4c       ??_C@_08LAEGFKJE@CPM_REAL?$AA@ 10003c4c     flags.obj
 0001:00002c58       ??_C@_08HNOHKPBK@CPM_FULL?$AA@ 10003c58     flags.obj
 0001:00002c64       ??_C@_0N@PJENIJFN@LINK_SYMLINK?$AA@ 10003c64     flags.obj
 0001:00002c74       ??_C@_0BA@GFPIOFMG@LINK_SYMLINKDIR?$AA@ 10003c74     flags.obj
 0001:00002c84       ??_C@_0BB@JDBEPJDK@LINK_SYMLINKFILE?$AA@ 10003c84     flags.obj
 0001:00002c98       ??_C@_0O@FIAPLKLH@LINK_VOLMOUNT?$AA@ 10003c98     flags.obj
 0001:00002ca8       ??_C@_0O@OOAFIIDA@LINK_JUNCTION?$AA@ 10003ca8     flags.obj
 0001:00002cb8       ??_C@_0O@KJFMBLFE@LINK_HARDLINK?$AA@ 10003cb8     flags.obj
 0001:00002cc8       ??_C@_0L@IADFDBJB@FCT_COLUMN?$AA@ 10003cc8     flags.obj
 0001:00002cd4       ??_C@_0L@CDAEILNM@FCT_STREAM?$AA@ 10003cd4     flags.obj
 0001:00002ce0       ??_C@_07BPEFOPGM@FCT_ANY?$AA@ 10003ce0     flags.obj
 0001:00002ce8       ??_C@_09EDBNDHCM@PSL_LOCAL?$AA@ 10003ce8     flags.obj
 0001:00002cf4       ??_C@_0M@JCGHGLJF@PSL_ROAMING?$AA@ 10003cf4     flags.obj
 0001:00002d00       ??_C@_0BB@GBBEBNKE@FSSF_PANELLAYOUT?$AA@ 10003d00     flags.obj
 0001:00002d14       ??_C@_0P@OCDADNBF@FSSF_INTERFACE?$AA@ 10003d14     flags.obj
 0001:00002d24       ??_C@_0M@CBDJLJIE@FSSF_DIALOG?$AA@ 10003d24     flags.obj
 0001:00002d30       ??_C@_0M@KEMGKEOF@FSSF_SCREEN?$AA@ 10003d30     flags.obj
 0001:00002d3c       ??_C@_0M@KJLIHDEL@FSSF_EDITOR?$AA@ 10003d3c     flags.obj
 0001:00002d48       ??_C@_0L@LBFNJGFB@FSSF_PANEL?$AA@ 10003d48     flags.obj
 0001:00002d54       ??_C@_0M@PIGDMPJB@FSSF_SYSTEM?$AA@ 10003d54     flags.obj
 0001:00002d60       ??_C@_0BD@PBIEGEHP@FSSF_CONFIRMATIONS?$AA@ 10003d60     flags.obj
 0001:00002d74       ??_C@_0BG@OHMIIBBD@FSSF_FOLDERSHORTCUT_9?$AA@ 10003d74     flags.obj
 0001:00002d8c       ??_C@_0BG@PONDLAFC@FSSF_FOLDERSHORTCUT_8?$AA@ 10003d8c     flags.obj
 0001:00002da4       ??_C@_0BG@HJELKMJN@FSSF_FOLDERSHORTCUT_7?$AA@ 10003da4     flags.obj
 0001:00002dbc       ??_C@_0BG@GAFAJNNM@FSSF_FOLDERSHORTCUT_6?$AA@ 10003dbc     flags.obj
 0001:00002dd4       ??_C@_0BG@ELHNMOBP@FSSF_FOLDERSHORTCUT_5?$AA@ 10003dd4     flags.obj
 0001:00002dec       ??_C@_0BG@FCGGPPFO@FSSF_FOLDERSHORTCUT_4?$AA@ 10003dec     flags.obj
 0001:00002e04       ??_C@_0BG@BNCHGJJJ@FSSF_FOLDERSHORTCUT_3?$AA@ 10003e04     flags.obj
 0001:00002e1c       ??_C@_0BG@EDMFINI@FSSF_FOLDERSHORTCUT_2?$AA@ 10003e1c     flags.obj
 0001:00002e34       ??_C@_0BG@CPBBALBL@FSSF_FOLDERSHORTCUT_1?$AA@ 10003e34     flags.obj
 0001:00002e4c       ??_C@_0BG@DGAKDKFK@FSSF_FOLDERSHORTCUT_0?$AA@ 10003e4c     flags.obj
 0001:00002e64       ??_C@_0BG@IFGEMJIF@FSSF_HISTORY_EXTERNAL?$AA@ 10003e64     flags.obj
 0001:00002e7c       ??_C@_0BC@CODELNPP@FSSF_HISTORY_EDIT?$AA@ 10003e7c     flags.obj
 0001:00002e90       ??_C@_0BC@NJCJCCNH@FSSF_HISTORY_VIEW?$AA@ 10003e90     flags.obj
 0001:00002ea4       ??_C@_0BE@BLPOFODL@FSSF_HISTORY_FOLDER?$AA@ 10003ea4     flags.obj
 0001:00002eb8       ??_C@_0BB@HDKCPBIO@FSSF_HISTORY_CMD?$AA@ 10003eb8     flags.obj
 0001:00002ecc       ??_C@_09OBBBBFPE@FSSF_ROOT?$AA@ 10003ecc     flags.obj
 0001:00002ed8       ??_C@_08EJJJCLIG@FST_DATA?$AA@ 10003ed8     flags.obj
 0001:00002ee4       ??_C@_0L@LPMPBKDL@FST_STRING?$AA@ 10003ee4     flags.obj
 0001:00002ef0       ??_C@_09LFEEAJIC@FST_QWORD?$AA@ 10003ef0     flags.obj
 0001:00002efc       ??_C@_0L@GGGOEGKJ@FST_SUBKEY?$AA@ 10003efc     flags.obj
 0001:00002f08       ??_C@_0M@OIOMMFOE@FST_UNKNOWN?$AA@ 10003f08     flags.obj
 0001:00002f14       ??_C@_0L@LGPEDLLD@FFT_CUSTOM?$AA@ 10003f14     flags.obj
 0001:00002f20       ??_C@_0L@EKPDMFDD@FFT_SELECT?$AA@ 10003f20     flags.obj
 0001:00002f2c       ??_C@_08KKCPIPGP@FFT_COPY?$AA@ 10003f2c     flags.obj
 0001:00002f38       ??_C@_0N@GMEDAGNH@FFT_FINDFILE?$AA@ 10003f38     flags.obj
 0001:00002f48       ??_C@_09BOODOHKD@FFT_PANEL?$AA@ 10003f48     flags.obj
 0001:00002f54       ??_C@_0P@KKEMMPNI@PFM_MODULENAME?$AA@ 10003f54     flags.obj
 0001:00002f64       ??_C@_08KBAMIIFB@PFM_GUID?$AA@ 10003f64     flags.obj
 0001:00002f70       ??_C@_08HHHKLJPB@PLT_PATH?$AA@ 10003f70     flags.obj
 0001:00002f7c       ??_C@_0P@NMOJJPOB@ECTYPE_DELETED?$AA@ 10003f7c     flags.obj
 0001:00002f8c       ??_C@_0N@MDEFMEEA@ECTYPE_ADDED?$AA@ 10003f8c     flags.obj
 0001:00002f9c       ??_C@_0P@DOBJCNIG@ECTYPE_CHANGED?$AA@ 10003f9c     flags.obj
 0001:00002fac       ??_C@_0P@BECIAJAM@ECSTATE_LOCKED?$AA@ 10003fac     flags.obj
 0001:00002fbc       ??_C@_0O@GBBGHDFM@ECSTATE_SAVED?$AA@ 10003fbc     flags.obj
 0001:00002fcc       ??_C@_0BB@BNPDAPGB@ECSTATE_MODIFIED?$AA@ 10003fcc     flags.obj
 0001:00002fe0       ??_C@_0N@EMEGNPLI@BTYPE_COLUMN?$AA@ 10003fe0     flags.obj
 0001:00002ff0       ??_C@_0N@OPHHGFPF@BTYPE_STREAM?$AA@ 10003ff0     flags.obj
 0001:00003000       ??_C@_0L@BJCBJJNB@BTYPE_NONE?$AA@ 10004000     flags.obj
 0001:0000300c       ??_C@_0BD@CLLAKGOA@EOPT_SHOWLINEBREAK?$AA@ 1000400c     flags.obj
 0001:00003020       ??_C@_08HMMLONBH@EOPT_BOM?$AA@ 10004020     flags.obj
 0001:0000302c       ??_C@_0BE@DDKCDJDC@EOPT_SHOWWHITESPACE?$AA@ 1000402c     flags.obj
 0001:00003040       ??_C@_0BH@CJPAGGLC@EOPT_EXPANDONLYNEWTABS?$AA@ 10004040     flags.obj
 0001:00003058       ??_C@_0BF@IMCOEIAL@EOPT_CURSORBEYONDEOL?$AA@ 10004058     flags.obj
 0001:00003070       ??_C@_0BI@PFHCGCAI@EOPT_AUTODETECTCODEPAGE?$AA@ 10004070     flags.obj
 0001:00003088       ??_C@_0BG@MBPADLG@EOPT_SAVEFILEPOSITION?$AA@ 10004088     flags.obj
 0001:000030a0       ??_C@_0BA@KPJEAKBD@EOPT_AUTOINDENT?$AA@ 100040a0     flags.obj
 0001:000030b0       ??_C@_0BG@PIIHHCAN@EOPT_DELREMOVESBLOCKS?$AA@ 100040b0     flags.obj
 0001:000030c8       ??_C@_0BG@BOINMDEK@EOPT_PERSISTENTBLOCKS?$AA@ 100040c8     flags.obj
 0001:000030e0       ??_C@_0BD@DKHPEOHH@EOPT_EXPANDALLTABS?$AA@ 100040e0     flags.obj
 0001:000030f4       ??_C@_0P@OONGIIBL@EXPAND_NEWTABS?$AA@ 100040f4     flags.obj
 0001:00003104       ??_C@_0P@MLHPCNDM@EXPAND_ALLTABS?$AA@ 10004104     flags.obj
 0001:00003114       ??_C@_0O@PKOIFEBO@EXPAND_NOTABS?$AA@ 10004114     flags.obj
 0001:00003124       ??_C@_08DHMMFAHF@EUR_REDO?$AA@ 10004124     flags.obj
 0001:00003130       ??_C@_08FCONALGE@EUR_UNDO?$AA@ 10004130     flags.obj
 0001:0000313c       ??_C@_07DDJDFJCN@EUR_END?$AA@ 1000413c     flags.obj
 0001:00003144       ??_C@_09FLEMPKKP@EUR_BEGIN?$AA@ 10004144     flags.obj
 0001:00003150       ??_C@_0M@FICNFPPA@ESPT_SETBOM?$AA@ 10004150     flags.obj
 0001:0000315c       ??_C@_0BE@MACJBCFP@ESPT_SHOWWHITESPACE?$AA@ 1000415c     flags.obj
 0001:00003170       ??_C@_0BA@FGEHLJDF@ESPT_GETWORDDIV?$AA@ 10004170     flags.obj
 0001:00003180       ??_C@_0BA@EIGIAOHM@ESPT_SETWORDDIV?$AA@ 10004180     flags.obj
 0001:00003190       ??_C@_0O@KCPDJCKC@ESPT_LOCKMODE?$AA@ 10004190     flags.obj
 0001:000031a0       ??_C@_0BG@HAPABMJH@ESPT_SAVEFILEPOSITION?$AA@ 100041a0     flags.obj
 0001:000031b8       ??_C@_0O@PIAOJINE@ESPT_CODEPAGE?$AA@ 100041b8     flags.obj
 0001:000031c8       ??_C@_0BC@OECOCGLJ@ESPT_CHARCODEBASE?$AA@ 100041c8     flags.obj
 0001:000031dc       ??_C@_0BF@LPNONOMF@ESPT_CURSORBEYONDEOL?$AA@ 100041dc     flags.obj
 0001:000031f4       ??_C@_0BA@KOADDMLI@ESPT_AUTOINDENT?$AA@ 100041f4     flags.obj
 0001:00003204       ??_C@_0BA@GOKHPFCK@ESPT_EXPANDTABS?$AA@ 10004204     flags.obj
 0001:00003214       ??_C@_0N@HKGMPMJE@ESPT_TABSIZE?$AA@ 10004214     flags.obj
 0001:00003224       ??_C@_0BB@MNODJNPE@SE_COMMONSYNCHRO?$AA@ 10004224     flags.obj
 0001:00003238       ??_C@_0O@ICBCOJCG@DE_DLGPROCEND?$AA@ 10004238     flags.obj
 0001:00003248       ??_C@_0BC@BMFEJAMO@DE_DEFDLGPROCINIT?$AA@ 10004248     flags.obj
 0001:0000325c       ??_C@_0P@MBHAHBBG@DE_DLGPROCINIT?$AA@ 1000425c     flags.obj
 0001:0000326c       ??_C@_09MIOGFFI@EE_CHANGE?$AA@ 1000426c     flags.obj
 0001:00003278       ??_C@_0N@ILLPMAJF@EE_KILLFOCUS?$AA@ 10004278     flags.obj
 0001:00003288       ??_C@_0M@CPNMNBMF@EE_GOTFOCUS?$AA@ 10004288     flags.obj
 0001:00003294       ??_C@_08NFPFGIG@EE_CLOSE?$AA@ 10004294     flags.obj
 0001:000032a0       ??_C@_09NPOPIKMK@EE_REDRAW?$AA@ 100042a0     flags.obj
 0001:000032ac       ??_C@_07KJGPGPOC@EE_SAVE?$AA@ 100042ac     flags.obj
 0001:000032b4       ??_C@_07BLBPFFLB@EE_READ?$AA@ 100042b4     flags.obj
 0001:000032bc       ??_C@_0N@ICHCAKIB@VE_KILLFOCUS?$AA@ 100042bc     flags.obj
 0001:000032cc       ??_C@_0M@FEFKOOMJ@VE_GOTFOCUS?$AA@ 100042cc     flags.obj
 0001:000032d8       ??_C@_08JIBCCIDC@VE_CLOSE?$AA@ 100042d8     flags.obj
 0001:000032e4       ??_C@_07OJCLGDHJ@VE_READ?$AA@ 100042e4     flags.obj
 0001:000032ec       ??_C@_08BDDNDBMJ@VMT_DUMP?$AA@ 100042ec     flags.obj
 0001:000032f8       ??_C@_07FLIHDEDA@VMT_HEX?$AA@ 100042f8     flags.obj
 0001:00003300       ??_C@_08FNEFFFEL@VMT_TEXT?$AA@ 10004300     flags.obj
 0001:0000330c       ??_C@_0O@INKALKJK@VSMT_WORDWRAP?$AA@ 1000430c     flags.obj
 0001:0000331c       ??_C@_09FLKONCNO@VSMT_WRAP?$AA@ 1000431c     flags.obj
 0001:00003328       ??_C@_0O@MCNCFBLF@VSMT_VIEWMODE?$AA@ 10004328     flags.obj
 0001:00003338       ??_C@_0M@GHGAPHPP@TBPS_PAUSED?$AA@ 10004338     flags.obj
 0001:00003344       ??_C@_0L@DFDPCOFD@TBPS_ERROR?$AA@ 10004344     flags.obj
 0001:00003350       ??_C@_0M@KHLNKPHE@TBPS_NORMAL?$AA@ 10004350     flags.obj
 0001:0000335c       ??_C@_0BD@HMEHMDAL@TBPS_INDETERMINATE?$AA@ 1000435c     flags.obj
 0001:00003370       ??_C@_0BA@IPEAOBGN@TBPS_NOPROGRESS?$AA@ 10004370     flags.obj
 0001:00003380       ??_C@_0L@BCEMNGOG@WTYPE_HELP?$AA@ 10004380     flags.obj
 0001:0000338c       ??_C@_0M@OMKLELFA@WTYPE_VMENU?$AA@ 1000438c     flags.obj
 0001:00003398       ??_C@_0N@PBFHKEGB@WTYPE_DIALOG?$AA@ 10004398     flags.obj
 0001:000033a8       ??_C@_0N@HJNGGOKO@WTYPE_EDITOR?$AA@ 100043a8     flags.obj
 0001:000033b8       ??_C@_0N@EJKMDMBK@WTYPE_VIEWER?$AA@ 100043b8     flags.obj
 0001:000033c8       ??_C@_0N@FNCFCPIG@WTYPE_PANELS?$AA@ 100043c8     flags.obj
 0001:000033d8       ??_C@_0O@DCGKMPOM@WTYPE_DESKTOP?$AA@ 100043d8     flags.obj
 0001:000033e8       ??_C@_0L@PMDDFEBD@FMVT_PANEL?$AA@ 100043e8     flags.obj
 0001:000033f4       ??_C@_0L@DJIKMOJA@FMVT_ARRAY?$AA@ 100043f4     flags.obj
 0001:00003400       ??_C@_08DDPDBBNO@FMVT_NIL?$AA@ 10004400     flags.obj
 0001:0000340c       ??_C@_0N@FMHCFNDF@FMVT_POINTER?$AA@ 1000440c     flags.obj
 0001:0000341c       ??_C@_0M@GKPDICDA@FMVT_BINARY?$AA@ 1000441c     flags.obj
 0001:00003428       ??_C@_0N@MHKOBOGF@FMVT_BOOLEAN?$AA@ 10004428     flags.obj
 0001:00003438       ??_C@_0M@CKDAIOEN@FMVT_DOUBLE?$AA@ 10004438     flags.obj
 0001:00003444       ??_C@_0M@LFMLDDKI@FMVT_STRING?$AA@ 10004444     flags.obj
 0001:00003450       ??_C@_0N@BDMFKEKE@FMVT_INTEGER?$AA@ 10004450     flags.obj
 0001:00003460       ??_C@_0N@IBOAADDD@FMVT_UNKNOWN?$AA@ 10004460     flags.obj
 0001:00003470       ??_C@_0L@FJDDLDNN@MPEC_ERROR?$AA@ 10004470     flags.obj
 0001:0000347c       ??_C@_0N@CGFFMLBC@MPEC_SUCCESS?$AA@ 1000447c     flags.obj
 0001:0000348c       ??_C@_0BM@OICPADFE@MACROSTATE_RECORDING_COMMON?$AA@ 1000448c     flags.obj
 0001:000034a8       ??_C@_0BF@BGODKPBB@MACROSTATE_RECORDING?$AA@ 100044a8     flags.obj
 0001:000034c0       ??_C@_0BM@EJOFDENO@MACROSTATE_EXECUTING_COMMON?$AA@ 100044c0     flags.obj
 0001:000034dc       ??_C@_0BF@PCDEFEGP@MACROSTATE_EXECUTING?$AA@ 100044dc     flags.obj
 0001:000034f4       ??_C@_0BD@DIKEKAIJ@MACROSTATE_NOMACRO?$AA@ 100044f4     flags.obj
 0001:00003508       ??_C@_0BB@JPEEDDOG@MACROAREA_COMMON?$AA@ 10004508     flags.obj
 0001:0000351c       ??_C@_0BP@OIHAIGBK@MACROAREA_DIALOGAUTOCOMPLETION?$AA@ 1000451c     flags.obj
 0001:0000353c       ??_C@_0BO@OMLEPJPM@MACROAREA_SHELLAUTOCOMPLETION?$AA@ 1000453c     flags.obj
 0001:0000355c       ??_C@_0BD@JCFMJGDE@MACROAREA_USERMENU?$AA@ 1000455c     flags.obj
 0001:00003570       ??_C@_0BF@FCHKCGLL@MACROAREA_FINDFOLDER?$AA@ 10004570     flags.obj
 0001:00003588       ??_C@_0BE@HBMEGBOC@MACROAREA_TREEPANEL?$AA@ 10004588     flags.obj
 0001:0000359c       ??_C@_0BF@NLJMHMPP@MACROAREA_QVIEWPANEL?$AA@ 1000459c     flags.obj
 0001:000035b4       ??_C@_0BE@MDJPICHC@MACROAREA_INFOPANEL?$AA@ 100045b4     flags.obj
 0001:000035c8       ??_C@_0P@DKPKIEO@MACROAREA_HELP?$AA@ 100045c8     flags.obj
 0001:000035d8       ??_C@_0P@LFLMAHBF@MACROAREA_MENU?$AA@ 100045d8     flags.obj
 0001:000035e8       ??_C@_0BD@IGOOIJP@MACROAREA_MAINMENU?$AA@ 100045e8     flags.obj
 0001:000035fc       ??_C@_0BA@KKMKOLIK@MACROAREA_DISKS?$AA@ 100045fc     flags.obj
 0001:0000360c       ??_C@_0BB@MLMLHIGE@MACROAREA_SEARCH?$AA@ 1000460c     flags.obj
 0001:00003620       ??_C@_0BB@CADENPFI@MACROAREA_DIALOG?$AA@ 10004620     flags.obj
 0001:00003634       ??_C@_0BB@KILFBFJH@MACROAREA_EDITOR?$AA@ 10004634     flags.obj
 0001:00003648       ??_C@_0BB@JIMPEHCD@MACROAREA_VIEWER?$AA@ 10004648     flags.obj
 0001:0000365c       ??_C@_0BA@DEBOOAEB@MACROAREA_SHELL?$AA@ 1000465c     flags.obj
 0001:0000366c       ??_C@_0BA@MMOAIEKP@MACROAREA_OTHER?$AA@ 1000466c     flags.obj
 0001:0000367c       ??_C@_0L@MOADGAEB@MSSC_CHECK?$AA@ 1000467c     flags.obj
 0001:00003688       ??_C@_09CEDFMINA@MSSC_POST?$AA@ 10004688     flags.obj
 0001:00003694       ??_C@_0BD@IPKOEBIA@ACTL_GETWINDOWTYPE?$AA@ 10004694     flags.obj
 0001:000036a8       ??_C@_0BE@NPJGMDBM@ACTL_PROGRESSNOTIFY?$AA@ 100046a8     flags.obj
 0001:000036bc       ??_C@_0BC@CAAPIEHK@ACTL_SETCURSORPOS?$AA@ 100046bc     flags.obj
 0001:000036d0       ??_C@_0BC@FELBEIDG@ACTL_GETCURSORPOS?$AA@ 100046d0     flags.obj
 0001:000036e4       ??_C@_0BA@LJCPDIKK@ACTL_GETFARRECT?$AA@ 100046e4     flags.obj
 0001:000036f4       ??_C@_09HNDBKLDC@ACTL_QUIT?$AA@ 100046f4     flags.obj
 0001:00003700       ??_C@_0BG@ICJFAPHK@ACTL_SETPROGRESSVALUE?$AA@ 10004700     flags.obj
 0001:00003718       ??_C@_0BG@IJPADENB@ACTL_SETPROGRESSSTATE?$AA@ 10004718     flags.obj
 0001:00003730       ??_C@_0N@DHPLJLHO@ACTL_SYNCHRO?$AA@ 10004730     flags.obj
 0001:00003740       ??_C@_0P@JECKFIA@ACTL_REDRAWALL?$AA@ 10004740     flags.obj
 0001:00003750       ??_C@_0BD@JFOOLBPN@ACTL_SETARRAYCOLOR?$AA@ 10004750     flags.obj
 0001:00003764       ??_C@_0BA@CLHFKJJP@ACTL_GETFARHWND?$AA@ 10004764     flags.obj
 0001:00003774       ??_C@_0M@IHHFGPPA@ACTL_COMMIT?$AA@ 10004774     flags.obj
 0001:00003780       ??_C@_0BG@MNKPOEEN@ACTL_SETCURRENTWINDOW?$AA@ 10004780     flags.obj
 0001:00003798       ??_C@_0BE@PJBIPKOD@ACTL_GETWINDOWCOUNT?$AA@ 10004798     flags.obj
 0001:000037ac       ??_C@_0BD@DIFEEKNN@ACTL_GETWINDOWINFO?$AA@ 100047ac     flags.obj
 0001:000037c0       ??_C@_0BD@OKPAACIK@ACTL_GETARRAYCOLOR?$AA@ 100047c0     flags.obj
 0001:000037d4       ??_C@_0O@CEHHJAFD@ACTL_GETCOLOR?$AA@ 100047d4     flags.obj
 0001:000037e4       ??_C@_0N@DPABJDML@ACTL_WAITKEY?$AA@ 100047e4     flags.obj
 0001:000037f4       ??_C@_0BK@PHBCABMB@ACTL_GETFARMANAGERVERSION?$AA@ 100047f4     flags.obj
 0001:00003810       ??_C@_0BI@CNPFKHKO@EEC_LOADING_INTERRUPTED?$AA@ 10004810     flags.obj
 0001:00003828       ??_C@_0BB@HALKEFOL@EEC_NOT_MODIFIED?$AA@ 10004828     flags.obj
 0001:0000383c       ??_C@_0N@GLMELIKF@EEC_MODIFIED?$AA@ 1000483c     flags.obj
 0001:0000384c       ??_C@_0P@FEMAMJLE@EEC_OPEN_ERROR?$AA@ 1000484c     flags.obj
 0001:0000385c       ??_C@_09KFKGJDHC@SM_CHTIME?$AA@ 1000485c     flags.obj
 0001:00003868       ??_C@_0M@OAFEBGNH@SM_FULLNAME?$AA@ 10004868     flags.obj
 0001:00003874       ??_C@_0P@PKGMDPMD@SM_STREAMSSIZE?$AA@ 10004874     flags.obj
 0001:00003884       ??_C@_0O@CCKEKPHL@SM_NUMSTREAMS?$AA@ 10004884     flags.obj
 0001:00003894       ??_C@_0M@PKNLKFI@SM_NUMLINKS?$AA@ 10004894     flags.obj
 0001:000038a0       ??_C@_0BC@NKDBNAHD@SM_COMPRESSEDSIZE?$AA@ 100048a0     flags.obj
 0001:000038b4       ??_C@_08MEAGCMBB@SM_OWNER?$AA@ 100048b4     flags.obj
 0001:000038c0       ??_C@_08BCBPOLMA@SM_DESCR?$AA@ 100048c0     flags.obj
 0001:000038cc       ??_C@_07OMPKMIKC@SM_SIZE?$AA@ 100048cc     flags.obj
 0001:000038d4       ??_C@_08CPOLNKCG@SM_ATIME?$AA@ 100048d4     flags.obj
 0001:000038e0       ??_C@_08GCCDHLCN@SM_CTIME?$AA@ 100048e0     flags.obj
 0001:000038ec       ??_C@_08FICJBKFN@SM_MTIME?$AA@ 100048ec     flags.obj
 0001:000038f8       ??_C@_06GJJJNNFE@SM_EXT?$AA@ 100048f8     flags.obj
 0001:00003900       ??_C@_07KIFHAGIL@SM_NAME?$AA@ 10004900     flags.obj
 0001:00003908       ??_C@_0M@JGBFGGEA@SM_UNSORTED?$AA@ 10004908     flags.obj
 0001:00003914       ??_C@_0L@OPHJOKKE@SM_DEFAULT?$AA@ 10004914     flags.obj
 0001:00003920       ??_C@_0BA@NKMDEBG@PTYPE_INFOPANEL?$AA@ 10004920     flags.obj
 0001:00003930       ??_C@_0BB@JBINOKAI@PTYPE_QVIEWPANEL?$AA@ 10004930     flags.obj
 0001:00003944       ??_C@_0BA@LPPHNHIG@PTYPE_TREEPANEL?$AA@ 10004944     flags.obj
 0001:00003954       ??_C@_0BA@KNHGEBNE@PTYPE_FILEPANEL?$AA@ 10004954     flags.obj
 0001:00003964       ??_C@_0L@KHCLMGFJ@CBET_MOUSE?$AA@ 10004964     flags.obj
 0001:00003970       ??_C@_08PPADCPCM@CBET_KEY?$AA@ 10004970     flags.obj
 0001:0000397c       ??_C@_0O@ILJOJGLD@BSTATE_TOGGLE?$AA@ 1000497c     flags.obj
 0001:0000398c       ??_C@_0O@KBIFGGHO@BSTATE_3STATE?$AA@ 1000498c     flags.obj
 0001:0000399c       ??_C@_0P@FALAMPGP@BSTATE_CHECKED?$AA@ 1000499c     flags.obj
 0001:000039ac       ??_C@_0BB@HLBBGMAN@BSTATE_UNCHECKED?$AA@ 100049ac     flags.obj
 0001:000039c0       ??_C@_07DIJJNCBA@DM_USER?$AA@ 100049c0     flags.obj
 0001:000039c8       ??_C@_0BD@NGEKAPIF@DN_DRAWDLGITEMDONE?$AA@ 100049c8     flags.obj
 0001:000039dc       ??_C@_0BC@MHCBFAAO@DN_DROPDOWNOPENED?$AA@ 100049dc     flags.obj
 0001:000039f0       ??_C@_0M@POIFBPFN@DN_GETVALUE?$AA@ 100049f0     flags.obj
 0001:000039fc       ??_C@_08EHEOFOJD@DN_CLOSE?$AA@ 100049fc     flags.obj
 0001:00003a08       ??_C@_0BA@FGOGLDBC@DN_CONTROLINPUT?$AA@ 10004a08     flags.obj
 0001:00003a18       ??_C@_08MDDLDGPO@DN_INPUT?$AA@ 10004a18     flags.obj
 0001:00003a24       ??_C@_0O@EONPBNNP@DN_LISTHOTKEY?$AA@ 10004a24     flags.obj
 0001:00003a34       ??_C@_0BC@FHPPFLKG@DN_DRAWDIALOGDONE?$AA@ 10004a34     flags.obj
 0001:00003a48       ??_C@_0BB@BOOOCAEG@DN_RESIZECONSOLE?$AA@ 10004a48     flags.obj
 0001:00003a5c       ??_C@_0L@MLMFBHN@DN_DRAGGED?$AA@ 10004a5c     flags.obj
 0001:00003a68       ??_C@_0O@CLPABIGO@DN_LISTCHANGE?$AA@ 10004a68     flags.obj
 0001:00003a78       ??_C@_0N@CHLLLNBO@DN_KILLFOCUS?$AA@ 10004a78     flags.obj
 0001:00003a88       ??_C@_0O@BJECHBCA@DN_INITDIALOG?$AA@ 10004a88     flags.obj
 0001:00003a98       ??_C@_09EDGJFAK@DN_HOTKEY?$AA@ 10004a98     flags.obj
 0001:00003aa4       ??_C@_07NJJEMKPA@DN_HELP?$AA@ 10004aa4     flags.obj
 0001:00003aac       ??_C@_0M@JHFIBKOO@DN_GOTFOCUS?$AA@ 10004aac     flags.obj
 0001:00003ab8       ??_C@_0N@OCGKCPJF@DN_ENTERIDLE?$AA@ 10004ab8     flags.obj
 0001:00003ac8       ??_C@_0O@JMKNGFLE@DN_EDITCHANGE?$AA@ 10004ac8     flags.obj
 0001:00003ad8       ??_C@_0P@KGKEDPBI@DN_DRAWDLGITEM?$AA@ 10004ad8     flags.obj
 0001:00003ae8       ??_C@_0O@NKBDPILK@DN_DRAWDIALOG?$AA@ 10004ae8     flags.obj
 0001:00003af8       ??_C@_0BD@JMFJPHPD@DN_CTLCOLORDLGLIST?$AA@ 10004af8     flags.obj
 0001:00003b0c       ??_C@_0BD@HFGBIBBL@DN_CTLCOLORDLGITEM?$AA@ 10004b0c     flags.obj
 0001:00003b20       ??_C@_0BC@MJFJAANN@DN_CTLCOLORDIALOG?$AA@ 10004b20     flags.obj
 0001:00003b34       ??_C@_0M@NNNAPNMA@DN_BTNCLICK?$AA@ 10004b34     flags.obj
 0001:00003b40       ??_C@_08COMJOMAC@DN_FIRST?$AA@ 10004b40     flags.obj
 0001:00003b4c       ??_C@_0BC@KJOLMFGG@DM_GETDIALOGTITLE?$AA@ 10004b4c     flags.obj
 0001:00003b60       ??_C@_0BB@GAPFMPKE@DM_GETDIALOGINFO?$AA@ 10004b60     flags.obj
 0001:00003b74       ??_C@_0BD@EMPBPAFP@DM_SETDLGITEMSHORT?$AA@ 10004b74     flags.obj
 0001:00003b88       ??_C@_0BD@HOOHICEG@DM_GETDLGITEMSHORT?$AA@ 10004b88     flags.obj
 0001:00003b9c       ??_C@_0BD@CJEPBACF@DM_GETCONSTTEXTPTR?$AA@ 10004b9c     flags.obj
 0001:00003bb0       ??_C@_0BE@KGBLNJKA@DM_GETCOMBOBOXEVENT?$AA@ 10004bb0     flags.obj
 0001:00003bc4       ??_C@_0BE@MCECGHBC@DM_SETCOMBOBOXEVENT?$AA@ 10004bc4     flags.obj
 0001:00003bd8       ??_C@_0BD@GKGFBKHH@DM_SETEDITPOSITION?$AA@ 10004bd8     flags.obj
 0001:00003bec       ??_C@_0BD@FIHDGIGO@DM_GETEDITPOSITION?$AA@ 10004bec     flags.obj
 0001:00003c00       ??_C@_0BA@GDNOBFED@DM_SETSELECTION?$AA@ 10004c00     flags.obj
 0001:00003c10       ??_C@_0BA@BHGANJAP@DM_GETSELECTION?$AA@ 10004c10     flags.obj
 0001:00003c20       ??_C@_0BD@LAOOKGHD@DM_LISTGETDATASIZE?$AA@ 10004c20     flags.obj
 0001:00003c34       ??_C@_0BB@DANLMDCJ@DM_SETCURSORSIZE?$AA@ 10004c34     flags.obj
 0001:00003c48       ??_C@_0BB@EPMFHAFO@DM_GETCURSORSIZE?$AA@ 10004c48     flags.obj
 0001:00003c5c       ??_C@_0L@KNFAKFKE@DM_LISTSET?$AA@ 10004c5c     flags.obj
 0001:00003c68       ??_C@_0P@OGLDKOHO@DM_SETITEMDATA?$AA@ 10004c68     flags.obj
 0001:00003c78       ??_C@_0P@OJKNHIPN@DM_GETITEMDATA?$AA@ 10004c78     flags.obj
 0001:00003c88       ??_C@_0BF@IAGIACOD@DM_EDITUNCHANGEDFLAG?$AA@ 10004c88     flags.obj
 0001:00003ca0       ??_C@_0BH@CFMLLNNM@DM_SETMOUSEEVENTNOTIFY?$AA@ 10004ca0     flags.obj
 0001:00003cb8       ??_C@_0BC@BENFKLNH@DM_SETINPUTNOTIFY?$AA@ 10004cb8     flags.obj
 0001:00003ccc       ??_C@_0BD@BPHAAEIM@DM_GETITEMPOSITION?$AA@ 10004ccc     flags.obj
 0001:00003ce0       ??_C@_0O@NPDKADMJ@DM_SETHISTORY?$AA@ 10004ce0     flags.obj
 0001:00003cf0       ??_C@_0BF@LJIGJNAO@DM_SETDROPDOWNOPENED?$AA@ 10004cf0     flags.obj
 0001:00003d08       ??_C@_0BF@JMINBGBA@DM_GETDROPDOWNOPENED?$AA@ 10004d08     flags.obj
 0001:00003d20       ??_C@_0BD@CNGGHGJF@DM_SETITEMPOSITION?$AA@ 10004d20     flags.obj
 0001:00003d34       ??_C@_0BA@ICDJCFLE@DM_RESIZEDIALOG?$AA@ 10004d34     flags.obj
 0001:00003d44       ??_C@_0BB@KPJPKCP@DM_LISTGETTITLES?$AA@ 10004d44     flags.obj
 0001:00003d58       ??_C@_0BB@CELMNLLN@DM_LISTSETTITLES?$AA@ 10004d58     flags.obj
 0001:00003d6c       ??_C@_0P@DGKKKCB@DM_LISTSETDATA?$AA@ 10004d6c     flags.obj
 0001:00003d7c       ??_C@_0P@PLJLJFPA@DM_LISTGETDATA?$AA@ 10004d7c     flags.obj
 0001:00003d8c       ??_C@_0M@EEAEBLKC@DM_LISTINFO?$AA@ 10004d8c     flags.obj
 0001:00003d98       ??_C@_0BC@MIFCLOBD@DM_LISTFINDSTRING?$AA@ 10004d98     flags.obj
 0001:00003dac       ??_C@_0O@GAAGMJJL@DM_LISTINSERT?$AA@ 10004dac     flags.obj
 0001:00003dbc       ??_C@_0O@PDFCNPKN@DM_LISTUPDATE?$AA@ 10004dbc     flags.obj
 0001:00003dcc       ??_C@_0O@HBHDMHP@DM_LISTADDSTR?$AA@ 10004dcc     flags.obj
 0001:00003ddc       ??_C@_0L@BMEAECNG@DM_LISTADD?$AA@ 10004ddc     flags.obj
 0001:00003de8       ??_C@_0O@NOPCAHGJ@DM_LISTDELETE?$AA@ 10004de8     flags.obj
 0001:00003df8       ??_C@_0BB@GKMJCDEM@DM_LISTSETCURPOS?$AA@ 10004df8     flags.obj
 0001:00003e0c       ??_C@_0BB@EEIMACNO@DM_LISTGETCURPOS?$AA@ 10004e0c     flags.obj
 0001:00003e20       ??_C@_0P@NFJNHAKH@DM_LISTGETITEM?$AA@ 10004e20     flags.obj
 0001:00003e30       ??_C@_0M@GEPBDDNC@DM_LISTSORT?$AA@ 10004e30     flags.obj
 0001:00003e3c       ??_C@_0N@MEGOPFGK@DM_SET3STATE?$AA@ 10004e3c     flags.obj
 0001:00003e4c       ??_C@_0M@DDGACGLO@DM_SETCHECK?$AA@ 10004e4c     flags.obj
 0001:00003e58       ??_C@_0M@MCEMDFMD@DM_GETCHECK?$AA@ 10004e58     flags.obj
 0001:00003e64       ??_C@_0O@GKKCFHIM@DM_ADDHISTORY?$AA@ 10004e64     flags.obj
 0001:00003e74       ??_C@_0M@NCOJHJKI@DM_SHOWITEM?$AA@ 10004e74     flags.obj
 0001:00003e80       ??_C@_0O@LGEKFPKK@DM_SETTEXTPTR?$AA@ 10004e80     flags.obj
 0001:00003e90       ??_C@_0BA@KPHABNOF@DM_SETCURSORPOS?$AA@ 10004e90     flags.obj
 0001:00003ea0       ??_C@_0BA@NLMONBKJ@DM_GETCURSORPOS?$AA@ 10004ea0     flags.obj
 0001:00003eb0       ??_C@_0M@JPHKGACH@DM_GETFOCUS?$AA@ 10004eb0     flags.obj
 0001:00003ebc       ??_C@_0O@BIFKIPIP@DM_SHOWDIALOG?$AA@ 10004ebc     flags.obj
 0001:00003ecc       ??_C@_0BE@LABEAIPD@DM_SETMAXTEXTLENGTH?$AA@ 10004ecc     flags.obj
 0001:00003ee0       ??_C@_0L@LDOCOEIP@DM_SETTEXT?$AA@ 10004ee0     flags.obj
 0001:00003eec       ??_C@_09ILPFEDOM@DM_REDRAW?$AA@ 10004eec     flags.obj
 0001:00003ef8       ??_C@_0M@GOFGHDFK@DM_SETFOCUS?$AA@ 10004ef8     flags.obj
 0001:00003f04       ??_C@_0O@GKEFJIKB@DM_SETDLGITEM?$AA@ 10004f04     flags.obj
 0001:00003f14       ??_C@_0O@EEEDHNPG@DM_SETDLGDATA?$AA@ 10004f14     flags.obj
 0001:00003f24       ??_C@_0O@DIPLLJEH@DM_MOVEDIALOG?$AA@ 10004f24     flags.obj
 0001:00003f34       ??_C@_06IKGPEGEJ@DM_KEY?$AA@ 10004f34     flags.obj
 0001:00003f3c       ??_C@_0L@ELBDNLFO@DM_GETTEXT?$AA@ 10004f3c     flags.obj
 0001:00003f48       ??_C@_0O@BEHCGMCL@DM_GETDLGRECT?$AA@ 10004f48     flags.obj
 0001:00003f58       ??_C@_0O@HEGKCPOI@DM_GETDLGITEM?$AA@ 10004f58     flags.obj
 0001:00003f68       ??_C@_0O@FKGMMKLP@DM_GETDLGDATA?$AA@ 10004f68     flags.obj
 0001:00003f78       ??_C@_0BA@KAMJGFDG@DM_ENABLEREDRAW?$AA@ 10004f78     flags.obj
 0001:00003f88       ??_C@_09KLJOCKAA@DM_ENABLE?$AA@ 10004f88     flags.obj
 0001:00003f94       ??_C@_08MJMBFJHA@DM_CLOSE?$AA@ 10004f94     flags.obj
 0001:00003fa0       ??_C@_08KAEGOLOB@DM_FIRST?$AA@ 10004fa0     flags.obj
 0001:00003fac       ??_C@_0P@GDJDPEIK@DI_USERCONTROL?$AA@ 10004fac     flags.obj
 0001:00003fbc       ??_C@_0L@ONDMPPPO@DI_LISTBOX?$AA@ 10004fbc     flags.obj
 0001:00003fc8       ??_C@_0M@MAKBFNGC@DI_COMBOBOX?$AA@ 10004fc8     flags.obj
 0001:00003fd4       ??_C@_0P@GIPCGMBE@DI_RADIOBUTTON?$AA@ 10004fd4     flags.obj
 0001:00003fe4       ??_C@_0M@MHFHGPHJ@DI_CHECKBOX?$AA@ 10004fe4     flags.obj
 0001:00003ff0       ??_C@_09GGAEMAPJ@DI_BUTTON?$AA@ 10004ff0     flags.obj
 0001:00003ffc       ??_C@_0L@MGOIMBKF@DI_FIXEDIT?$AA@ 10004ffc     flags.obj
 0001:00004008       ??_C@_0L@EOMEIIFM@DI_PSWEDIT?$AA@ 10005008     flags.obj
 0001:00004014       ??_C@_07DOLIFAEF@DI_EDIT?$AA@ 10005014     flags.obj
 0001:0000401c       ??_C@_0N@EDCLIEAE@DI_DOUBLEBOX?$AA@ 1000501c     flags.obj
 0001:0000402c       ??_C@_0N@IGKKGFMF@DI_SINGLEBOX?$AA@ 1000502c     flags.obj
 0001:0000403c       ??_C@_08HODBDEHE@DI_VTEXT?$AA@ 1000503c     flags.obj
 0001:00004048       ??_C@_07MGGAEAFF@DI_TEXT?$AA@ 10005048     flags.obj
 0001:00004050       ??_C@_0BN@PPNDCHHA@EDITOR_COLOR_NORMAL_PRIORITY?$AA@ 10005050     flags.obj
 0001:00004070       ??_C@_0P@NHNDIKJ@CURRENT_EDITOR?$AA@ 10005070     flags.obj
 0001:00004080       ??_C@_0N@HLIFAAPJ@EEREDRAW_ALL?$AA@ 10005080     flags.obj
 0001:00004090       ??_C@_0L@GOEBPENN@PANEL_STOP?$AA@ 10005090     flags.obj
 0001:0000409c       ??_C@_0O@HPKEABPN@PANEL_PASSIVE?$AA@ 1000509c     flags.obj
 0001:000040ac       ??_C@_0N@LPMKALBG@PANEL_ACTIVE?$AA@ 100050ac     flags.obj
 0001:000040bc       ??_C@_0L@EHFOPLFD@PANEL_NONE?$AA@ 100050bc     flags.obj
 0001:000040c8       ??_C@_09ENNBLPJC@ALPHAMASK?$AA@ 100050c8     flags.obj
 0001:000040d4       ??_C@_09BLFIDJLF@COLORMASK?$AA@ 100050d4     flags.obj
 0001:000040e0       ??_C@_09MNAPNKKC@INDEXMASK?$AA@ 100050e0     flags.obj
 0001:000040ec       ??_C@_0M@OMCMFJHA@CP_REDETECT?$AA@ 100050ec     flags.obj
 0001:000040f8       ??_C@_0L@JDNPCEDH@CP_DEFAULT?$AA@ 100050f8     flags.obj
 0001:00004104       ??_C@_0O@MNMCMEJH@CP_REVERSEBOM?$AA@ 10005104     flags.obj
 0001:00004114       ??_C@_0L@MIDBGFJO@CP_UNICODE?$AA@ 10005114     flags.obj
 0001:00004120       ??_C@_0BI@MOOFLFPC@FARMANAGERVERSION_STAGE?$AA@ 10005120     flags.obj
 0001:00004138       ??_C@_0BI@OLPFLLDD@FARMANAGERVERSION_BUILD?$AA@ 10005138     flags.obj
 0001:00004150       ??_C@_0BL@NMALNAFP@FARMANAGERVERSION_REVISION?$AA@ 10005150     flags.obj
 0001:0000416c       ??_C@_0BI@DMLKEAFC@FARMANAGERVERSION_MINOR?$AA@ 1000516c     flags.obj
 0001:00004184       ??_C@_0BI@IDKIJMME@FARMANAGERVERSION_MAJOR?$AA@ 10005184     flags.obj
 0001:000049c0       _Vals                      100059c0     flags.obj
 0001:00008164       ??_C@_05GALAPKHH@Guids?$AA@ 10009164     keysandcolors.obj
 0001:0000816c       ??_C@_06ICDCBJPI@Colors?$AA@ 1000916c     keysandcolors.obj
 0001:000089a0       ??_C@_01EEMJAFIK@?6?$AA@   100099a0     lflua.obj
 0001:000089a4       ??_C@_0BB@BJDGDOHH@cannot?5?$CFs?5?$CFs?3?5?$CFs?$AA@ 100099a4     lflua.obj
 0001:000089b8       ??_C@_03PKPBNCAL@?o?$LL?$LP?$AA@ 100099b8     lflua.obj
 0001:000089bc       ??_C@_04POLDLDMI@read?$AA@ 100099bc     lflua.obj
 0001:000089c4       ??_C@_06IEGCHAII@reopen?$AA@ 100099c4     lflua.obj
 0001:000089cc       ??_C@_15JJPIMNBO@?$AAr?$AAb?$AA?$AA@ 100099cc     lflua.obj
 0001:000089d4       ??_C@_04PMOCAHAA@open?$AA@ 100099d4     lflua.obj
 0001:000089dc       ??_C@_01EOFPKCAF@?$EA?$AA@ 100099dc     lflua.obj
 0001:000089e0       ??_C@_06CCPPALKB@?$DNstdin?$AA@ 100099e0     lflua.obj
 0001:000089e8       ??_C@_02LOCGON@?$AA?$AA?$AA@ 100099e8     lflua.obj
 0001:000089ec       ??_C@_07PPMFDHAH@gmatchW?$AA@ 100099ec     lregex.obj
 0001:000089f4       ??_C@_06DPFCLDIO@gmatch?$AA@ 100099f4     lregex.obj
 0001:000089fc       ??_C@_04BDLIKKMN@__gc?$AA@ 100099fc     lregex.obj
 0001:00008a04       ??_C@_0O@OJAOCNID@bracketscount?$AA@ 10009a04     lregex.obj
 0001:00008a14       ??_C@_06NNKFJOLC@matchW?$AA@ 10009a14     lregex.obj
 0001:00008a1c       ??_C@_05HPGHPNC@gsubW?$AA@ 10009a1c     lregex.obj
 0001:00008a24       ??_C@_05GFGPIPHI@findW?$AA@ 10009a24     lregex.obj
 0001:00008a2c       ??_C@_05FNONLPDI@match?$AA@ 10009a2c     lregex.obj
 0001:00008a34       ??_C@_04GOLEAPFD@gsub?$AA@ 10009a34     lregex.obj
 0001:00008a3c       ??_C@_04CKFJHKAP@find?$AA@ 10009a3c     lregex.obj
 0001:00009270       _regex_methods             1000a270     lregex.obj
 0001:000092c0       _regex_functions           1000a2c0     lregex.obj
 0001:00009310       ??_C@_0BO@PBOFMCLL@attempt?5to?5access?5freed?5regex?$AA@ 1000a310     lregex.obj
 0001:00009330       ??_C@_09KIEPBIJC@far_regex?$AA@ 1000a330     lregex.obj
 0001:0000933c       ??_C@_07IHINEPFG@?$CFs?5?$CI?$CFp?$CJ?$AA@ 1000a33c     lregex.obj
 0001:00009344       ??_C@_01KMDKNFGN@?1?$AA@   1000a344     lregex.obj
 0001:00009348       ??_C@_0BL@HEFMPIBG@invalid?5regular?5expression?$AA@ 1000a348     lregex.obj
 0001:00009364       ??_C@_0BE@BBBEAHLK@RECTL_CREATE?5failed?$AA@ 1000a364     lregex.obj
 0001:00009378       ??_C@_0BK@JCLHPPNA@cannot?5add?5?$CFd?5stack?5slots?$AA@ 1000a378     lregex.obj
 0001:00009394       ??_C@_0BE@KPDOHKBE@invalid?5return?5type?$AA@ 1000a394     lregex.obj
 0001:000093a8       ??_C@_0BJ@IMAIDFKH@invalid?5replacement?5type?$AA@ 1000a3a8     lregex.obj
 0001:000093c4       ??_C@_0CG@IDFLGMFM@replace?5string?3?5invalid?5capture?5@ 1000a3c4     lregex.obj
 0001:000093ec       ??_C@_0BM@MOHHGMBK@string?5or?5table?5or?5function?$AA@ 1000a3ec     lregex.obj
 0001:00009408       ??_C@_05FGAODPCE@regex?$AA@ 1000a408     lregex.obj
 0001:00009410       ??_C@_07NHABFFHN@__index?$AA@ 1000a410     lregex.obj
 0001:00009c50       ??_C@_0BC@PMGNICBE@MacroPluginReturn?$AA@ 1000ac50     luamacro.obj
 0001:00009c68       ??_C@_1FA@DAFHIDEP@?$AAt?$AAo?$AAo?$AA?5?$AAm?$AAa?$AAn?$AAy?$AA?5?$AAv?$AAa?$AAl?$AAu?$AAe?$AAs?$AA?5?$AAt?$AAo?$AA?5?$AAp?$AAl?$AAa?$AAc?$AAe?$AA?5?$AAo?$AAn?$AAt?$AAo?$AA?5?$AAL?$AAu@ 1000ac68     luamacro.obj
 0001:00009cb8       ??_C@_1BC@GBFPAMBP@?$AAL?$AAu?$AAa?$AAM?$AAa?$AAc?$AAr?$AAo?$AA?$AA@ 1000acb8     luamacro.obj
 0001:00009ccc       ??_C@_15PMCGDJNJ@?$AAO?$AAK?$AA?$AA@ 1000accc     luamacro.obj
 0001:00009cd4       ??_C@_02JIEIHMJD@wl?$AA@   1000acd4     luamacro.obj
 0001:00009cd8       ??_C@_0BB@FCMFBGOM@invalid?5argument?$AA@ 1000acd8     luamacro.obj
 0001:00009cec       ??_C@_0BN@ICDOMFBB@invalid?5argument?5?$CD?$CFd?5to?5?8?$CFs?8?$AA@ 1000acec     luamacro.obj
 0001:00009d0c       ??_C@_0BC@KFJDHEIC@CreateUserControl?$AA@ 1000ad0c     lusercontrol.obj
 0001:00009d20       ??_C@_0L@GADKNKH@__newindex?$AA@ 1000ad20     lusercontrol.obj
 0001:00009d2c       ??_C@_05MNDELLDN@__len?$AA@ 1000ad2c     lusercontrol.obj
 0001:0000a558       _usercontrol_methods       1000b558     lusercontrol.obj
 0001:0000a580       _usercontrol_functions     1000b580     lusercontrol.obj
 0001:0000a590       ??_C@_0BA@MDNLMOMP@far_usercontrol?$AA@ 1000b590     lusercontrol.obj
 0001:0000a5a0       ??_C@_0BH@DOPNHMGD@bounds?5checking?5failed?$AA@ 1000b5a0     lusercontrol.obj
 0001:0000a5b8       ??_C@_0L@PLFFHFAH@Attributes?$AA@ 1000b5b8     lusercontrol.obj
 0001:0000a5c4       ??_C@_04IMAAEPPE@Char?$AA@ 1000b5c4     lusercontrol.obj
 0001:0000a5cc       ??_C@_0BD@MIGOMCGP@Y?5must?5be?5positive?$AA@ 1000b5cc     lusercontrol.obj
 0001:0000a5e0       ??_C@_0BD@BPIMECDH@X?5must?5be?5positive?$AA@ 1000b5e0     lusercontrol.obj
 0001:0000a5f4       ??_C@_03IGHFHLNJ@jit?$AA@  1000b5f4     service.obj
 0001:0000a5f8       ??_C@_03DIJDOPEA@ffi?$AA@  1000b5f8     service.obj
 0001:0000a5fc       ??_C@_03EDMBFDDG@bit?$AA@  1000b5fc     service.obj
 0001:0000a600       ??_C@_03JECLAOEA@win?$AA@  1000b600     service.obj
 0001:0000a604       ??_C@_07GAJMMAJO@unicode?$AA@ 1000b604     service.obj
 0001:0000a60c       ??_C@_04CFDJAKFL@math?$AA@ 1000b60c     service.obj
 0001:0000a614       ??_C@_06ICGJLFIM@string?$AA@ 1000b614     service.obj
 0001:0000a61c       ??_C@_02EHCHIAMF@os?$AA@   1000b61c     service.obj
 0001:0000a620       ??_C@_02KFNNKBCK@io?$AA@   1000b620     service.obj
 0001:0000a624       ??_C@_05LCLENNFI@table?$AA@ 1000b624     service.obj
 0001:0000a62c       ??_C@_05NHFJDMOA@Timer?$AA@ 1000b62c     service.obj
 0001:0000a634       ??_C@_04JLAJABDJ@Show?$AA@ 1000b634     service.obj
 0001:0000a63c       ??_C@_0O@BJEAJNBH@MakeMenuItems?$AA@ 1000b63c     service.obj
 0001:0000a64c       ??_C@_0BB@JBNBALEM@GetNumberOfLinks?$AA@ 1000b64c     service.obj
 0001:0000a660       ??_C@_0N@MOMBJEKA@GetFileOwner?$AA@ 1000b660     service.obj
 0001:0000a670       ??_C@_0BE@DJLJEKBK@GetCurrentDirectory?$AA@ 1000b670     service.obj
 0001:0000a684       ??_C@_0BD@ELMHPHAC@CPluginStartupInfo?$AA@ 1000b684     service.obj
 0001:0000a698       ??_C@_08KJBLDCDF@FarClock?$AA@ 1000b698     service.obj
 0001:0000a6a4       ??_C@_0P@BGLLKGOI@FormatFileSize?$AA@ 1000b6a4     service.obj
 0001:0000a6b4       ??_C@_04OCDKHGII@XLat?$AA@ 1000b6b4     service.obj
 0001:0000a6bc       ??_C@_0M@HKHGOOHG@ConvertPath?$AA@ 1000b6bc     service.obj
 0001:0000a6c8       ??_C@_0BA@CLEHBIPM@RecursiveSearch?$AA@ 1000b6c8     service.obj
 0001:0000a6d8       ??_C@_08BNEIIKEJ@TruncStr?$AA@ 1000b6d8     service.obj
 0001:0000a6e4       ??_C@_0N@CCDDAJK@TruncPathStr?$AA@ 1000b6e4     service.obj
 0001:0000a6f4       ??_C@_06DKBBJCCG@MkLink?$AA@ 1000b6f4     service.obj
 0001:0000a6fc       ??_C@_06ILCHIEBO@MkTemp?$AA@ 1000b6fc     service.obj
 0001:0000a704       ??_C@_09GLKFOOEP@LUpperBuf?$AA@ 1000b704     service.obj
 0001:0000a710       ??_C@_09LPKAHGM@LLowerBuf?$AA@ 1000b710     service.obj
 0001:0000a71c       ??_C@_08FHLJMDJK@LIsUpper?$AA@ 1000b71c     service.obj
 0001:0000a728       ??_C@_08MAHKICD@LIsLower?$AA@ 1000b728     service.obj
 0001:0000a734       ??_C@_0M@LKJIEECA@LIsAlphanum?$AA@ 1000b734     service.obj
 0001:0000a740       ??_C@_08DNJCLFF@LIsAlpha?$AA@ 1000b740     service.obj
 0001:0000a74c       ??_C@_0BE@EPGHGPJC@GetReparsePointInfo?$AA@ 1000b74c     service.obj
 0001:0000a760       ??_C@_0M@KFCNKLDK@GetPathRoot?$AA@ 1000b760     service.obj
 0001:0000a76c       ??_C@_0M@KPPMMAOL@ProcessName?$AA@ 1000b76c     service.obj
 0001:0000a778       ??_C@_09GALOFBAC@LStrnicmp?$AA@ 1000b778     service.obj
 0001:0000a784       ??_C@_08HGLFNLMB@LStricmp?$AA@ 1000b784     service.obj
 0001:0000a790       ??_C@_0BC@FFNOIDFI@NameToInputRecord?$AA@ 1000b790     service.obj
 0001:0000a7a4       ??_C@_0BC@FJDIKOMH@InputRecordToName?$AA@ 1000b7a4     service.obj
 0001:0000a7b8       ??_C@_0BD@PLIHDKFC@PasteFromClipboard?$AA@ 1000b7b8     service.obj
 0001:0000a7cc       ??_C@_0BA@EOCNNPOG@CopyToClipboard?$AA@ 1000b7cc     service.obj
 0001:0000a7dc       ??_C@_0M@IFKFGKML@ColorDialog?$AA@ 1000b7dc     service.obj
 0001:0000a7e8       ??_C@_0N@GOMOBHDB@FreeSettings?$AA@ 1000b7e8     service.obj
 0001:0000a7f8       ??_C@_0P@HMKEDHIE@CreateSettings?$AA@ 1000b7f8     service.obj
 0001:0000a808       ??_C@_0P@IKAEEPOB@IsPluginLoaded?$AA@ 1000b808     service.obj
 0001:0000a818       ??_C@_0L@JIDCIJHM@GetPlugins?$AA@ 1000b818     service.obj
 0001:0000a824       ??_C@_0BF@KLOGLFMF@GetPluginInformation?$AA@ 1000b824     service.obj
 0001:0000a83c       ??_C@_0L@DACPHGGH@FindPlugin?$AA@ 1000b83c     service.obj
 0001:0000a848       ??_C@_0BB@IJHIBGJA@ForcedLoadPlugin?$AA@ 1000b848     service.obj
 0001:0000a85c       ??_C@_0N@DHIONCLI@UnloadPlugin?$AA@ 1000b85c     service.obj
 0001:0000a86c       ??_C@_0L@CHJBHF@LoadPlugin?$AA@ 1000b86c     service.obj
 0001:0000a878       ??_C@_0BB@BICELPOF@CreateFileFilter?$AA@ 1000b878     service.obj
 0001:0000a88c       ??_C@_0N@COEPENFH@MacroExecute?$AA@ 1000b88c     service.obj
 0001:0000a89c       ??_C@_0BC@MJDKBAPF@MacroGetLastError?$AA@ 1000b89c     service.obj
 0001:0000a8b0       ??_C@_0M@KFMHCNNB@MacroDelete?$AA@ 1000b8b0     service.obj
 0001:0000a8bc       ??_C@_08KAFLEHAN@MacroAdd?$AA@ 1000b8bc     service.obj
 0001:0000a8c8       ??_C@_0L@KBAKOGFP@MacroCheck?$AA@ 1000b8c8     service.obj
 0001:0000a8d4       ??_C@_09KGKKBHMO@MacroPost?$AA@ 1000b8d4     service.obj
 0001:0000a8e0       ??_C@_0N@PNLHCOIE@MacroGetArea?$AA@ 1000b8e0     service.obj
 0001:0000a8f0       ??_C@_0O@KGHDMPAJ@MacroGetState?$AA@ 1000b8f0     service.obj
 0001:0000a900       ??_C@_0N@NAGBAPAE@MacroSaveAll?$AA@ 1000b900     service.obj
 0001:0000a910       ??_C@_0N@GHGEMEN@MacroLoadAll?$AA@ 1000b910     service.obj
 0001:0000a920       ??_C@_0L@HHLOIHOP@AdvControl?$AA@ 1000b920     service.obj
 0001:0000a92c       ??_C@_08IAADAJIH@InputBox?$AA@ 1000b92c     service.obj
 0001:0000a938       ??_C@_08DAHHHDJC@ShowHelp?$AA@ 1000b938     service.obj
 0001:0000a944       ??_C@_0L@PGGGPLFK@SaveScreen?$AA@ 1000b944     service.obj
 0001:0000a950       ??_C@_0O@CGLFPNOD@RestoreScreen?$AA@ 1000b950     service.obj
 0001:0000a960       ??_C@_07BEIHKDLJ@Message?$AA@ 1000b960     service.obj
 0001:0000a968       ??_C@_04IFEHPILC@Menu?$AA@ 1000b968     service.obj
 0001:0000a970       ??_C@_0BB@HIDBFOJJ@GetPluginDirList?$AA@ 1000b970     service.obj
 0001:0000a984       ??_C@_06KCCBBIBJ@GetMsg?$AA@ 1000b984     service.obj
 0001:0000a98c       ??_C@_0L@MCFABBED@GetDirList?$AA@ 1000b98c     service.obj
 0001:0000a998       ??_C@_0BK@EBIPEKDH@SubscribeDialogDrawEvents?$AA@ 1000b998     service.obj
 0001:0000a9b4       ??_C@_0L@DEGEGMGN@SetDlgItem?$AA@ 1000b9b4     service.obj
 0001:0000a9c0       ??_C@_0L@CKELNLCE@GetDlgItem?$AA@ 1000b9c0     service.obj
 0001:0000a9cc       ??_C@_0P@HLOFPDFP@SendDlgMessage?$AA@ 1000b9cc     service.obj
 0001:0000a9dc       ??_C@_0L@DLFLHLOO@DialogFree?$AA@ 1000b9dc     service.obj
 0001:0000a9e8       ??_C@_09DBEDLMHB@DialogRun?$AA@ 1000b9e8     service.obj
 0001:0000a9f4       ??_C@_0L@PJAHNOGM@DialogInit?$AA@ 1000b9f4     service.obj
 0001:0000aa00       ??_C@_0BC@BIIKJLKB@PluginStartupInfo?$AA@ 1000ba00     service.obj
 0001:0000aa14       ??_C@_0M@EICBHAOA@UpdatePanel?$AA@ 1000ba14     service.obj
 0001:0000aa20       ??_C@_0M@IENJPEBA@SetViewMode?$AA@ 1000ba20     service.obj
 0001:0000aa2c       ??_C@_0O@LHNNDOB@SetUserScreen?$AA@ 1000ba2c     service.obj
 0001:0000aa3c       ??_C@_0N@HCHLALN@SetSortOrder?$AA@ 1000ba3c     service.obj
 0001:0000aa4c       ??_C@_0M@CMMMGIDG@SetSortMode?$AA@ 1000ba4c     service.obj
 0001:0000aa58       ??_C@_0N@NMDFLOPL@SetSelection?$AA@ 1000ba58     service.obj
 0001:0000aa68       ??_C@_0BC@PDKEABHF@SetPanelDirectory?$AA@ 1000ba68     service.obj
 0001:0000aa7c       ??_C@_0P@NPNKOENM@SetNumericSort?$AA@ 1000ba7c     service.obj
 0001:0000aa8c       ??_C@_0BE@PAPEKLCP@SetDirectoriesFirst?$AA@ 1000ba8c     service.obj
 0001:0000aaa0       ??_C@_0BE@IPNAPCDL@SetCmdLineSelection?$AA@ 1000baa0     service.obj
 0001:0000aab4       ??_C@_0O@KECGHKDH@SetCmdLinePos?$AA@ 1000bab4     service.obj
 0001:0000aac4       ??_C@_0L@LAFNHJLF@SetCmdLine?$AA@ 1000bac4     service.obj
 0001:0000aad0       ??_C@_0BF@LKMKIFPG@SetCaseSensitiveSort?$AA@ 1000bad0     service.obj
 0001:0000aae8       ??_C@_0P@OPKJJMLB@SetActivePanel?$AA@ 1000bae8     service.obj
 0001:0000aaf8       ??_C@_0M@LCEPDNPK@RedrawPanel?$AA@ 1000baf8     service.obj
 0001:0000ab04       ??_C@_0O@OMMHIHHH@IsActivePanel?$AA@ 1000bb04     service.obj
 0001:0000ab14       ??_C@_0O@EHOCCHAL@InsertCmdLine?$AA@ 1000bb14     service.obj
 0001:0000ab24       ??_C@_0O@HEGDGAJG@GetUserScreen?$AA@ 1000bb24     service.obj
 0001:0000ab34       ??_C@_0BF@MEMFMMGB@GetSelectedPanelItem?$AA@ 1000bb34     service.obj
 0001:0000ab4c       ??_C@_0P@HCBKDPMP@GetPanelPrefix?$AA@ 1000bb4c     service.obj
 0001:0000ab5c       ??_C@_0N@HAFLAIHA@GetPanelItem?$AA@ 1000bb5c     service.obj
 0001:0000ab6c       ??_C@_0N@HPIPGDFA@GetPanelInfo?$AA@ 1000bb6c     service.obj
 0001:0000ab7c       ??_C@_0BB@LCMBHPNI@GetPanelHostFile?$AA@ 1000bb7c     service.obj
 0001:0000ab90       ??_C@_0P@GODLFFFJ@GetPanelFormat?$AA@ 1000bb90     service.obj
 0001:0000aba0       ??_C@_0BC@NGKPIKGL@GetPanelDirectory?$AA@ 1000bba0     service.obj
 0001:0000abb4       ??_C@_0BE@JPAIJBCI@GetCurrentPanelItem?$AA@ 1000bbb4     service.obj
 0001:0000abc8       ??_C@_0BA@DJGLDCBG@GetColumnWidths?$AA@ 1000bbc8     service.obj
 0001:0000abd8       ??_C@_0P@CMFANDFM@GetColumnTypes?$AA@ 1000bbd8     service.obj
 0001:0000abe8       ??_C@_0BE@CBPLLCEH@GetCmdLineSelection?$AA@ 1000bbe8     service.obj
 0001:0000abfc       ??_C@_0O@NLDIMJEA@GetCmdLinePos?$AA@ 1000bbfc     service.obj
 0001:0000ac0c       ??_C@_0L@KOHCMOPM@GetCmdLine?$AA@ 1000bc0c     service.obj
 0001:0000ac18       ??_C@_0P@DFBDDHFA@ClearSelection?$AA@ 1000bc18     service.obj
 0001:0000ac28       ??_C@_0BB@PJGDGIKA@CheckPanelsExist?$AA@ 1000bc28     service.obj
 0001:0000ac3c       ??_C@_06PJECNADJ@Viewer?$AA@ 1000bc3c     service.obj
 0001:0000ac44       ??_C@_07JMDLHPJF@SetMode?$AA@ 1000bc44     service.obj
 0001:0000ac4c       ??_C@_08IBJJAHJG@UndoRedo?$AA@ 1000bc4c     service.obj
 0001:0000ac58       ??_C@_09JFBCONJH@TabToReal?$AA@ 1000bc58     service.obj
 0001:0000ac64       ??_C@_0BF@LIMPGNED@SubscribeChangeEvent?$AA@ 1000bc64     service.obj
 0001:0000ac7c       ??_C@_08JNAOBKMI@GetTitle?$AA@ 1000bc7c     service.obj
 0001:0000ac88       ??_C@_08GMCCAJLF@SetTitle?$AA@ 1000bc88     service.obj
 0001:0000ac94       ??_C@_0L@JNHIIHDG@SetStringW?$AA@ 1000bc94     service.obj
 0001:0000aca0       ??_C@_09FPPPFNNC@SetString?$AA@ 1000bca0     service.obj
 0001:0000acac       ??_C@_0M@GKIFPNAD@SetPosition?$AA@ 1000bcac     service.obj
 0001:0000acb8       ??_C@_08CCKJEGOF@SetParam?$AA@ 1000bcb8     service.obj
 0001:0000acc4       ??_C@_09PPEOOGEC@SetKeyBar?$AA@ 1000bcc4     service.obj
 0001:0000acd0       ??_C@_06HJGPBJLE@Select?$AA@ 1000bcd0     service.obj
 0001:0000acd8       ??_C@_08FBDDPFPJ@SaveFile?$AA@ 1000bcd8     service.obj
 0001:0000ace4       ??_C@_06KAPLBEK@Redraw?$AA@ 1000bce4     service.obj
 0001:0000acec       ??_C@_09DBPLBJBJ@RealToTab?$AA@ 1000bcec     service.obj
 0001:0000acf8       ??_C@_09KINLOJJJ@ReadInput?$AA@ 1000bcf8     service.obj
 0001:0000ad04       ??_C@_04GMBKPCGK@Quit?$AA@ 1000bd04     service.obj
 0001:0000ad0c       ??_C@_0N@FNCEPAJJ@ProcessInput?$AA@ 1000bd0c     service.obj
 0001:0000ad1c       ??_C@_0BE@IEBIGOAP@PrevSessionBookmark?$AA@ 1000bd1c     service.obj
 0001:0000ad30       ??_C@_0BE@CNGODNDI@NextSessionBookmark?$AA@ 1000bd30     service.obj
 0001:0000ad44       ??_C@_0M@BINOKANK@InsertTextW?$AA@ 1000bd44     service.obj
 0001:0000ad50       ??_C@_0L@JMOIGJIA@InsertText?$AA@ 1000bd50     service.obj
 0001:0000ad5c       ??_C@_0N@ICPGLOEG@InsertString?$AA@ 1000bd5c     service.obj
 0001:0000ad6c       ??_C@_0L@IDFHDAHP@GetStringW?$AA@ 1000bd6c     service.obj
 0001:0000ad78       ??_C@_09HBLKHMEA@GetString?$AA@ 1000bd78     service.obj
 0001:0000ad84       ??_C@_0BE@LBJJGOGD@GetSessionBookmarks?$AA@ 1000bd84     service.obj
 0001:0000ad98       ??_C@_0N@KIILHCLH@GetSelection?$AA@ 1000bd98     service.obj
 0001:0000ada8       ??_C@_07NAJNLNAF@GetInfo?$AA@ 1000bda8     service.obj
 0001:0000adb0       ??_C@_0M@FECPLAMN@GetFileName?$AA@ 1000bdb0     service.obj
 0001:0000adbc       ??_C@_08JOPFJIPE@GetColor?$AA@ 1000bdbc     service.obj
 0001:0000adc8       ??_C@_0N@MGAOADJN@GetBookmarks?$AA@ 1000bdc8     service.obj
 0001:0000add8       ??_C@_0L@HDLPOLMA@ExpandTabs?$AA@ 1000bdd8     service.obj
 0001:0000ade4       ??_C@_06MJDIICIN@Editor?$AA@ 1000bde4     service.obj
 0001:0000adec       ??_C@_0N@EKENACAE@DeleteString?$AA@ 1000bdec     service.obj
 0001:0000adfc       ??_C@_0BG@KOELEFCN@DeleteSessionBookmark?$AA@ 1000bdfc     service.obj
 0001:0000ae14       ??_C@_0L@BCLIBKOC@DeleteChar?$AA@ 1000be14     service.obj
 0001:0000ae20       ??_C@_0M@LPIECDD@DeleteBlock?$AA@ 1000be20     service.obj
 0001:0000ae2c       ??_C@_08PDEJHGJI@DelColor?$AA@ 1000be2c     service.obj
 0001:0000ae38       ??_C@_0BG@IGFHDIIN@ClearSessionBookmarks?$AA@ 1000be38     service.obj
 0001:0000ae50       ??_C@_0BD@DOFEEDDC@AddSessionBookmark?$AA@ 1000be50     service.obj
 0001:0000ae64       ??_C@_08EGJLHNCO@AddColor?$AA@ 1000be64     service.obj
 0001:0000ae70       ??_C@_0L@CPCKAMD@OpenSubkey?$AA@ 1000be70     service.obj
 0001:0000ae7c       ??_C@_0N@OELJMCEC@CreateSubkey?$AA@ 1000be7c     service.obj
 0001:0000ae8c       ??_C@_03CEMDFJG@Set?$AA@   1000be8c     service.obj
 0001:0000ae90       ??_C@_03NNDHPFFO@Get?$AA@  1000be90     service.obj
 0001:0000ae94       ??_C@_04HJMOFLDF@Free?$AA@ 1000be94     service.obj
 0001:0000ae9c       ??_C@_04PAFOOALK@Enum?$AA@ 1000be9c     service.obj
 0001:0000aea4       ??_C@_06JBKGCNBB@Delete?$AA@ 1000bea4     service.obj
 0001:0000aeac       ??_C@_04MIIPNNEF@send?$AA@ 1000beac     service.obj
 0001:0000aeb4       ??_C@_09LDLEBFOB@rawhandle?$AA@ 1000beb4     service.obj
 0001:0000aec0       ??_C@_0P@JDMCHDIM@IsFileInFilter?$AA@ 1000bec0     service.obj
 0001:0000aed0       ??_C@_0BB@OPPOFOAK@StartingToFilter?$AA@ 1000bed0     service.obj
 0001:0000aee4       ??_C@_0BA@JGEOEAE@OpenFiltersMenu?$AA@ 1000bee4     service.obj
 0001:0000aef4       ??_C@_0P@LKPINHLK@FreeFileFilter?$AA@ 1000bef4     service.obj
 0001:0000af04       ??_C@_09MBBEHOCK@OEM_CLEAR?$AA@ 1000bf04     service.obj
 0001:0000af10       ??_C@_03KCLDMPAE@PA1?$AA@  1000bf10     service.obj
 0001:0000af14       ??_C@_06LJIOOKLP@NONAME?$AA@ 1000bf14     service.obj
 0001:0000af1c       ??_C@_04LGBIGMFG@ZOOM?$AA@ 1000bf1c     service.obj
 0001:0000af24       ??_C@_04MKCNCBEG@PLAY?$AA@ 1000bf24     service.obj
 0001:0000af2c       ??_C@_05CCFENDFJ@EREOF?$AA@ 1000bf2c     service.obj
 0001:0000af34       ??_C@_05OKOOKOOH@EXSEL?$AA@ 1000bf34     service.obj
 0001:0000af3c       ??_C@_05HGAHFFFL@CRSEL?$AA@ 1000bf3c     service.obj
 0001:0000af44       ??_C@_04BNGOAFAJ@ATTN?$AA@ 1000bf44     service.obj
 0001:0000af4c       ??_C@_0L@OCAIHDP@OEM_WSCTRL?$AA@ 1000bf4c     service.obj
 0001:0000af58       ??_C@_07DLOIGGME@OEM_PA3?$AA@ 1000bf58     service.obj
 0001:0000af60       ??_C@_07CCPDFHIF@OEM_PA2?$AA@ 1000bf60     service.obj
 0001:0000af68       ??_C@_07JNOAEEG@OEM_PA1?$AA@ 1000bf68     service.obj
 0001:0000af70       ??_C@_08INMNLJCK@OEM_JUMP?$AA@ 1000bf70     service.obj
 0001:0000af7c       ??_C@_09CAKPMKHM@OEM_RESET?$AA@ 1000bf7c     service.obj
 0001:0000af88       ??_C@_06HOICDKCB@PACKET?$AA@ 1000bf88     service.obj
 0001:0000af90       ??_C@_0L@EFLJCPAM@PROCESSKEY?$AA@ 1000bf90     service.obj
 0001:0000af9c       ??_C@_07PEFKMFIE@OEM_102?$AA@ 1000bf9c     service.obj
 0001:0000afa4       ??_C@_05DJCBGEEK@OEM_8?$AA@ 1000bfa4     service.obj
 0001:0000afac       ??_C@_05LOLJHIIF@OEM_7?$AA@ 1000bfac     service.obj
 0001:0000afb4       ??_C@_05KHKCEJME@OEM_6?$AA@ 1000bfb4     service.obj
 0001:0000afbc       ??_C@_05IMIPBKAH@OEM_5?$AA@ 1000bfbc     service.obj
 0001:0000afc4       ??_C@_05JFJECLEG@OEM_4?$AA@ 1000bfc4     service.obj
 0001:0000afcc       ??_C@_05NKNFLNIB@OEM_3?$AA@ 1000bfcc     service.obj
 0001:0000afd4       ??_C@_05MDMOIMMA@OEM_2?$AA@ 1000bfd4     service.obj
 0001:0000afdc       ??_C@_0L@DNNMNDGM@OEM_PERIOD?$AA@ 1000bfdc     service.obj
 0001:0000afe8       ??_C@_09OGMLCNMG@OEM_MINUS?$AA@ 1000bfe8     service.obj
 0001:0000aff4       ??_C@_09CLPFJEOD@OEM_COMMA?$AA@ 1000bff4     service.obj
 0001:0000b000       ??_C@_08LDJEIPBH@OEM_PLUS?$AA@ 1000c000     service.obj
 0001:0000b00c       ??_C@_05OIODNPAD@OEM_1?$AA@ 1000c00c     service.obj
 0001:0000b014       ??_C@_0M@ONJENAPP@LAUNCH_APP2?$AA@ 1000c014     service.obj
 0001:0000b020       ??_C@_0M@MGLJIDDM@LAUNCH_APP1?$AA@ 1000c020     service.obj
 0001:0000b02c       ??_C@_0BE@FADJJAPM@LAUNCH_MEDIA_SELECT?$AA@ 1000c02c     service.obj
 0001:0000b040       ??_C@_0M@GCIKMBID@LAUNCH_MAIL?$AA@ 1000c040     service.obj
 0001:0000b04c       ??_C@_0BB@HAEMIJHO@MEDIA_PLAY_PAUSE?$AA@ 1000c04c     service.obj
 0001:0000b060       ??_C@_0L@KBJOCDHK@MEDIA_STOP?$AA@ 1000c060     service.obj
 0001:0000b06c       ??_C@_0BB@CMOIJKPH@MEDIA_PREV_TRACK?$AA@ 1000c06c     service.obj
 0001:0000b080       ??_C@_0BB@KLAENPA@MEDIA_NEXT_TRACK?$AA@ 1000c080     service.obj
 0001:0000b094       ??_C@_09MGPMNMJC@VOLUME_UP?$AA@ 1000c094     service.obj
 0001:0000b0a0       ??_C@_0M@JOOBBDNO@VOLUME_DOWN?$AA@ 1000c0a0     service.obj
 0001:0000b0ac       ??_C@_0M@ENOHKBMG@VOLUME_MUTE?$AA@ 1000c0ac     service.obj
 0001:0000b0b8       ??_C@_0N@NOOKCEKA@BROWSER_HOME?$AA@ 1000c0b8     service.obj
 0001:0000b0c8       ??_C@_0BC@BOMJIH@BROWSER_FAVORITES?$AA@ 1000c0c8     service.obj
 0001:0000b0dc       ??_C@_0P@BEAEBJDD@BROWSER_SEARCH?$AA@ 1000c0dc     service.obj
 0001:0000b0ec       ??_C@_0N@HKPDGANH@BROWSER_STOP?$AA@ 1000c0ec     service.obj
 0001:0000b0fc       ??_C@_0BA@GDNDIDGJ@BROWSER_REFRESH?$AA@ 1000c0fc     service.obj
 0001:0000b10c       ??_C@_0BA@ENOAJOGH@BROWSER_FORWARD?$AA@ 1000c10c     service.obj
 0001:0000b11c       ??_C@_0N@OAJIELLG@BROWSER_BACK?$AA@ 1000c11c     service.obj
 0001:0000b12c       ??_C@_05LOBKMKIM@RMENU?$AA@ 1000c12c     service.obj
 0001:0000b134       ??_C@_05IHMGKJGH@LMENU?$AA@ 1000c134     service.obj
 0001:0000b13c       ??_C@_08OOMMENPF@RCONTROL?$AA@ 1000c13c     service.obj
 0001:0000b148       ??_C@_08IKMONEBG@LCONTROL?$AA@ 1000c148     service.obj
 0001:0000b154       ??_C@_06HIJMMPFL@RSHIFT?$AA@ 1000c154     service.obj
 0001:0000b15c       ??_C@_06EPHNCIMI@LSHIFT?$AA@ 1000c15c     service.obj
 0001:0000b164       ??_C@_0M@FOJHECMP@OEM_FJ_ROYA?$AA@ 1000c164     service.obj
 0001:0000b170       ??_C@_0M@IBEHGLCM@OEM_FJ_LOYA?$AA@ 1000c170     service.obj
 0001:0000b17c       ??_C@_0P@NIEOFNLG@OEM_FJ_TOUROKU?$AA@ 1000c17c     service.obj
 0001:0000b18c       ??_C@_0P@JKGCFGCD@OEM_FJ_MASSHOU?$AA@ 1000c18c     service.obj
 0001:0000b19c       ??_C@_0O@DBBJDALK@OEM_NEC_EQUAL?$AA@ 1000c19c     service.obj
 0001:0000b1ac       ??_C@_06FNIKALAE@SCROLL?$AA@ 1000c1ac     service.obj
 0001:0000b1b4       ??_C@_07FLMEHHJP@NUMLOCK?$AA@ 1000c1b4     service.obj
 0001:0000b1bc       ??_C@_03PMABOFAL@F24?$AA@  1000c1bc     service.obj
 0001:0000b1c0       ??_C@_03LDEAHDMM@F23?$AA@  1000c1c0     service.obj
 0001:0000b1c4       ??_C@_03KKFLECIN@F22?$AA@  1000c1c4     service.obj
 0001:0000b1c8       ??_C@_03IBHGBBEO@F21?$AA@  1000c1c8     service.obj
 0001:0000b1cc       ??_C@_03JIGNCAAP@F20?$AA@  1000c1cc     service.obj
 0001:0000b1d0       ??_C@_03ELOJCFBP@F19?$AA@  1000c1d0     service.obj
 0001:0000b1d4       ??_C@_03FCPCBEFO@F18?$AA@  1000c1d4     service.obj
 0001:0000b1d8       ??_C@_03NFGKAIJB@F17?$AA@  1000c1d8     service.obj
 0001:0000b1dc       ??_C@_03MMHBDJNA@F16?$AA@  1000c1dc     service.obj
 0001:0000b1e0       ??_C@_03OHFMGKBD@F15?$AA@  1000c1e0     service.obj
 0001:0000b1e4       ??_C@_03POEHFLFC@F14?$AA@  1000c1e4     service.obj
 0001:0000b1e8       ??_C@_03LBAGMNJF@F13?$AA@  1000c1e8     service.obj
 0001:0000b1ec       ??_C@_03KIBNPMNE@F12?$AA@  1000c1ec     service.obj
 0001:0000b1f0       ??_C@_03IDDAKPBH@F11?$AA@  1000c1f0     service.obj
 0001:0000b1f4       ??_C@_03JKCLJOFG@F10?$AA@  1000c1f4     service.obj
 0001:0000b1f8       ??_C@_02HKCNFKCF@F9?$AA@   1000c1f8     service.obj
 0001:0000b1fc       ??_C@_02GDDGGLGE@F8?$AA@   1000c1fc     service.obj
 0001:0000b200       ??_C@_02OEKOHHKL@F7?$AA@   1000c200     service.obj
 0001:0000b204       ??_C@_02PNLFEGOK@F6?$AA@   1000c204     service.obj
 0001:0000b208       ??_C@_02NGJIBFCJ@F5?$AA@   1000c208     service.obj
 0001:0000b20c       ??_C@_02MPIDCEGI@F4?$AA@   1000c20c     service.obj
 0001:0000b210       ??_C@_02IAMCLCKP@F3?$AA@   1000c210     service.obj
 0001:0000b214       ??_C@_02JJNJIDOO@F2?$AA@   1000c214     service.obj
 0001:0000b218       ??_C@_02LCPENACN@F1?$AA@   1000c218     service.obj
 0001:0000b21c       ??_C@_06FBFCJJMP@DIVIDE?$AA@ 1000c21c     service.obj
 0001:0000b224       ??_C@_07LJPMJDLL@DECIMAL?$AA@ 1000c224     service.obj
 0001:0000b22c       ??_C@_08MGBEENML@SUBTRACT?$AA@ 1000c22c     service.obj
 0001:0000b238       ??_C@_09POPINEFK@SEPARATOR?$AA@ 1000c238     service.obj
 0001:0000b244       ??_C@_03BOJFLAKG@ADD?$AA@  1000c244     service.obj
 0001:0000b248       ??_C@_08LDEOAAGM@MULTIPLY?$AA@ 1000c248     service.obj
 0001:0000b254       ??_C@_07GENHHNO@NUMPAD9?$AA@ 1000c254     service.obj
 0001:0000b25c       ??_C@_07BPFGEGJP@NUMPAD8?$AA@ 1000c25c     service.obj
 0001:0000b264       ??_C@_07JIMOFKFA@NUMPAD7?$AA@ 1000c264     service.obj
 0001:0000b26c       ??_C@_07IBNFGLBB@NUMPAD6?$AA@ 1000c26c     service.obj
 0001:0000b274       ??_C@_07KKPIDINC@NUMPAD5?$AA@ 1000c274     service.obj
 0001:0000b27c       ??_C@_07LDODAJJD@NUMPAD4?$AA@ 1000c27c     service.obj
 0001:0000b284       ??_C@_07PMKCJPFE@NUMPAD3?$AA@ 1000c284     service.obj
 0001:0000b28c       ??_C@_07OFLJKOBF@NUMPAD2?$AA@ 1000c28c     service.obj
 0001:0000b294       ??_C@_07MOJEPNNG@NUMPAD1?$AA@ 1000c294     service.obj
 0001:0000b29c       ??_C@_07NHIPMMJH@NUMPAD0?$AA@ 1000c29c     service.obj
 0001:0000b2a4       ??_C@_05DJAECLDN@SLEEP?$AA@ 1000c2a4     service.obj
 0001:0000b2ac       ??_C@_04GKGJFGJO@APPS?$AA@ 1000c2ac     service.obj
 0001:0000b2b4       ??_C@_04DMGFHHJG@RWIN?$AA@ 1000c2b4     service.obj
 0001:0000b2bc       ??_C@_04ODLFFOHF@LWIN?$AA@ 1000c2bc     service.obj
 0001:0000b2c4       ??_C@_01POHCFINO@Z?$AA@    1000c2c4     service.obj
 0001:0000b2c8       ??_C@_01NFFPALBN@Y?$AA@    1000c2c8     service.obj
 0001:0000b2cc       ??_C@_01MMEEDKFM@X?$AA@    1000c2cc     service.obj
 0001:0000b2d0       ??_C@_01ELNMCGJD@W?$AA@    1000c2d0     service.obj
 0001:0000b2d4       ??_C@_01FCMHBHNC@V?$AA@    1000c2d4     service.obj
 0001:0000b2d8       ??_C@_01HJOKEEBB@U?$AA@    1000c2d8     service.obj
 0001:0000b2dc       ??_C@_01GAPBHFFA@T?$AA@    1000c2dc     service.obj
 0001:0000b2e0       ??_C@_01CPLAODJH@S?$AA@    1000c2e0     service.obj
 0001:0000b2e4       ??_C@_01DGKLNCNG@R?$AA@    1000c2e4     service.obj
 0001:0000b2e8       ??_C@_01BNIGIBBF@Q?$AA@    1000c2e8     service.obj
 0001:0000b2ec       ??_C@_01EJNLAFE@P?$AA@     1000c2ec     service.obj
 0001:0000b2f0       ??_C@_01MJMHLOMK@O?$AA@    1000c2f0     service.obj
 0001:0000b2f4       ??_C@_01NANMIPIL@N?$AA@    1000c2f4     service.obj
 0001:0000b2f8       ??_C@_01PLPBNMEI@M?$AA@    1000c2f8     service.obj
 0001:0000b2fc       ??_C@_01OCOKONAJ@L?$AA@    1000c2fc     service.obj
 0001:0000b300       ??_C@_01KNKLHLMO@K?$AA@    1000c300     service.obj
 0001:0000b304       ??_C@_01LELAEKIP@J?$AA@    1000c304     service.obj
 0001:0000b308       ??_C@_01JPJNBJEM@I?$AA@    1000c308     service.obj
 0001:0000b30c       ??_C@_01IGIGCIAN@H?$AA@    1000c30c     service.obj
 0001:0000b310       ??_C@_01BBODEMC@G?$AA@     1000c310     service.obj
 0001:0000b314       ??_C@_01BIAFAFID@F?$AA@    1000c314     service.obj
 0001:0000b318       ??_C@_01DDCIFGEA@E?$AA@    1000c318     service.obj
 0001:0000b31c       ??_C@_01CKDDGHAB@D?$AA@    1000c31c     service.obj
 0001:0000b320       ??_C@_01GFHCPBMG@C?$AA@    1000c320     service.obj
 0001:0000b324       ??_C@_01HMGJMAIH@B?$AA@    1000c324     service.obj
 0001:0000b328       ??_C@_01FHEEJDEE@A?$AA@    1000c328     service.obj
 0001:0000b32c       ??_C@_01LAKCGALK@9?$AA@    1000c32c     service.obj
 0001:0000b330       ??_C@_01KJLJFBPL@8?$AA@    1000c330     service.obj
 0001:0000b334       ??_C@_01COCBENDE@7?$AA@    1000c334     service.obj
 0001:0000b338       ??_C@_01DHDKHMHF@6?$AA@    1000c338     service.obj
 0001:0000b33c       ??_C@_01BMBHCPLG@5?$AA@    1000c33c     service.obj
 0001:0000b340       ??_C@_01FAMBOPH@4?$AA@     1000c340     service.obj
 0001:0000b344       ??_C@_01EKENIIDA@3?$AA@    1000c344     service.obj
 0001:0000b348       ??_C@_01FDFGLJHB@2?$AA@    1000c348     service.obj
 0001:0000b34c       ??_C@_01HIHLOKLC@1?$AA@    1000c34c     service.obj
 0001:0000b350       ??_C@_01GBGANLPD@0?$AA@    1000c350     service.obj
 0001:0000b354       ??_C@_04DOKPJKJF@HELP?$AA@ 1000c354     service.obj
 0001:0000b35c       ??_C@_06FKDAMKFP@DELETE?$AA@ 1000c35c     service.obj
 0001:0000b364       ??_C@_06OEMEAEKN@INSERT?$AA@ 1000c364     service.obj
 0001:0000b36c       ??_C@_08EMOKHGD@SNAPSHOT?$AA@ 1000c36c     service.obj
 0001:0000b378       ??_C@_07LBDEDADF@EXECUTE?$AA@ 1000c378     service.obj
 0001:0000b380       ??_C@_05ECKPOFCN@PRINT?$AA@ 1000c380     service.obj
 0001:0000b388       ??_C@_06LCPJPOPK@SELECT?$AA@ 1000c388     service.obj
 0001:0000b390       ??_C@_04FANAOELO@DOWN?$AA@ 1000c390     service.obj
 0001:0000b398       ??_C@_05PMAFOJDE@RIGHT?$AA@ 1000c398     service.obj
 0001:0000b3a0       ??_C@_02NAHCJHOC@UP?$AA@   1000c3a0     service.obj
 0001:0000b3a4       ??_C@_04KCNEHMIH@LEFT?$AA@ 1000c3a4     service.obj
 0001:0000b3ac       ??_C@_04GHGFPGNC@HOME?$AA@ 1000c3ac     service.obj
 0001:0000b3b4       ??_C@_03JMGAKCCH@END?$AA@  1000c3b4     service.obj
 0001:0000b3b8       ??_C@_04MOKMKBJN@NEXT?$AA@ 1000c3b8     service.obj
 0001:0000b3c0       ??_C@_05BFDHCIJM@PRIOR?$AA@ 1000c3c0     service.obj
 0001:0000b3c8       ??_C@_05CAEOFMEP@SPACE?$AA@ 1000c3c8     service.obj
 0001:0000b3d0       ??_C@_0L@HEHNEBED@MODECHANGE?$AA@ 1000c3d0     service.obj
 0001:0000b3dc       ??_C@_06INBBKPI@ACCEPT?$AA@ 1000c3dc     service.obj
 0001:0000b3e4       ??_C@_0L@ODNCKDCK@NONCONVERT?$AA@ 1000c3e4     service.obj
 0001:0000b3f0       ??_C@_06CDPDIIDH@ESCAPE?$AA@ 1000c3f0     service.obj
 0001:0000b3f8       ??_C@_05CHABPOPI@HANJA?$AA@ 1000c3f8     service.obj
 0001:0000b400       ??_C@_05JEIAEFOF@FINAL?$AA@ 1000c400     service.obj
 0001:0000b408       ??_C@_05PPKJGOLB@JUNJA?$AA@ 1000c408     service.obj
 0001:0000b410       ??_C@_04KGDAIAGM@KANA?$AA@ 1000c410     service.obj
 0001:0000b418       ??_C@_07OPCFNGJB@CAPITAL?$AA@ 1000c418     service.obj
 0001:0000b420       ??_C@_05DIAHPDGL@PAUSE?$AA@ 1000c420     service.obj
 0001:0000b428       ??_C@_04IILMDFMO@MENU?$AA@ 1000c428     service.obj
 0001:0000b430       ??_C@_07DBEDOPMC@CONTROL?$AA@ 1000c430     service.obj
 0001:0000b438       ??_C@_05OAHIEJBI@SHIFT?$AA@ 1000c438     service.obj
 0001:0000b440       ??_C@_06LJMOENAO@RETURN?$AA@ 1000c440     service.obj
 0001:0000b448       ??_C@_05PONODPI@CLEAR?$AA@ 1000c448     service.obj
 0001:0000b450       ??_C@_03CJMDHCGG@TAB?$AA@  1000c450     service.obj
 0001:0000b454       ??_C@_04FJBHJJME@BACK?$AA@ 1000c454     service.obj
 0001:0000b45c       ??_C@_08MEKGJEIF@XBUTTON2?$AA@ 1000c45c     service.obj
 0001:0000b468       ??_C@_08OPILMHEG@XBUTTON1?$AA@ 1000c468     service.obj
 0001:0000b474       ??_C@_07DLFCFDDG@MBUTTON?$AA@ 1000c474     service.obj
 0001:0000b47c       ??_C@_06JHILMIHF@CANCEL?$AA@ 1000c47c     service.obj
 0001:0000b484       ??_C@_07JOMJHALB@RBUTTON?$AA@ 1000c484     service.obj
 0001:0000b48c       ??_C@_07PHPIFDKI@LBUTTON?$AA@ 1000c48c     service.obj
 0001:0000bcc0       _FarFileFilterType         1000ccc0     service.obj
 0001:0000bcd0       _FarTimerType              1000ccd0     service.obj
 0001:0000bcdc       _FarDialogType             1000ccdc     service.obj
 0001:0000bce8       _SettingsType              1000cce8     service.obj
 0001:0000bcf4       _SettingsHandles           1000ccf4     service.obj
 0001:0000bd08       _PluginHandleType          1000cd08     service.obj
 0001:0000bd18       _AddMacroDataType          1000cd18     service.obj
 0001:0000bd28       _SavedScreenType           1000cd28     service.obj
 0001:0000bd38       _FAR_VIRTUALKEYS           1000cd38     service.obj
 0001:0000bd48       _FAR_FLAGSTABLE            1000cd48     service.obj
 0001:0000bd54       _FAR_DN_STORAGE            1000cd54     service.obj
 0001:0000bd94       _timer_methods             1000cd94     service.obj
 0001:0000bdbc       _filefilter_methods        1000cdbc     service.obj
 0001:0000bdf4       _dialog_methods            1000cdf4     service.obj
 0001:0000be20       _Settings_methods          1000ce20     service.obj
 0001:0000be70       _editor_funcs              1000ce70     service.obj
 0001:0000bfb8       _viewer_funcs              1000cfb8     service.obj
 0001:0000c008       _panel_funcs               1000d008     service.obj
 0001:0000c120       _far_funcs                 1000d120     service.obj
 0001:0000c360       _far_Dialog                1000d360     service.obj
 0001:0000c5f0       _api_functions             1000d5f0     service.obj
 0001:0000c650       ??_C@_0M@DOFFFIEL@luaopen_jit?$AA@ 1000d650     service.obj
 0001:0000c65c       ??_C@_0M@IALDMMNC@luaopen_ffi?$AA@ 1000d65c     service.obj
 0001:0000c668       ??_C@_0M@PLOBHAKE@luaopen_bit?$AA@ 1000d668     service.obj
 0001:0000c674       ??_C@_09GJGOMOL@lua51?4dll?$AA@ 1000d674     service.obj
 0001:0000c680       ??_C@_0BE@OEPKKAAB@integer?5or?5userdata?$AA@ 1000d680     service.obj
 0001:0000c694       ??_C@_0N@JJLBBDOC@invalid?5flag?$AA@ 1000d694     service.obj
 0001:0000c6a4       ??_C@_0BJ@MIKGPOKL@invalid?5flag?5combination?$AA@ 1000d6a4     service.obj
 0001:0000c6c0       ??_C@_0L@EMFBJIPA@EventFlags?$AA@ 1000d6c0     service.obj
 0001:0000c6cc       ??_C@_0M@BJAICPIE@ButtonState?$AA@ 1000d6cc     service.obj
 0001:0000c6d8       ??_C@_0P@FJMHICKO@MousePositionY?$AA@ 1000d6d8     service.obj
 0001:0000c6e8       ??_C@_0P@EANMLDOP@MousePositionX?$AA@ 1000d6e8     service.obj
 0001:0000c6f8       __real@41f0000000000000    1000d6f8     service.obj
 0001:0000c700       ??_C@_08LLJICOLD@Overtype?$AA@ 1000d700     service.obj
 0001:0000c70c       ??_C@_07GDAKJHLE@LeftPos?$AA@ 1000d70c     service.obj
 0001:0000c714       ??_C@_0O@OKGGHEJK@TopScreenLine?$AA@ 1000d714     service.obj
 0001:0000c724       ??_C@_09EGONKHKB@CurTabPos?$AA@ 1000d724     service.obj
 0001:0000c730       ??_C@_06EDBJMJDC@CurPos?$AA@ 1000d730     service.obj
 0001:0000c738       ??_C@_07EEJLMCNH@CurLine?$AA@ 1000d738     service.obj
 0001:0000c740       ??_C@_0L@JLHCLFBG@PluginGuid?$AA@ 1000d740     service.obj
 0001:0000c74c       ??_C@_09HOIHBHIM@ModuleDir?$AA@ 1000d74c     service.obj
 0001:0000c758       ??_C@_0L@GEIEADPN@ModuleName?$AA@ 1000d758     service.obj
 0001:0000c764       ??_C@_08CPAOHJDL@CurState?$AA@ 1000d764     service.obj
 0001:0000c770       ??_C@_0BF@ODFKBFAK@SessionBookmarkCount?$AA@ 1000d770     service.obj
 0001:0000c788       ??_C@_0O@EBLDFOPH@BookmarkCount?$AA@ 1000d788     service.obj
 0001:0000c798       ??_C@_07FLDNELFM@TabSize?$AA@ 1000d798     service.obj
 0001:0000c7a0       ??_C@_07KHIHFBFN@Options?$AA@ 1000d7a0     service.obj
 0001:0000c7a8       ??_C@_0P@GAEEHNHE@BlockStartLine?$AA@ 1000d7a8     service.obj
 0001:0000c7b8       ??_C@_09HKBEFIPN@BlockType?$AA@ 1000d7b8     service.obj
 0001:0000c7c8       __real@3ff0000000000000    1000d7c8     service.obj
 0001:0000c7d0       ??_C@_0L@PMKENHMA@TotalLines?$AA@ 1000d7d0     service.obj
 0001:0000c7dc       ??_C@_0M@DGCKFKDM@WindowSizeY?$AA@ 1000d7dc     service.obj
 0001:0000c7e8       ??_C@_0M@CPDBGLHN@WindowSizeX?$AA@ 1000d7e8     service.obj
 0001:0000c7f4       ??_C@_08GGMFPBHM@EditorID?$AA@ 1000d7f4     service.obj
 0001:0000c800       ??_C@_09IBGOAAEM@StringEOL?$AA@ 1000d800     service.obj
 0001:0000c80c       ??_C@_0L@IFNFGDGN@StringText?$AA@ 1000d80c     service.obj
 0001:0000c818       ??_C@_06JLEHDHII@SelEnd?$AA@ 1000d818     service.obj
 0001:0000c820       ??_C@_08JPMALCFA@SelStart?$AA@ 1000d820     service.obj
 0001:0000c82c       ??_C@_0N@DAJMJAE@StringLength?$AA@ 1000d82c     service.obj
 0001:0000c83c       ??_C@_0CG@LAKEGANL@must?5be?5?8redraw?8?0?5?8restore?8?0?5or?5@ 1000d83c     service.obj
 0001:0000c864       ??_C@_07HICINA@restore?$AA@ 1000d864     service.obj
 0001:0000c86c       ??_C@_06MFLCIING@redraw?$AA@ 1000d86c     service.obj
 0001:0000c874       ??_C@_0L@GDDEHGKI@ScreenLine?$AA@ 1000d874     service.obj
 0001:0000c880       ??_C@_06OIIFPIKD@Cursor?$AA@ 1000d880     service.obj
 0001:0000c888       ??_C@_04LIDDHMOL@Line?$AA@ 1000d888     service.obj
 0001:0000c890       ??_C@_0M@NKKGBDGK@BlockHeight?$AA@ 1000d890     service.obj
 0001:0000c89c       ??_C@_0L@EKLJJHPF@BlockWidth?$AA@ 1000d89c     service.obj
 0001:0000c8a8       ??_C@_0O@CIAFMMMB@BlockStartPos?$AA@ 1000d8a8     service.obj
 0001:0000c8b8       ??_C@_06KGHIGMHC@EndPos?$AA@ 1000d8b8     service.obj
 0001:0000c8c0       ??_C@_07DCKCOCOC@EndLine?$AA@ 1000d8c0     service.obj
 0001:0000c8c8       ??_C@_08JBNOANJG@StartPos?$AA@ 1000d8c8     service.obj
 0001:0000c8d4       ??_C@_09JFPCGCOC@StartLine?$AA@ 1000d8d4     service.obj
 0001:0000c8e0       ??_C@_0BA@DPMBBMBG@BackgroundColor?$AA@ 1000d8e0     service.obj
 0001:0000c8f0       ??_C@_0BA@HNIJJEO@ForegroundColor?$AA@ 1000d8f0     service.obj
 0001:0000c900       ??_C@_0O@NHKEGDJF@GUID?5required?$AA@ 1000d900     service.obj
 0001:0000c910       __real@41e0000000000000    1000d910     service.obj
 0001:0000c918       ??_C@_0BJ@BMOGHFAN@table?5or?5number?5expected?$AA@ 1000d918     service.obj
 0001:0000c934       ??_C@_05PDOBBJNA@Color?$AA@ 1000d934     service.obj
 0001:0000c93c       ??_C@_08KGEIBGG@Priority?$AA@ 1000d93c     service.obj
 0001:0000c948       ??_C@_08GPNNBNIL@SetFocus?$AA@ 1000d948     service.obj
 0001:0000c954       ??_C@_09GEJJJAHL@CommandId?$AA@ 1000d954     service.obj
 0001:0000c960       ??_C@_05HBOCJOBH@SizeY?$AA@ 1000d960     service.obj
 0001:0000c968       ??_C@_05GIPJKPFG@SizeX?$AA@ 1000d968     service.obj
 0001:0000c970       ??_C@_0M@PBJKDIHH@UnicodeChar?$AA@ 1000d970     service.obj
 0001:0000c97c       ??_C@_0BA@KCCLHPM@VirtualScanCode?$AA@ 1000d97c     service.obj
 0001:0000c98c       ??_C@_0M@FGGHEADP@RepeatCount?$AA@ 1000d98c     service.obj
 0001:0000c998       ??_C@_07HPHPOAEG@KeyDown?$AA@ 1000d998     service.obj
 0001:0000c9a0       ??_C@_09KDLBEGCN@EventType?$AA@ 1000d9a0     service.obj
 0001:0000c9ac       ??_C@_0M@BEDENHPD@invalid?5key?$AA@ 1000d9ac     service.obj
 0001:0000c9b8       ??_C@_08PNHLLJE@BreakKey?$AA@ 1000d9b8     service.obj
 0001:0000c9c4       ??_C@_08MMCKBNNI@AccelKey?$AA@ 1000d9c4     service.obj
 0001:0000c9d0       ??_C@_06JIKFICKK@hidden?$AA@ 1000d9d0     service.obj
 0001:0000c9d8       ??_C@_06JHIAOIKD@grayed?$AA@ 1000d9d8     service.obj
 0001:0000c9e0       ??_C@_07DBNODEFN@disable?$AA@ 1000d9e0     service.obj
 0001:0000c9e8       ??_C@_09MOAJOJKN@separator?$AA@ 1000d9e8     service.obj
 0001:0000c9f4       ??_C@_07FJOBMBFC@checked?$AA@ 1000d9f4     service.obj
 0001:0000c9fc       ??_C@_02HOGEDOAB@Id?$AA@   1000d9fc     service.obj
 0001:0000ca00       ??_C@_0M@GGMLPAIK@SelectIndex?$AA@ 1000da00     service.obj
 0001:0000ca0c       ??_C@_09CFELDMD@HelpTopic?$AA@ 1000da0c     service.obj
 0001:0000ca18       ??_C@_06DDHCBBGN@Bottom?$AA@ 1000da18     service.obj
 0001:0000ca20       ??_C@_09FDAFFNEA@MaxHeight?$AA@ 1000da20     service.obj
 0001:0000ca2c       ??_C@_0BF@OOLFJKGP@must?5be?5table?5or?5nil?$AA@ 1000da2c     service.obj
 0001:0000ca44       ??_C@_19IBCFILMC@?$AAM?$AAe?$AAn?$AAu?$AA?$AA@ 1000da44     service.obj
 0001:0000ca50       ??_C@_1BI@KMMIHPHF@?$AAR?$AAe?$AAt?$AAr?$AAy?$AAC?$AAa?$AAn?$AAc?$AAe?$AAl?$AA?$AA@ 1000da50     service.obj
 0001:0000ca68       ??_C@_1BI@BNDFIGCI@?$AAY?$AAe?$AAs?$AAN?$AAo?$AAC?$AAa?$AAn?$AAc?$AAe?$AAl?$AA?$AA@ 1000da68     service.obj
 0001:0000ca80       ??_C@_1M@GGPOIMAD@?$AAY?$AAe?$AAs?$AAN?$AAo?$AA?$AA@ 1000da80     service.obj
 0001:0000ca8c       ??_C@_1CC@HODOHOHB@?$AAA?$AAb?$AAo?$AAr?$AAt?$AAR?$AAe?$AAt?$AAr?$AAy?$AAI?$AAg?$AAn?$AAo?$AAr?$AAe?$AA?$AA@ 1000da8c     service.obj
 0001:0000cab0       ??_C@_1BC@IBCAPFAE@?$AAO?$AAk?$AAC?$AAa?$AAn?$AAc?$AAe?$AAl?$AA?$AA@ 1000dab0     service.obj
 0001:0000cac4       ??_C@_15FMBEJGOH@?$AAO?$AAk?$AA?$AA@ 1000dac4     service.obj
 0001:0000cacc       ??_C@_1M@ILHOPKA@?$AAE?$AAr?$AAr?$AAo?$AAr?$AA?$AA@ 1000dacc     service.obj
 0001:0000cad8       ??_C@_15JCKODCLA@?$AA?6?$AA?7?$AA?$AA@ 1000dad8     service.obj
 0001:0000cae0       ??_C@_19FFLPMPBO@?$AA?6?$AA?5?$AA?5?$AA?5?$AA?$AA@ 1000dae0     service.obj
 0001:0000caec       ??_C@_15IEGBJKPD@?$AA?3?$AA?6?$AA?$AA@ 1000daec     service.obj
 0001:0000caf4       ??_C@_1DG@LMKDDADI@?$AA?$DM?$AAn?$AAo?$AAn?$AA?9?$AAs?$AAt?$AAr?$AAi?$AAn?$AAg?$AA?5?$AAe?$AAr?$AAr?$AAo?$AAr?$AA?5?$AAm?$AAe?$AAs?$AAs?$AAa?$AAg?$AAe?$AA?$DO?$AA?$AA@ 1000daf4     service.obj
 0001:0000cb2c       ??_C@_17PAGBAIDI@?$AA?$DL?$AAO?$AAK?$AA?$AA@ 1000db2c     service.obj
 0001:0000cb34       ??_C@_1BA@HHOMBECE@?$AAM?$AAe?$AAs?$AAs?$AAa?$AAg?$AAe?$AA?$AA@ 1000db34     service.obj
 0001:0000cb44       ??_C@_0BJ@JOELOGM@cannot?5convert?5to?5string?$AA@ 1000db44     service.obj
 0001:0000cb60       ??_C@_08FNIIFOJC@tostring?$AA@ 1000db60     service.obj
 0001:0000cb6c       ??_C@_08CENECNJD@SortMode?$AA@ 1000db6c     service.obj
 0001:0000cb78       ??_C@_08IMMBLBLF@ViewMode?$AA@ 1000db78     service.obj
 0001:0000cb84       ??_C@_0N@CDHIFJIH@TopPanelItem?$AA@ 1000db84     service.obj
 0001:0000cb94       ??_C@_0M@JMILNLLF@CurrentItem?$AA@ 1000db94     service.obj
 0001:0000cba0       ??_C@_0BE@EOBAHHNK@SelectedItemsNumber?$AA@ 1000dba0     service.obj
 0001:0000cbb4       ??_C@_0M@DDGFKGKJ@ItemsNumber?$AA@ 1000dbb4     service.obj
 0001:0000cbc0       ??_C@_09MCEJMINN@PanelRect?$AA@ 1000dbc0     service.obj
 0001:0000cbcc       ??_C@_06PMMPCIPB@bottom?$AA@ 1000dbcc     service.obj
 0001:0000cbd4       ??_C@_05DHJDAOHK@right?$AA@ 1000dbd4     service.obj
 0001:0000cbdc       ??_C@_03FGFCOCMD@top?$AA@  1000dbdc     service.obj
 0001:0000cbe0       ??_C@_04GOOOJOPP@left?$AA@ 1000dbe0     service.obj
 0001:0000cbe8       ??_C@_09BKHPOLGD@PanelType?$AA@ 1000dbe8     service.obj
 0001:0000cbf4       ??_C@_0N@CCPLCIHE@PluginHandle?$AA@ 1000dbf4     service.obj
 0001:0000cc04       ??_C@_09ENKGJCEC@OwnerGuid?$AA@ 1000dc04     service.obj
 0001:0000cc10       ??_C@_08HGEAFCFN@PluginId?$AA@ 1000dc10     service.obj
 0001:0000cc1c       ??_C@_04PBAHLACE@File?$AA@ 1000dc1c     service.obj
 0001:0000cc24       ??_C@_05LOJBNELM@Param?$AA@ 1000dc24     service.obj
 0001:0000cc2c       ??_C@_04FABLJDN@Name?$AA@  1000dc2c     service.obj
 0001:0000cc34       ??_C@_0BA@MLHECKCE@table?5or?5string?$AA@ 1000dc34     service.obj
 0001:0000cc44       ??_C@_0BA@GNKNKKDM@number?5or?5table?$AA@ 1000dc44     service.obj
 0001:0000cc54       ??_C@_0BD@CKJHMJBG@non?9positive?5index?$AA@ 1000dc54     service.obj
 0001:0000cc68       ??_C@_0CI@DDAJHJKO@?$CFs?5?9?5unsupported?5type?5in?5dialog?5@ 1000dc68     service.obj
 0001:0000cc90       ??_C@_0CD@JIANOKII@unsupported?5flag?5in?5dialog?5item?5@ 1000dc90     service.obj
 0001:0000ccb4       ??_C@_0CB@EOGFCCCC@value?5at?5index?5?$CFd?5is?5not?5a?5table@ 1000dcb4     service.obj
 0001:0000ccd8       ??_C@_0O@FEBHKEHB@closed?5dialog?$AA@ 1000dcd8     service.obj
 0001:0000cce8       ??_C@_0BK@NEMPGLFN@operation?5not?5implemented?$AA@ 1000dce8     service.obj
 0001:0000cd04       ??_C@_05FNNGFGLF@Index?$AA@ 1000dd04     service.obj
 0001:0000cd0c       ??_C@_09OGCBKCAK@MaxLength?$AA@ 1000dd0c     service.obj
 0001:0000cd18       ??_C@_06DJONBJOP@TopPos?$AA@ 1000dd18     service.obj
 0001:0000cd20       ??_C@_09IMOCKOO@SelectPos?$AA@ 1000dd20     service.obj
 0001:0000cd2c       ??_C@_07NOCIGAPP@Pattern?$AA@ 1000dd2c     service.obj
 0001:0000cd34       ??_C@_05IJGIMMHE@Count?$AA@ 1000dd34     service.obj
 0001:0000cd3c       ??_C@_0L@CECHCPAP@StartIndex?$AA@ 1000dd3c     service.obj
 0001:0000cd48       ??_C@_0CK@JHNDGJBB@element?5?$CD?$CFd?5in?5argument?5?$CD4?5is?5no@ 1000dd48     service.obj
 0001:0000cd74       ??_C@_05DADPALEM@Right?$AA@ 1000dd74     service.obj
 0001:0000cd7c       ??_C@_03PGGAENPN@Top?$AA@  1000dd7c     service.obj
 0001:0000cd80       ??_C@_04KPCPLBPL@Left?$AA@ 1000dd80     service.obj
 0001:0000cd88       ??_C@_05LPIJGKJ@Value?$AA@ 1000dd88     service.obj
 0001:0000cd90       ??_C@_07MMLMCDAI@ValType?$AA@ 1000dd90     service.obj
 0001:0000cd98       ??_C@_07GHGHLGFI@GetType?$AA@ 1000dd98     service.obj
 0001:0000cda0       ??_C@_0P@NABDHFON@getvaluestring?$AA@ 1000dda0     service.obj
 0001:0000cdb0       ??_C@_0L@LPFMIAHH@helpstring?$AA@ 1000ddb0     service.obj
 0001:0000cdbc       ??_C@_0BJ@IINAPFDG@Items?$FL?$CFd?$FN?5is?5not?5a?5table?$AA@ 1000ddbc     service.obj
 0001:0000cdd8       ??_C@_0CC@GBOJFNBI@error?5occured?5in?5dialog?5procedur@ 1000ddd8     service.obj
 0001:0000cdfc       ??_C@_0M@EHMONPJO@?$CFs?5?$CIclosed?$CJ?$AA@ 1000ddfc     service.obj
 0001:0000ce08       ??_C@_07FBAHDBGN@CurMode?$AA@ 1000de08     service.obj
 0001:0000ce10       ??_C@_07MJHBHMFM@FilePos?$AA@ 1000de10     service.obj
 0001:0000ce18       ??_C@_08GDAJJKGC@ViewerID?$AA@ 1000de18     service.obj
 0001:0000ce24       ??_C@_06IMBBKDFH@iParam?$AA@ 1000de24     service.obj
 0001:0000ce2c       ??_C@_1CA@PCDNIBFH@?$AAE?$AAn?$AAt?$AAe?$AAr?$AA?5?$AAt?$AAh?$AAe?$AA?5?$AAt?$AAe?$AAx?$AAt?$AA?3?$AA?$AA@ 1000de2c     service.obj
 0001:0000ce4c       ??_C@_1BE@CGKCNEEP@?$AAI?$AAn?$AAp?$AAu?$AAt?$AA?5?$AAB?$AAo?$AAx?$AA?$AA@ 1000de4c     service.obj
 0001:0000ce60       ??_C@_0BG@GAFLOAPP@command?5not?5supported?$AA@ 1000de60     service.obj
 0001:0000ce78       ??_C@_08NNKIOIN@TypeName?$AA@ 1000de78     service.obj
 0001:0000ce84       ??_C@_03FCCPIJGJ@Pos?$AA@  1000de84     service.obj
 0001:0000ce88       ??_C@_0P@DJOANNIK@?$CFd?4?$CFd?4?$CFd?4?$CFd?4?$CFd?$AA@ 1000de88     service.obj
 0001:0000ce98       ??_C@_05KGEAEGFG@Total?$AA@ 1000de98     service.obj
 0001:0000cea0       __real@4059000000000000    1000dea0     service.obj
 0001:0000cea8       ??_C@_09MIJAKHKB@Completed?$AA@ 1000dea8     service.obj
 0001:0000ceb4       ??_C@_06HBEFEBCM@ErrSrc?$AA@ 1000deb4     service.obj
 0001:0000cebc       ??_C@_07KACFJJFN@ErrPosY?$AA@ 1000debc     service.obj
 0001:0000cec4       ??_C@_07LJDOKIBM@ErrPosX?$AA@ 1000dec4     service.obj
 0001:0000cecc       ??_C@_07ONPPLIAF@ErrCode?$AA@ 1000decc     service.obj
 0001:0000ced4       ??_C@_03CAOIPBNL@arg?$AA@  1000ded4     service.obj
 0001:0000ced8       ??_C@_04CIMGMMMG@text?$AA@ 1000ded8     service.obj
 0001:0000cee0       ??_C@_06GBEMGMMA@?$CF?$CKd?$CFs?5?$AA@ 1000dee0     service.obj
 0001:0000cee8       ??_C@_0CH@OINAPBOJ@tostring?$CI?$CJ?5returned?5a?5non?9string@ 1000dee8     service.obj
 0001:0000cf10       ??_C@_0CC@JIGPFMKG@global?5?$GAtostring?8?5is?5not?5functio@ 1000df10     service.obj
 0001:0000cf34       ??_C@_06LDIMCHFC@?$CF?$CKs?$CFs?5?$AA@ 1000df34     service.obj
 0001:0000cf40       ??_C@_0ME@JDKAEDFJ@local?5items?0n?$DN?4?4?4?6local?5bottom?$DNn@ 1000df40     service.obj
 0001:0000d004       ??_C@_0CG@FGNNCNLL@attempt?5to?5access?5invalid?5file?5f@ 1000e004     service.obj
 0001:0000d02c       ??_C@_07BJOIOONN@Strings?$AA@ 1000e02c     service.obj
 0001:0000d034       ??_C@_05HMEFBOHK@GInfo?$AA@ 1000e034     service.obj
 0001:0000d03c       ??_C@_05GCJGCMFJ@PInfo?$AA@ 1000e03c     service.obj
 0001:0000d044       ??_C@_0N@IEACHFBM@PluginConfig?$AA@ 1000e044     service.obj
 0001:0000d054       ??_C@_0L@NHENMPLN@PluginMenu?$AA@ 1000e054     service.obj
 0001:0000d060       ??_C@_08FGAFMHLF@DiskMenu?$AA@ 1000e060     service.obj
 0001:0000d06c       ??_C@_0N@GAMEMCEE@invalid?5GUID?$AA@ 1000e06c     service.obj
 0001:0000d07c       ??_C@_0BP@NJEEOHDB@attempt?5to?5access?5closed?5timer?$AA@ 1000e07c     service.obj
 0001:0000d09c       ??_C@_0CE@LHJCBGGH@attempt?5to?5call?5non?9existent?5met@ 1000e09c     service.obj
 0001:0000d0c0       ??_C@_06EFCDMIMC@Closed?$AA@ 1000e0c0     service.obj
 0001:0000d0c8       ??_C@_07CIINKFND@OnTimer?$AA@ 1000e0c8     service.obj
 0001:0000d0d0       ??_C@_08KDKDEPAG@Interval?$AA@ 1000e0d0     service.obj
 0001:0000d0dc       ??_C@_07DOAOMMKG@Enabled?$AA@ 1000e0dc     service.obj
 0001:0000d0e4       ??_C@_05LGELBCGM@Close?$AA@ 1000e0e4     service.obj
 0001:0000d0ec       ??_C@_0BO@PNFLEJKN@attempt?5to?5access?5a?5closed?5?$CFs?$AA@ 1000e0ec     service.obj
 0001:0000d10c       ??_C@_04LADJNOK@Lock?$AA@  1000e10c     service.obj
 0001:0000d114       ??_C@_04OKOFBOPB@Time?$AA@ 1000e114     service.obj
 0001:0000d11c       ??_C@_1CC@OPOAGCKN@?$AA?2?$AAl?$AAu?$AAa?$AAf?$AAa?$AAr?$AA_?$AAi?$AAn?$AAi?$AAt?$AA?4?$AAl?$AAu?$AAa?$AA?$AA@ 1000e11c     service.obj
 0001:0000d140       ??_C@_1BG@BDOBMIBP@?$AAF?$AAA?$AAR?$AAP?$AAR?$AAO?$AAF?$AAI?$AAL?$AAE?$AA?$AA@ 1000e140     service.obj
 0001:0000d158       ??_C@_08BNNFLGCJ@loadfile?$AA@ 1000e158     service.obj
 0001:0000d164       ??_C@_06ONNDGCDK@dofile?$AA@ 1000e164     service.obj
 0001:0000d16c       ??_C@_04LHHHFLPP@utf8?$AA@ 1000e16c     service.obj
 0001:0000d174       ??_C@_03OFAPEBGM@?$CFs?6?$AA@ 1000e174     service.obj
 0001:0000d178       ??_C@_06BPGFKLEK@__mode?$AA@ 1000e178     service.obj
 0001:0000d180       ??_C@_01DICPFPGM@k?$AA@    1000e180     service.obj
 0001:0000d184       ??_C@_06DGPPOJKF@viewer?$AA@ 1000e184     service.obj
 0001:0000d18c       ??_C@_06GIFLLBB@editor?$AA@ 1000e18c     service.obj
 0001:0000d194       ??_C@_0BC@JJHHFNMP@FarMacroCallToLua?$AA@ 1000e194     service.obj
 0001:0000d1a8       ??_C@_0N@ECMJOJJG@MacroCallFar?$AA@ 1000e1a8     service.obj
 0001:0000d1b8       ??_C@_09GCBMKPBD@utf8valid?$AA@ 1000e1b8     slnunico.obj
 0001:0000d1c4       ??_C@_05NECKJAMC@upper?$AA@ 1000e1c4     slnunico.obj
 0001:0000d1cc       ??_C@_07KOIEOCCE@reverse?$AA@ 1000e1cc     slnunico.obj
 0001:0000d1d4       ??_C@_03HOKODIMJ@rep?$AA@  1000e1d4     slnunico.obj
 0001:0000d1d8       ??_C@_05IPJEPLHL@lower?$AA@ 1000e1d8     slnunico.obj
 0001:0000d1e0       ??_C@_03BKCJCHLK@len?$AA@  1000e1e0     slnunico.obj
 0001:0000d1e4       ??_C@_05EIEIBDFD@gfind?$AA@ 1000e1e4     slnunico.obj
 0001:0000d1ec       ??_C@_06DLEPGFEF@format?$AA@ 1000e1ec     slnunico.obj
 0001:0000d1f4       ??_C@_04GGLOKIEE@dump?$AA@ 1000e1f4     slnunico.obj
 0001:0000d1fc       ??_C@_04ENMBGAPA@char?$AA@ 1000e1fc     slnunico.obj
 0001:0000d204       ??_C@_04IHGKJMLH@byte?$AA@ 1000e204     slnunico.obj
 0001:0000d298       ??_C@_04GMGOKAFF@mode?$AA@ 1000e298     slnunico.obj
 0001:0000d2a0       ??_C@_0BG@DFAIEAEC@string?5slice?5too?5long?$AA@ 1000e2a0     slnunico.obj
 0001:0000d2b8       ??_C@_0O@EAJJMEEM@invalid?5value?$AA@ 1000e2b8     slnunico.obj
 0001:0000d2c8       ??_C@_0BO@BNLBHKJN@unable?5to?5dump?5given?5function?$AA@ 1000e2c8     slnunico.obj
 0001:0000d2e8       ??_C@_0BG@LEHNKOGD@invalid?5capture?5index?$AA@ 1000e2e8     slnunico.obj
 0001:0000d300       ??_C@_0BI@ECNPHIBF@invalid?5pattern?5capture?$AA@ 1000e300     slnunico.obj
 0001:0000d318       ??_C@_0CD@PLJBIEHA@malformed?5pattern?5?$CIends?5with?5?8?$CF?$CF@ 1000e318     slnunico.obj
 0001:0000d33c       ??_C@_0CA@CFGACOGB@malformed?5pattern?5?$CImissing?5?8?$FN?8?$CJ?$AA@ 1000e33c     slnunico.obj
 0001:0000d35c       ??_C@_0BD@NGJIMPLI@unbalanced?5pattern?$AA@ 1000e35c     slnunico.obj
 0001:0000d370       ??_C@_0BC@IMEAEJPD@too?5many?5captures?$AA@ 1000e370     slnunico.obj
 0001:0000d384       ??_C@_0BD@BFKNEALP@unfinished?5capture?$AA@ 1000e384     slnunico.obj
 0001:0000d398       ??_C@_0L@NLFJOONJ@?$FO$?$CK?$CL?$DP?4?$CI?$FL?$CF?9?$AA@ 1000e398     slnunico.obj
 0001:0000d3a4       ??_C@_0CO@MAGJPEI@?8string?4gfind?8?5was?5renamed?5to?5?8s@ 1000e3a4     slnunico.obj
 0001:0000d3d4       ??_C@_0BP@PPPOBACA@string?1function?1table?5expected?$AA@ 1000e3d4     slnunico.obj
 0001:0000d3f4       ??_C@_0CB@LPDIHGGA@invalid?5replacement?5value?5?$CIa?5?$CFs?$CJ@ 1000e3f4     slnunico.obj
 0001:0000d418       ??_C@_04MPDIABOK@?2000?$AA@ 1000e418     slnunico.obj
 0001:0000d420       ??_C@_02HIBBOKEN@?2r?$AA@  1000e420     slnunico.obj
 0001:0000d424       ??_C@_0CN@KALFEKPN@invalid?5format?5?$CIwidth?5or?5precisi@ 1000e424     slnunico.obj
 0001:0000d454       ??_C@_0CA@COOMGCAO@invalid?5format?5?$CIrepeated?5flags?$CJ?$AA@ 1000e454     slnunico.obj
 0001:0000d474       ??_C@_05GGBDHNF@?9?$CL?5?$CD0?$AA@ 1000e474     slnunico.obj
 0001:0000d47c       ??_C@_0CC@KIPBEOBI@invalid?5option?5?8?$CF?$CF?$CFc?8?5to?5?8format@ 1000e47c     slnunico.obj
 0001:0000d4a0       ??_C@_0N@DKIDGKBP@unicode?4utf8?$AA@ 1000e4a0     slnunico.obj
 0001:0000d4b0       ??_C@_0BB@EFCDCNG@unicode?4grapheme?$AA@ 1000e4b0     slnunico.obj
 0001:0000d4c4       ??_C@_0P@CMOFLLND@unicode?4latin1?$AA@ 1000e4c4     slnunico.obj
 0001:0000d4d4       ??_C@_0O@EJMKHGFJ@unicode?4ascii?$AA@ 1000e4d4     slnunico.obj
 0001:0000d4e4       ??_C@_07HHBPNGAN@setvbuf?$AA@ 1000e4e4     uliolib51.obj
 0001:0000d4ec       ??_C@_04EDECCOGL@seek?$AA@ 1000e4ec     uliolib51.obj
 0001:0000d4f4       ??_C@_05NGFEDHGN@write?$AA@ 1000e4f4     uliolib51.obj
 0001:0000d4fc       ??_C@_07FKJPAINK@tmpfile?$AA@ 1000e4fc     uliolib51.obj
 0001:0000d504       ??_C@_05IACAFMHP@popen?$AA@ 1000e504     uliolib51.obj
 0001:0000d50c       ??_C@_05DENOCHIP@lines?$AA@ 1000e50c     uliolib51.obj
 0001:0000d514       ??_C@_05GLCAEPFP@flush?$AA@ 1000e514     uliolib51.obj
 0001:0000d51c       ??_C@_05LBOHBHFK@close?$AA@ 1000e51c     uliolib51.obj
 0001:0000d524       ??_C@_04HJPCFDOP@line?$AA@ 1000e524     uliolib51.obj
 0001:0000d52c       ??_C@_04PLMLMMEO@full?$AA@ 1000e52c     uliolib51.obj
 0001:0000d534       ??_C@_02KAJCLHKP@no?$AA@   1000e534     uliolib51.obj
 0001:0000d538       ??_C@_03JBJLGPFL@end?$AA@  1000e538     uliolib51.obj
 0001:0000d53c       ??_C@_03LIBLMJMB@cur?$AA@  1000e53c     uliolib51.obj
 0001:0000d540       ??_C@_03KCHOJKKI@set?$AA@  1000e540     uliolib51.obj
 0001:0000d544       ??_C@_06DKIGHACF@output?$AA@ 1000e544     uliolib51.obj
 0001:0000d54c       ??_C@_05DFJCHPDH@input?$AA@ 1000e54c     uliolib51.obj
 0001:0000d648       ??_C@_02DKCKIIND@?$CFs?$AA@ 1000e648     uliolib51.obj
 0001:0000d64c       ??_C@_06DJHOIPC@?$CFs?3?5?$CFs?$AA@ 1000e64c     uliolib51.obj
 0001:0000d654       ??_C@_04DAMGJPCA@file?$AA@ 1000e654     uliolib51.obj
 0001:0000d65c       ??_C@_0M@IBKPHHKH@closed?5file?$AA@ 1000e65c     uliolib51.obj
 0001:0000d668       ??_C@_05KCHOJJD@FILE?$CK?$AA@ 1000e668     uliolib51.obj
 0001:0000d670       ??_C@_0BN@LPOOHAOM@attempt?5to?5use?5a?5closed?5file?$AA@ 1000e670     uliolib51.obj
 0001:0000d690       ??_C@_0BL@PEFGCPAG@cannot?5close?5standard?5file?$AA@ 1000e690     uliolib51.obj
 0001:0000d6ac       ??_C@_07DMJMBBKE@__close?$AA@ 1000e6ac     uliolib51.obj
 0001:0000d6b4       ??_C@_09BPMAMLLD@file?5?$CI?$CFp?$CJ?$AA@ 1000e6b4     uliolib51.obj
 0001:0000d6c0       ??_C@_0O@PLFAPHPG@file?5?$CIclosed?$CJ?$AA@ 1000e6c0     uliolib51.obj
 0001:0000d6d0       ??_C@_0CP@DHGANCPP@invalid?5mode?5?8?$CFs?8?5?$CIshould?5match?5@ 1000e6d0     uliolib51.obj
 0001:0000d700       ??_C@_17OBBFBLGE@?$AAr?$AAw?$AAa?$AA?$AA@ 1000e700     uliolib51.obj
 0001:0000d708       ??_C@_0BL@JMNLNGCA@standard?5?$CFs?5file?5is?5closed?$AA@ 1000e708     uliolib51.obj
 0001:0000d724       ??_C@_13CIFDLIMG@?$AAw?$AA?$AA@ 1000e724     uliolib51.obj
 0001:0000d728       ??_C@_03DLDNIBIK@?$CFlf?$AA@ 1000e728     uliolib51.obj
 0001:0000d72c       ??_C@_0P@CENJCLHM@invalid?5format?$AA@ 1000e72c     uliolib51.obj
 0001:0000d73c       ??_C@_0P@PJFAGLMH@invalid?5option?$AA@ 1000e73c     uliolib51.obj
 0001:0000d74c       ??_C@_0BD@IOJAAODF@too?5many?5arguments?$AA@ 1000e74c     uliolib51.obj
 0001:0000d760       ??_C@_0BH@PBGIDLEF@file?5is?5already?5closed?$AA@ 1000e760     uliolib51.obj
 0001:0000d778       ??_C@_05CGOEHEFE@?$CF?414g?$AA@ 1000e778     uliolib51.obj
 0001:0000d780       ??_C@_06FJGNEBG@stderr?$AA@ 1000e780     uliolib51.obj
 0001:0000d788       ??_C@_06DJDOIFHB@stdout?$AA@ 1000e788     uliolib51.obj
 0001:0000d790       ??_C@_05MHOFLBOO@stdin?$AA@ 1000e790     uliolib51.obj
 0001:0000d798       ??_C@_07FFLLPPLH@require?$AA@ 1000e798     uloadlib51.obj
 0001:0000d7a0       ??_C@_06BIEEJMKO@module?$AA@ 1000e7a0     uloadlib51.obj
 0001:0000d7a8       ??_C@_06LNOHAKGK@seeall?$AA@ 1000e7a8     uloadlib51.obj
 0001:0000d7b0       ??_C@_07KOEABFCN@loadlib?$AA@ 1000e7b0     uloadlib51.obj
 0001:0000d800       ??_C@_0BN@GMPFCLAN@unable?5to?5get?5ModuleFileName?$AA@ 1000e800     uloadlib51.obj
 0001:0000d820       ??_C@_13MGDFOILI@?$AA?$CB?$AA?$AA@ 1000e820     uloadlib51.obj
 0001:0000d824       ??_C@_08HNNNOMMJ@_LOADLIB?$AA@ 1000e824     uloadlib51.obj
 0001:0000d830       ??_C@_04HDOCAJNK@?$CFs?$CFs?$AA@ 1000e830     uloadlib51.obj
 0001:0000d838       ??_C@_09GMLHALBF@LOADLIB?3?5?$AA@ 1000e838     uloadlib51.obj
 0001:0000d844       ??_C@_04HKFDNBLD@init?$AA@ 1000e844     uloadlib51.obj
 0001:0000d84c       ??_C@_0P@NEBKIMDC@?6?7no?5file?5?8?$CFs?8?$AA@ 1000e84c     uloadlib51.obj
 0001:0000d85c       ??_C@_13HGPDMIBE@?$AA?$DP?$AA?$AA@ 1000e85c     uloadlib51.obj
 0001:0000d860       ??_C@_0CE@EPEHLLIH@?8package?4?$CFs?8?5contains?5invalid?5UT@ 1000e860     uloadlib51.obj
 0001:0000d884       ??_C@_0BO@COFCKCAL@?8package?4?$CFs?8?5must?5be?5a?5string?$AA@ 1000e884     uloadlib51.obj
 0001:0000d8a4       ??_C@_13JOFGPIOO@?$AA?4?$AA?$AA@ 1000e8a4     uloadlib51.obj
 0001:0000d8a8       ??_C@_13FPGAJAPJ@?$AA?2?$AA?$AA@ 1000e8a8     uloadlib51.obj
 0001:0000d8ac       ??_C@_0CO@KHMIPLKM@error?5loading?5module?5?8?$CFs?8?5from?5f@ 1000e8ac     uloadlib51.obj
 0001:0000d8dc       ??_C@_04LNEJFJGI@path?$AA@ 1000e8dc     uloadlib51.obj
 0001:0000d8e4       ??_C@_0L@KHKMBFOE@luaopen_?$CFs?$AA@ 1000e8e4     uloadlib51.obj
 0001:0000d8f0       ??_C@_01LFCBOECM@?4?$AA@   1000e8f0     uloadlib51.obj
 0001:0000d8f4       ??_C@_01IDAFKMJL@_?$AA@    1000e8f4     uloadlib51.obj
 0001:0000d8f8       ??_C@_05EEMJHCCC@cpath?$AA@ 1000e8f8     uloadlib51.obj
 0001:0000d900       ??_C@_0BO@KOILFIGK@?6?7no?5module?5?8?$CFs?8?5in?5file?5?8?$CFs?8?$AA@ 1000e900     uloadlib51.obj
 0001:0000d920       ??_C@_0CB@NPNABMBF@?6?7no?5field?5package?4preload?$FL?8?$CFs?8?$FN@ 1000e920     uloadlib51.obj
 0001:0000d944       ??_C@_0CC@CCJHFBLH@?8package?4preload?8?5must?5be?5a?5tabl@ 1000e944     uloadlib51.obj
 0001:0000d968       ??_C@_0BJ@HFHHABH@module?5?8?$CFs?8?5not?5found?3?$CFs?$AA@ 1000e968     uloadlib51.obj
 0001:0000d984       ??_C@_0CC@IGEJMOFI@?8package?4loaders?8?5must?5be?5a?5tabl@ 1000e984     uloadlib51.obj
 0001:0000d9a8       ??_C@_07JAOCDFCG@loaders?$AA@ 1000e9a8     uloadlib51.obj
 0001:0000d9b0       ??_C@_0CL@DIEJCPFH@loop?5or?5previous?5error?5loading?5m@ 1000e9b0     uloadlib51.obj
 0001:0000d9dc       ??_C@_07PINPBNPB@_LOADED?$AA@ 1000e9dc     uloadlib51.obj
 0001:0000d9e4       ??_C@_0CI@GKOMOAFD@?8module?8?5not?5called?5from?5a?5Lua?5f@ 1000e9e4     uloadlib51.obj
 0001:0000da0c       ??_C@_01INIBCBCB@f?$AA@    1000ea0c     uloadlib51.obj
 0001:0000da10       ??_C@_08HONLOGDK@_PACKAGE?$AA@ 1000ea10     uloadlib51.obj
 0001:0000da1c       ??_C@_05ICMCJINN@_NAME?$AA@ 1000ea1c     uloadlib51.obj
 0001:0000da24       ??_C@_02CCIJHOCI@_M?$AA@   1000ea24     uloadlib51.obj
 0001:0000da28       ??_C@_0BO@CBJIAGLF@name?5conflict?5for?5module?5?8?$CFs?8?$AA@ 1000ea28     uloadlib51.obj
 0001:0000da48       ??_C@_13GGAHEHIG@?$AA?$AB?$AA?$AA@ 1000ea48     uloadlib51.obj
 0001:0000da4c       ??_C@_15HKKNGJC@?$AA?$DL?$AA?$DL?$AA?$AA@ 1000ea4c     uloadlib51.obj
 0001:0000da54       ??_C@_17KOAMMDLI@?$AA?$DL?$AA?$AB?$AA?$DL?$AA?$AA@ 1000ea54     uloadlib51.obj
 0001:0000da5c       ??_C@_06IILMCCFO@loaded?$AA@ 1000ea5c     uloadlib51.obj
 0001:0000da64       ??_C@_06HEJKKHEK@config?$AA@ 1000ea64     uloadlib51.obj
 0001:0000da6c       ??_C@_1BE@CKNDCMBB@?$AA?2?$AA?6?$AA?$DL?$AA?6?$AA?$DP?$AA?6?$AA?$CB?$AA?6?$AA?9?$AA?$AA@ 1000ea6c     uloadlib51.obj
 0001:0000da80       ??_C@_1BE@EFNILHBI@?$AAL?$AAU?$AAA?$AA_?$AAC?$AAP?$AAA?$AAT?$AAH?$AA?$AA@ 1000ea80     uloadlib51.obj
 0001:0000da94       ??_C@_1DM@FGPGEDD@?$AA?4?$AA?2?$AA?$DP?$AA?4?$AAd?$AAl?$AAl?$AA?$DL?$AA?$CB?$AA?2?$AA?$DP?$AA?4?$AAd?$AAl?$AAl?$AA?$DL?$AA?$CB?$AA?2?$AAl?$AAo?$AAa?$AAd?$AAa?$AAl?$AAl?$AA?4?$AAd?$AAl?$AAl?$AA?$AA@ 1000ea94     uloadlib51.obj
 0001:0000dad0       ??_C@_1BC@ILFFIBFI@?$AAL?$AAU?$AAA?$AA_?$AAP?$AAA?$AAT?$AAH?$AA?$AA@ 1000ead0     uloadlib51.obj
 0001:0000dae8       ??_C@_1HE@JLDBNBHO@?$AA?4?$AA?2?$AA?$DP?$AA?4?$AAl?$AAu?$AAa?$AA?$DL?$AA?$CB?$AA?2?$AAl?$AAu?$AAa?$AA?2?$AA?$DP?$AA?4?$AAl?$AAu?$AAa?$AA?$DL?$AA?$CB?$AA?2?$AAl?$AAu?$AAa?$AA?2?$AA?$DP?$AA?2?$AAi?$AAn?$AAi?$AAt@ 1000eae8     uloadlib51.obj
 0001:0000db5c       ??_C@_04NOFELICG@lenW?$AA@ 1000eb5c     ustring.obj
 0001:0000db64       ??_C@_06FHFOAHML@system?$AA@ 1000eb64     ustring.obj
 0001:0000db6c       ??_C@_04GFOHBGIO@subW?$AA@ 1000eb6c     ustring.obj
 0001:0000db74       ??_C@_0BE@LJADKLBD@WideCharToMultiByte?$AA@ 1000eb74     ustring.obj
 0001:0000db88       ??_C@_04NDFIEGPL@Uuid?$AA@ 1000eb88     ustring.obj
 0001:0000db90       ??_C@_0M@GJGCILHG@Utf8ToUtf16?$AA@ 1000eb90     ustring.obj
 0001:0000db9c       ??_C@_09LCEKPEGC@Utf8ToOem?$AA@ 1000eb9c     ustring.obj
 0001:0000dba8       ??_C@_0M@KJELMDJD@Utf16ToUtf8?$AA@ 1000eba8     ustring.obj
 0001:0000dbb4       ??_C@_05PFDOMJEF@Sleep?$AA@ 1000ebb4     ustring.obj
 0001:0000dbbc       ??_C@_0M@KINCEKFL@SetFileAttr?$AA@ 1000ebbc     ustring.obj
 0001:0000dbc8       ??_C@_0O@IHAPJIOC@SetCurrentDir?$AA@ 1000ebc8     ustring.obj
 0001:0000dbd8       ??_C@_0L@PMCLJMMJ@SearchPath?$AA@ 1000ebd8     ustring.obj
 0001:0000dbe4       ??_C@_0BA@MNJFBAJH@SHGetFolderPath?$AA@ 1000ebe4     ustring.obj
 0001:0000dbf4       ??_C@_0BC@NFCPMJFM@OutputDebugString?$AA@ 1000ebf4     ustring.obj
 0001:0000dc08       ??_C@_09EPINLGBH@OemToUtf8?$AA@ 1000ec08     ustring.obj
 0001:0000dc14       ??_C@_0BE@HCIKGJGE@MultiByteToWideChar?$AA@ 1000ec14     ustring.obj
 0001:0000dc28       ??_C@_0BD@IHIHPGDL@GlobalMemoryStatus?$AA@ 1000ec28     ustring.obj
 0001:0000dc3c       ??_C@_08OMCNFONF@GetOEMCP?$AA@ 1000ec3c     ustring.obj
 0001:0000dc48       ??_C@_0BH@KKAFOIJJ@GetLogicalDriveStrings?$AA@ 1000ec48     ustring.obj
 0001:0000dc60       ??_C@_0M@KHMMJMNI@GetFileAttr?$AA@ 1000ec60     ustring.obj
 0001:0000dc6c       ??_C@_0N@IIBOJKJ@GetDriveType?$AA@ 1000ec6c     ustring.obj
 0001:0000dc7c       ??_C@_0O@PIBBCLJF@GetCurrentDir?$AA@ 1000ec7c     ustring.obj
 0001:0000dc8c       ??_C@_09HLFMNDA@GetCPInfo?$AA@ 1000ec8c     ustring.obj
 0001:0000dc98       ??_C@_06FMJLOCAF@GetACP?$AA@ 1000ec98     ustring.obj
 0001:0000dca0       ??_C@_0BE@DEHGONAH@EnumSystemCodePages?$AA@ 1000eca0     ustring.obj
 0001:0000dcb8       _ustring_funcs             1000ecb8     ustring.obj
 0001:0000dd88       ??_C@_0BJ@MEAJDMDL@invalid?5multibyte?5string?$AA@ 1000ed88     ustring.obj
 0001:0000dda4       ??_C@_0BG@ELIKBHAO@invalid?5UTF?916?5string?$AA@ 1000eda4     ustring.obj
 0001:0000ddbc       ??_C@_0N@IFJMFGJK@unknown?5type?$AA@ 1000edbc     ustring.obj
 0001:0000ddcc       ??_C@_07BHCBOAMP@ramdisk?$AA@ 1000edcc     ustring.obj
 0001:0000ddd4       ??_C@_05POABADMF@cdrom?$AA@ 1000edd4     ustring.obj
 0001:0000dddc       ??_C@_06IMIHEKN@remote?$AA@ 1000eddc     ustring.obj
 0001:0000dde4       ??_C@_05OFLEIIDM@fixed?$AA@ 1000ede4     ustring.obj
 0001:0000ddec       ??_C@_09HPGMKNKO@removable?$AA@ 1000edec     ustring.obj
 0001:0000ddf8       ??_C@_0BC@GPFCFLGN@no?5root?5directory?$AA@ 1000edf8     ustring.obj
 0001:0000de0c       ??_C@_0P@KJDDGAFH@FileAttributes?$AA@ 1000ee0c     ustring.obj
 0001:0000de1c       ??_C@_07JOJHCKGP@ustring?$AA@ 1000ee1c     ustring.obj
 0001:0000de24       ??_C@_0BB@BLJKPILH@system?5error?5?$CFd?6?$AA@ 1000ee24     ustring.obj
 0001:0000de38       ??_C@_0N@DJCOCBOB@CodePageName?$AA@ 1000ee38     ustring.obj
 0001:0000de48       ??_C@_0BD@CBNPFFPH@UnicodeDefaultChar?$AA@ 1000ee48     ustring.obj
 0001:0000de5c       ??_C@_08HIIJAENB@LeadByte?$AA@ 1000ee5c     ustring.obj
 0001:0000de68       ??_C@_0M@IMOFNPBB@DefaultChar?$AA@ 1000ee68     ustring.obj
 0001:0000de74       ??_C@_0M@KJGJBDLL@MaxCharSize?$AA@ 1000ee74     ustring.obj
 0001:0000de80       ??_C@_0BF@KKNLCGDE@AvailExtendedVirtual?$AA@ 1000ee80     ustring.obj
 0001:0000de98       ??_C@_0N@EGHLANBF@AvailVirtual?$AA@ 1000ee98     ustring.obj
 0001:0000dea8       ??_C@_0N@LCJEOHMM@TotalVirtual?$AA@ 1000eea8     ustring.obj
 0001:0000deb8       ??_C@_0O@LLHOKNF@AvailPageFile?$AA@ 1000eeb8     ustring.obj
 0001:0000dec8       ??_C@_0O@PEEMGPEP@TotalPageFile?$AA@ 1000eec8     ustring.obj
 0001:0000ded8       ??_C@_09KFOEOLH@AvailPhys?$AA@ 1000eed8     ustring.obj
 0001:0000dee4       ??_C@_09MMAOIBBJ@TotalPhys?$AA@ 1000eee4     ustring.obj
 0001:0000def0       ??_C@_0L@PLJFMBIJ@MemoryLoad?$AA@ 1000eef0     ustring.obj
 0001:0000e720       ??_C@_0DJ@KKHMCMAP@bad?5field?5?$FL?$CFd?$FN?5in?5table?5stackpos@ 1000f720     util.obj
 0001:0000e75c       ??_C@_0DJ@PFHHGAMM@bad?5field?5?8?$CFs?8?5in?5table?5stackpos@ 1000f75c     util.obj
 0001:0000e798       ??_C@_06EBGNBFIA@number?$AA@ 1000f798     util.obj
 0001:0000e7a0       ??_C@_06DNONFAKH@wcscmp?$AA@ 1000f7a0     win.obj
 0001:0000e7a8       ??_C@_0BF@HBHGIPOG@SystemTimeToFileTime?$AA@ 1000f7a8     win.obj
 0001:0000e7c0       ??_C@_0N@BFFIJKHB@ShellExecute?$AA@ 1000f7c0     win.obj
 0001:0000e7d0       ??_C@_09ELCNCICB@SetRegKey?$AA@ 1000f7d0     win.obj
 0001:0000e7dc       ??_C@_06LDCDJLBI@SetEnv?$AA@ 1000f7dc     win.obj
 0001:0000e7e4       ??_C@_0L@HBAGBENL@RenameFile?$AA@ 1000f7e4     win.obj
 0001:0000e7f0       ??_C@_09EDKALOCB@RemoveDir?$AA@ 1000f7f0     win.obj
 0001:0000e7fc       ??_C@_08CALLHOCI@MoveFile?$AA@ 1000f7fc     win.obj
 0001:0000e808       ??_C@_0P@GGGHOPAD@GetVirtualKeys?$AA@ 1000f808     win.obj
 0001:0000e818       ??_C@_0BI@ENMDHCMK@GetSystemTimeAsFileTime?$AA@ 1000f818     win.obj
 0001:0000e830       ??_C@_09GFGIAJLD@GetRegKey?$AA@ 1000f830     win.obj
 0001:0000e83c       ??_C@_0M@EINGHLOA@GetFileInfo?$AA@ 1000f83c     win.obj
 0001:0000e848       ??_C@_06CALCCDMF@GetEnv?$AA@ 1000f848     win.obj
 0001:0000e850       ??_C@_0BL@NAIJNMLL@GetConsoleScreenBufferInfo?$AA@ 1000f850     win.obj
 0001:0000e86c       ??_C@_0BF@KPJNHALE@FileTimeToSystemTime?$AA@ 1000f86c     win.obj
 0001:0000e884       ??_C@_0BI@EKFDIGHI@FileTimeToLocalFileTime?$AA@ 1000f884     win.obj
 0001:0000e89c       ??_C@_0L@MGMEFCAE@ExtractKey?$AA@ 1000f89c     win.obj
 0001:0000e8a8       ??_C@_0N@PFFNCIBD@EnumRegValue?$AA@ 1000f8a8     win.obj
 0001:0000e8b8       ??_C@_0L@DGAGCFOP@EnumRegKey?$AA@ 1000f8b8     win.obj
 0001:0000e8c4       ??_C@_0P@PCCDOIAL@DeleteRegValue?$AA@ 1000f8c4     win.obj
 0001:0000e8d4       ??_C@_0N@FOJPHHPH@DeleteRegKey?$AA@ 1000f8d4     win.obj
 0001:0000e8e4       ??_C@_0L@GPLPOFDC@DeleteFile?$AA@ 1000f8e4     win.obj
 0001:0000e8f0       ??_C@_09INHPLKKM@CreateDir?$AA@ 1000f8f0     win.obj
 0001:0000e8fc       ??_C@_08PPLNFCGA@CopyFile?$AA@ 1000f8fc     win.obj
 0001:0000e908       ??_C@_0O@CFPMOCDP@CompareString?$AA@ 1000f908     win.obj
 0001:0000f138       _win_funcs                 10010138     win.obj
 0001:0000f208       ??_C@_0DA@DKALLFDI@must?5be?5?8HKLM?8?0?5?8HKCC?8?0?5?8HKCR?8?0?5@ 10010208     win.obj
 0001:0000f238       ??_C@_03DLBIJLAB@HKU?$AA@  10010238     win.obj
 0001:0000f23c       ??_C@_04KIFLFONO@HKCU?$AA@ 1001023c     win.obj
 0001:0000f244       ??_C@_04OHBKMIBJ@HKCR?$AA@ 10010244     win.obj
 0001:0000f24c       ??_C@_04LEMDOLAJ@HKCC?$AA@ 1001024c     win.obj
 0001:0000f254       ??_C@_04CBBMIBLK@HKLM?$AA@ 10010254     win.obj
 0001:0000f25c       ??_C@_0BH@NOJOGNJM@unsupported?5value?5type?$AA@ 1001025c     win.obj
 0001:0000f274       ??_C@_0M@PEGIPCHN@multistring?$AA@ 10010274     win.obj
 0001:0000f280       ??_C@_0N@CBOMHLPN@expandstring?$AA@ 10010280     win.obj
 0001:0000f290       ??_C@_06FNFBAEBE@binary?$AA@ 10010290     win.obj
 0001:0000f298       ??_C@_05KDALNKAH@dword?$AA@ 10010298     win.obj
 0001:0000f2a0       ??_C@_0BI@COLHBIIE@RegQueryValueEx?5failed?4?$AA@ 100102a0     win.obj
 0001:0000f2b8       ??_C@_0BD@MJODDCFG@OpenRegKey?5failed?4?$AA@ 100102b8     win.obj
 0001:0000f2cc       ??_C@_0BG@HHFHBIKG@RegOpenKeyExW?5failed?4?$AA@ 100102cc     win.obj
 0001:0000f2e4       ??_C@_0O@HBAPEOKP@wMilliseconds?$AA@ 100102e4     win.obj
 0001:0000f2f4       ??_C@_07IIEDHHJN@wSecond?$AA@ 100102f4     win.obj
 0001:0000f2fc       ??_C@_07HPODENI@wMinute?$AA@ 100102fc     win.obj
 0001:0000f304       ??_C@_05BMOPCGDH@wHour?$AA@ 10010304     win.obj
 0001:0000f30c       ??_C@_04NBLBJIPP@wDay?$AA@ 1001030c     win.obj
 0001:0000f314       ??_C@_0L@OAHPHHP@wDayOfWeek?$AA@ 10010314     win.obj
 0001:0000f320       ??_C@_06MGNNJGBJ@wMonth?$AA@ 10010320     win.obj
 0001:0000f328       ??_C@_05DFPNHDMN@wYear?$AA@ 10010328     win.obj
 0001:0000f330       ??_C@_01LKDEMHDF@s?$AA@    10010330     win.obj
 0001:0000f334       ??_C@_0BD@BKPAAFMJ@MaximumWindowSizeY?$AA@ 10010334     win.obj
 0001:0000f348       ??_C@_0BD@DOLDEII@MaximumWindowSizeX?$AA@ 10010348     win.obj
 0001:0000f35c       ??_C@_0N@JPIJCAOJ@WindowBottom?$AA@ 1001035c     win.obj
 0001:0000f36c       ??_C@_0M@HHPHMPGH@WindowRight?$AA@ 1001036c     win.obj
 0001:0000f378       ??_C@_09JHGOALHG@WindowTop?$AA@ 10010378     win.obj
 0001:0000f384       ??_C@_0L@NFCEOFBF@WindowLeft?$AA@ 10010384     win.obj
 0001:0000f390       ??_C@_0BA@JJEFAHJN@CursorPositionY?$AA@ 10010390     win.obj
 0001:0000f3a0       ??_C@_0BA@IAFODGNM@CursorPositionX?$AA@ 100103a0     win.obj
 0001:0000f3b0       ??_C@_0BJ@LPJMBJJL@directory?5already?5exists?$AA@ 100103b0     win.obj
 0001:0000f3cc       ??_C@_01PFHFFBPC@t?$AA@    100103cc     win.obj
 0001:0000f3d0       __FPinit                   100103d0     LIBCMT:_fpinit_.obj
 0001:0000f3d8       ??_C@_0EA@FCLIIPNN@Visual?5C?$CL?$CL?5CRT?3?5Not?5enough?5memor@ 100103d8     LIBCMT:strerror.obj
 0001:0000f418       ??_C@_01KICIPPFI@?2?$AA@   10010418     LIBCMT:popen.obj
 0001:0000f41c       ??_C@_19IJOJOJIB@?$AAP?$AAA?$AAT?$AAH?$AA?$AA@ 1001041c     LIBCMT:wpopen.obj
 0001:0000f428       ??_C@_19FNCMDGGJ@?$AA?5?$AA?1?$AAc?$AA?5?$AA?$AA@ 10010428     LIBCMT:wpopen.obj
 0001:0000f434       ??_C@_1BA@DBKIDAPL@?$AAc?$AAm?$AAd?$AA?4?$AAe?$AAx?$AAe?$AA?$AA@ 10010434     LIBCMT:wpopen.obj
 0001:0000f444       ??_C@_1BA@HMCCKBDK@?$AAC?$AAO?$AAM?$AAS?$AAP?$AAE?$AAC?$AA?$AA@ 10010444     LIBCMT:wpopen.obj
 0001:0000f454       ??_C@_15JBFELBFC@?$AA?1?$AAc?$AA?$AA@ 10010454     LIBCMT:wsystem.obj
 0001:0000f45c       __pRawDllMain              1001045c     LIBCMT:dllcrt0.obj
 0001:0000f45c       __pDefaultRawDllMain       1001045c     LIBCMT:dllcrt0.obj
 0001:0000f460       ??_C@_05KLBDPFGC@e?$CL000?$AA@ 10010460     LIBCMT:cvt.obj
 0001:0000f468       ??_C@_1O@CEDCILHN@?$AA?$CI?$AAn?$AAu?$AAl?$AAl?$AA?$CJ?$AA?$AA@ 10010468     LIBCMT:output.obj
 0001:0000f478       ??_C@_06OJHGLDPL@?$CInull?$CJ?$AA@ 10010478     LIBCMT:output.obj
 0001:0000f480       ___lookuptable             10010480     LIBCMT:output.obj
 0001:0000f4dc       ??_C@_0P@MIGLKIOC@CorExitProcess?$AA@ 100104dc     LIBCMT:crt0dat.obj
 0001:0000f4ec       ??_C@_1BI@BGOHAHKC@?$AAm?$AAs?$AAc?$AAo?$AAr?$AAe?$AAe?$AA?4?$AAd?$AAl?$AAl?$AA?$AA@ 100104ec     LIBCMT:crt0dat.obj
 0001:0000f504       ??_C@_1BO@BKOMIGKJ@?$AAr?$AAu?$AAn?$AAt?$AAi?$AAm?$AAe?$AA?5?$AAe?$AAr?$AAr?$AAo?$AAr?$AA?5?$AA?$AA@ 10010504     LIBCMT:crt0msg.obj
 0001:0000f524       ??_C@_15JNBOKNOG@?$AA?$AN?$AA?6?$AA?$AA@ 10010524     LIBCMT:crt0msg.obj
 0001:0000f52c       ??_C@_1BM@JBBEPPHI@?$AAT?$AAL?$AAO?$AAS?$AAS?$AA?5?$AAe?$AAr?$AAr?$AAo?$AAr?$AA?$AN?$AA?6?$AA?$AA@ 1001052c     LIBCMT:crt0msg.obj
 0001:0000f548       ??_C@_1BK@KMOMNAAI@?$AAS?$AAI?$AAN?$AAG?$AA?5?$AAe?$AAr?$AAr?$AAo?$AAr?$AA?$AN?$AA?6?$AA?$AA@ 10010548     LIBCMT:crt0msg.obj
 0001:0000f564       ??_C@_1BO@BFCDCGC@?$AAD?$AAO?$AAM?$AAA?$AAI?$AAN?$AA?5?$AAe?$AAr?$AAr?$AAo?$AAr?$AA?$AN?$AA?6?$AA?$AA@ 10010564     LIBCMT:crt0msg.obj
 0001:0000f588       ??_C@_1BOO@KGEDBGAJ@?$AAR?$AA6?$AA0?$AA3?$AA3?$AA?$AN?$AA?6?$AA?9?$AA?5?$AAA?$AAt?$AAt?$AAe?$AAm?$AAp?$AAt?$AA?5?$AAt?$AAo?$AA?5?$AAu?$AAs?$AAe?$AA?5?$AAM?$AAS?$AAI?$AAL?$AA?5?$AAc?$AAo?$AAd@ 10010588     LIBCMT:crt0msg.obj
 0001:0000f778       ??_C@_1GG@GOPILAJP@?$AAR?$AA6?$AA0?$AA3?$AA2?$AA?$AN?$AA?6?$AA?9?$AA?5?$AAn?$AAo?$AAt?$AA?5?$AAe?$AAn?$AAo?$AAu?$AAg?$AAh?$AA?5?$AAs?$AAp?$AAa?$AAc?$AAe?$AA?5?$AAf?$AAo?$AAr?$AA?5?$AAl?$AAo@ 10010778     LIBCMT:crt0msg.obj
 0001:0000f7e0       ??_C@_1MG@ENCOOIDF@?$AAR?$AA6?$AA0?$AA3?$AA1?$AA?$AN?$AA?6?$AA?9?$AA?5?$AAA?$AAt?$AAt?$AAe?$AAm?$AAp?$AAt?$AA?5?$AAt?$AAo?$AA?5?$AAi?$AAn?$AAi?$AAt?$AAi?$AAa?$AAl?$AAi?$AAz?$AAe?$AA?5?$AAt@ 100107e0     LIBCMT:crt0msg.obj
 0001:0000f8a8       ??_C@_1DO@BMFCDCD@?$AAR?$AA6?$AA0?$AA3?$AA0?$AA?$AN?$AA?6?$AA?9?$AA?5?$AAC?$AAR?$AAT?$AA?5?$AAn?$AAo?$AAt?$AA?5?$AAi?$AAn?$AAi?$AAt?$AAi?$AAa?$AAl?$AAi?$AAz?$AAe?$AAd?$AA?$AN?$AA?6?$AA?$AA@ 100108a8     LIBCMT:crt0msg.obj
 0001:0000f8e8       ??_C@_1EK@HHFLMAOL@?$AAR?$AA6?$AA0?$AA2?$AA8?$AA?$AN?$AA?6?$AA?9?$AA?5?$AAu?$AAn?$AAa?$AAb?$AAl?$AAe?$AA?5?$AAt?$AAo?$AA?5?$AAi?$AAn?$AAi?$AAt?$AAi?$AAa?$AAl?$AAi?$AAz?$AAe?$AA?5?$AAh?$AAe@ 100108e8     LIBCMT:crt0msg.obj
 0001:0000f938       ??_C@_1GK@MFGOKLAG@?$AAR?$AA6?$AA0?$AA2?$AA7?$AA?$AN?$AA?6?$AA?9?$AA?5?$AAn?$AAo?$AAt?$AA?5?$AAe?$AAn?$AAo?$AAu?$AAg?$AAh?$AA?5?$AAs?$AAp?$AAa?$AAc?$AAe?$AA?5?$AAf?$AAo?$AAr?$AA?5?$AAl?$AAo@ 10010938     LIBCMT:crt0msg.obj
 0001:0000f9a8       ??_C@_1GK@MCAAGJMO@?$AAR?$AA6?$AA0?$AA2?$AA6?$AA?$AN?$AA?6?$AA?9?$AA?5?$AAn?$AAo?$AAt?$AA?5?$AAe?$AAn?$AAo?$AAu?$AAg?$AAh?$AA?5?$AAs?$AAp?$AAa?$AAc?$AAe?$AA?5?$AAf?$AAo?$AAr?$AA?5?$AAs?$AAt@ 100109a8     LIBCMT:crt0msg.obj
 0001:0000fa18       ??_C@_1EM@MAADIHMB@?$AAR?$AA6?$AA0?$AA2?$AA5?$AA?$AN?$AA?6?$AA?9?$AA?5?$AAp?$AAu?$AAr?$AAe?$AA?5?$AAv?$AAi?$AAr?$AAt?$AAu?$AAa?$AAl?$AA?5?$AAf?$AAu?$AAn?$AAc?$AAt?$AAi?$AAo?$AAn?$AA?5?$AAc@ 10010a18     LIBCMT:crt0msg.obj
 0001:0000fa68       ??_C@_1GK@FHCKBEFA@?$AAR?$AA6?$AA0?$AA2?$AA4?$AA?$AN?$AA?6?$AA?9?$AA?5?$AAn?$AAo?$AAt?$AA?5?$AAe?$AAn?$AAo?$AAu?$AAg?$AAh?$AA?5?$AAs?$AAp?$AAa?$AAc?$AAe?$AA?5?$AAf?$AAo?$AAr?$AA?5?$AA_?$AAo@ 10010a68     LIBCMT:crt0msg.obj
 0001:0000fad8       ??_C@_1FC@ECHBIFBC@?$AAR?$AA6?$AA0?$AA1?$AA9?$AA?$AN?$AA?6?$AA?9?$AA?5?$AAu?$AAn?$AAa?$AAb?$AAl?$AAe?$AA?5?$AAt?$AAo?$AA?5?$AAo?$AAp?$AAe?$AAn?$AA?5?$AAc?$AAo?$AAn?$AAs?$AAo?$AAl?$AAe?$AA?5@ 10010ad8     LIBCMT:crt0msg.obj
 0001:0000fb30       ??_C@_1EC@JIBHAOPH@?$AAR?$AA6?$AA0?$AA1?$AA8?$AA?$AN?$AA?6?$AA?9?$AA?5?$AAu?$AAn?$AAe?$AAx?$AAp?$AAe?$AAc?$AAt?$AAe?$AAd?$AA?5?$AAh?$AAe?$AAa?$AAp?$AA?5?$AAe?$AAr?$AAr?$AAo?$AAr?$AA?$AN?$AA?6@ 10010b30     LIBCMT:crt0msg.obj
 0001:0000fb78       ??_C@_1FK@BEOGODMC@?$AAR?$AA6?$AA0?$AA1?$AA7?$AA?$AN?$AA?6?$AA?9?$AA?5?$AAu?$AAn?$AAe?$AAx?$AAp?$AAe?$AAc?$AAt?$AAe?$AAd?$AA?5?$AAm?$AAu?$AAl?$AAt?$AAi?$AAt?$AAh?$AAr?$AAe?$AAa?$AAd?$AA?5@ 10010b78     LIBCMT:crt0msg.obj
 0001:0000fbd8       ??_C@_1FI@LOGNIKDM@?$AAR?$AA6?$AA0?$AA1?$AA6?$AA?$AN?$AA?6?$AA?9?$AA?5?$AAn?$AAo?$AAt?$AA?5?$AAe?$AAn?$AAo?$AAu?$AAg?$AAh?$AA?5?$AAs?$AAp?$AAa?$AAc?$AAe?$AA?5?$AAf?$AAo?$AAr?$AA?5?$AAt?$AAh@ 10010bd8     LIBCMT:crt0msg.obj
 0001:0000fc30       ??_C@_1EG@BEHAGFJD@?$AAR?$AA6?$AA0?$AA1?$AA0?$AA?$AN?$AA?6?$AA?9?$AA?5?$AAa?$AAb?$AAo?$AAr?$AAt?$AA?$CI?$AA?$CJ?$AA?5?$AAh?$AAa?$AAs?$AA?5?$AAb?$AAe?$AAe?$AAn?$AA?5?$AAc?$AAa?$AAl?$AAl?$AAe?$AAd@ 10010c30     LIBCMT:crt0msg.obj
 0001:0000fc78       ??_C@_1FI@HONFMGBI@?$AAR?$AA6?$AA0?$AA0?$AA9?$AA?$AN?$AA?6?$AA?9?$AA?5?$AAn?$AAo?$AAt?$AA?5?$AAe?$AAn?$AAo?$AAu?$AAg?$AAh?$AA?5?$AAs?$AAp?$AAa?$AAc?$AAe?$AA?5?$AAf?$AAo?$AAr?$AA?5?$AAe?$AAn@ 10010c78     LIBCMT:crt0msg.obj
 0001:0000fcd0       ??_C@_1FE@LLNEDJMD@?$AAR?$AA6?$AA0?$AA0?$AA8?$AA?$AN?$AA?6?$AA?9?$AA?5?$AAn?$AAo?$AAt?$AA?5?$AAe?$AAn?$AAo?$AAu?$AAg?$AAh?$AA?5?$AAs?$AAp?$AAa?$AAc?$AAe?$AA?5?$AAf?$AAo?$AAr?$AA?5?$AAa?$AAr@ 10010cd0     LIBCMT:crt0msg.obj
 0001:0000fd28       ??_C@_1FK@PGACCAFB@?$AAR?$AA6?$AA0?$AA0?$AA2?$AA?$AN?$AA?6?$AA?9?$AA?5?$AAf?$AAl?$AAo?$AAa?$AAt?$AAi?$AAn?$AAg?$AA?5?$AAp?$AAo?$AAi?$AAn?$AAt?$AA?5?$AAs?$AAu?$AAp?$AAp?$AAo?$AAr?$AAt?$AA?5@ 10010d28     LIBCMT:crt0msg.obj
 0001:0000fe38       ??_C@_1EK@MBDPDCGA@?$AAM?$AAi?$AAc?$AAr?$AAo?$AAs?$AAo?$AAf?$AAt?$AA?5?$AAV?$AAi?$AAs?$AAu?$AAa?$AAl?$AA?5?$AAC?$AA?$CL?$AA?$CL?$AA?5?$AAR?$AAu?$AAn?$AAt?$AAi?$AAm?$AAe?$AA?5?$AAL?$AAi?$AAb@ 10010e38     LIBCMT:crt0msg.obj
 0001:0000fe84       ??_C@_15IABLJNFO@?$AA?6?$AA?6?$AA?$AA@ 10010e84     LIBCMT:crt0msg.obj
 0001:0000fe8c       ??_C@_17LGKOMLJ@?$AA?4?$AA?4?$AA?4?$AA?$AA@ 10010e8c     LIBCMT:crt0msg.obj
 0001:0000fe94       ??_C@_1CO@EAEJAADC@?$AA?$DM?$AAp?$AAr?$AAo?$AAg?$AAr?$AAa?$AAm?$AA?5?$AAn?$AAa?$AAm?$AAe?$AA?5?$AAu?$AAn?$AAk?$AAn?$AAo?$AAw?$AAn?$AA?$DO?$AA?$AA@ 10010e94     LIBCMT:crt0msg.obj
 0001:0000fec4       ??_C@_1DE@JNGNBFGO@?$AAR?$AAu?$AAn?$AAt?$AAi?$AAm?$AAe?$AA?5?$AAE?$AAr?$AAr?$AAo?$AAr?$AA?$CB?$AA?6?$AA?6?$AAP?$AAr?$AAo?$AAg?$AAr?$AAa?$AAm?$AA?3?$AA?5?$AA?$AA@ 10010ec4     LIBCMT:crt0msg.obj
 0001:0000ff30       ??_C@_0BG@KLEAJEFJ@Illegal?5byte?5sequence?$AA@ 10010f30     LIBCMT:syserr.obj
 0001:0000ff48       ??_C@_0BE@ICMCHPHH@Directory?5not?5empty?$AA@ 10010f48     LIBCMT:syserr.obj
 0001:0000ff5c       ??_C@_0BJ@IHEHINLI@Function?5not?5implemented?$AA@ 10010f5c     LIBCMT:syserr.obj
 0001:0000ff78       ??_C@_0BD@CLHBCGPB@No?5locks?5available?$AA@ 10010f78     LIBCMT:syserr.obj
 0001:0000ff8c       ??_C@_0BC@BEDIHIDK@Filename?5too?5long?$AA@ 10010f8c     LIBCMT:syserr.obj
 0001:0000ffa0       ??_C@_0BK@JAEBMJJM@Resource?5deadlock?5avoided?$AA@ 10010fa0     LIBCMT:syserr.obj
 0001:0000ffbc       ??_C@_0BB@FCBJFCAJ@Result?5too?5large?$AA@ 10010fbc     LIBCMT:syserr.obj
 0001:0000ffd0       ??_C@_0N@MMJPGLJK@Domain?5error?$AA@ 10010fd0     LIBCMT:syserr.obj
 0001:0000ffe0       ??_C@_0M@LHEPIIOM@Broken?5pipe?$AA@ 10010fe0     LIBCMT:syserr.obj
 0001:0000ffec       ??_C@_0P@PKCJJLLM@Too?5many?5links?$AA@ 10010fec     LIBCMT:syserr.obj
 0001:0000fffc       ??_C@_0BG@DDBFNKBH@Read?9only?5file?5system?$AA@ 10010ffc     LIBCMT:syserr.obj
 0001:00010014       ??_C@_0N@FEHLOILP@Invalid?5seek?$AA@ 10011014     LIBCMT:syserr.obj
 0001:00010024       ??_C@_0BI@FEALHKLD@No?5space?5left?5on?5device?$AA@ 10011024     LIBCMT:syserr.obj
 0001:0001003c       ??_C@_0P@LFMMIPAE@File?5too?5large?$AA@ 1001103c     LIBCMT:syserr.obj
 0001:0001004c       ??_C@_0CE@ONOKNLPF@Inappropriate?5I?1O?5control?5operat@ 1001104c     LIBCMT:syserr.obj
 0001:00010070       ??_C@_0BE@INBJMKGG@Too?5many?5open?5files?$AA@ 10011070     LIBCMT:syserr.obj
 0001:00010084       ??_C@_0BO@IIFBODJE@Too?5many?5open?5files?5in?5system?$AA@ 10011084     LIBCMT:syserr.obj
 0001:000100a4       ??_C@_0BB@HMGGCEBG@Invalid?5argument?$AA@ 100110a4     LIBCMT:syserr.obj
 0001:000100b8       ??_C@_0P@NDHGCGKE@Is?5a?5directory?$AA@ 100110b8     LIBCMT:syserr.obj
 0001:000100c8       ??_C@_0BA@CJBACOOL@Not?5a?5directory?$AA@ 100110c8     LIBCMT:syserr.obj
 0001:000100d8       ??_C@_0P@NLEIANHE@No?5such?5device?$AA@ 100110d8     LIBCMT:syserr.obj
 0001:000100e8       ??_C@_0O@OAMDNOCP@Improper?5link?$AA@ 100110e8     LIBCMT:syserr.obj
 0001:000100f8       ??_C@_0M@NAAJNNGH@File?5exists?$AA@ 100110f8     LIBCMT:syserr.obj
 0001:00010104       ??_C@_0BA@BIBLIOEK@Resource?5device?$AA@ 10011104     LIBCMT:syserr.obj
 0001:00010114       ??_C@_0O@NIPGCINC@Unknown?5error?$AA@ 10011114     LIBCMT:syserr.obj
 0001:00010124       ??_C@_0M@LOEHLCJD@Bad?5address?$AA@ 10011124     LIBCMT:syserr.obj
 0001:00010130       ??_C@_0BC@HFNFNKAI@Permission?5denied?$AA@ 10011130     LIBCMT:syserr.obj
 0001:00010144       ??_C@_0BB@IMDKMPFB@Not?5enough?5space?$AA@ 10011144     LIBCMT:syserr.obj
 0001:00010158       ??_C@_0CB@EPFKGNAK@Resource?5temporarily?5unavailable@ 10011158     LIBCMT:syserr.obj
 0001:0001017c       ??_C@_0BD@LOHELEP@No?5child?5processes?$AA@ 1001117c     LIBCMT:syserr.obj
 0001:00010190       ??_C@_0BE@NFGDDCEF@Bad?5file?5descriptor?$AA@ 10011190     LIBCMT:syserr.obj
 0001:000101a4       ??_C@_0BC@HKPNECK@Exec?5format?5error?$AA@ 100111a4     LIBCMT:syserr.obj
 0001:000101b8       ??_C@_0BC@MFFGCDFL@Arg?5list?5too?5long?$AA@ 100111b8     LIBCMT:syserr.obj
 0001:000101cc       ??_C@_0BK@DPKMCKJ@No?5such?5device?5or?5address?$AA@ 100111cc     LIBCMT:syserr.obj
 0001:000101e8       ??_C@_0BD@KKNFOBBD@Input?1output?5error?$AA@ 100111e8     LIBCMT:syserr.obj
 0001:000101fc       ??_C@_0BK@FJBOAFDK@Interrupted?5function?5call?$AA@ 100111fc     LIBCMT:syserr.obj
 0001:00010218       ??_C@_0BA@FKIAIBGA@No?5such?5process?$AA@ 10011218     LIBCMT:syserr.obj
 0001:00010228       ??_C@_0BK@FMDHKPNF@No?5such?5file?5or?5directory?$AA@ 10011228     LIBCMT:syserr.obj
 0001:00010244       ??_C@_0BI@BJFCGOHL@Operation?5not?5permitted?$AA@ 10011244     LIBCMT:syserr.obj
 0001:0001025c       ??_C@_08INEPGKHH@No?5error?$AA@ 1001125c     LIBCMT:syserr.obj
 0001:00010268       ??_C@_1BK@DBDEIDLH@?$AAK?$AAE?$AAR?$AAN?$AAE?$AAL?$AA3?$AA2?$AA?4?$AAD?$AAL?$AAL?$AA?$AA@ 10011268     LIBCMT:tidtable.obj
 0001:00010284       ??_C@_07PEJMOBNF@FlsFree?$AA@ 10011284     LIBCMT:tidtable.obj
 0001:0001028c       ??_C@_0M@JCPCPOEF@FlsSetValue?$AA@ 1001128c     LIBCMT:tidtable.obj
 0001:00010298       ??_C@_0M@GDNOONDI@FlsGetValue?$AA@ 10011298     LIBCMT:tidtable.obj
 0001:000102a4       ??_C@_08KNHFBNJ@FlsAlloc?$AA@ 100112a4     LIBCMT:tidtable.obj
 0001:000102b0       ___newctype                100112b0     LIBCMT:ctype.obj
 0001:000105b0       __wctype                   100115b0     LIBCMT:ctype.obj
 0001:000107b8       ___newclmap                100117b8     LIBCMT:ctype.obj
 0001:00010938       ___newcumap                10011938     LIBCMT:ctype.obj
 0001:00010ab8       ??_C@_1BC@GDGBMEMK@?$AAH?$AAH?$AA?3?$AAm?$AAm?$AA?3?$AAs?$AAs?$AA?$AA@ 10011ab8     LIBCMT:nlsdata2.obj
 0001:00010acc       ??_C@_1CI@KNAKOEBC@?$AAd?$AAd?$AAd?$AAd?$AA?0?$AA?5?$AAM?$AAM?$AAM?$AAM?$AA?5?$AAd?$AAd?$AA?0?$AA?5?$AAy?$AAy?$AAy?$AAy?$AA?$AA@ 10011acc     LIBCMT:nlsdata2.obj
 0001:00010af4       ??_C@_1BC@IEBCMHCM@?$AAM?$AAM?$AA?1?$AAd?$AAd?$AA?1?$AAy?$AAy?$AA?$AA@ 10011af4     LIBCMT:nlsdata2.obj
 0001:00010b08       ??_C@_15CLMNNGEL@?$AAP?$AAM?$AA?$AA@ 10011b08     LIBCMT:nlsdata2.obj
 0001:00010b10       ??_C@_15ODEHAHHF@?$AAA?$AAM?$AA?$AA@ 10011b10     LIBCMT:nlsdata2.obj
 0001:00010b18       ??_C@_1BC@FEMKIFH@?$AAD?$AAe?$AAc?$AAe?$AAm?$AAb?$AAe?$AAr?$AA?$AA@ 10011b18     LIBCMT:nlsdata2.obj
 0001:00010b2c       ??_C@_1BC@BGLIFPF@?$AAN?$AAo?$AAv?$AAe?$AAm?$AAb?$AAe?$AAr?$AA?$AA@ 10011b2c     LIBCMT:nlsdata2.obj
 0001:00010b40       ??_C@_1BA@EPANDLNG@?$AAO?$AAc?$AAt?$AAo?$AAb?$AAe?$AAr?$AA?$AA@ 10011b40     LIBCMT:nlsdata2.obj
 0001:00010b50       ??_C@_1BE@DKAAMBJL@?$AAS?$AAe?$AAp?$AAt?$AAe?$AAm?$AAb?$AAe?$AAr?$AA?$AA@ 10011b50     LIBCMT:nlsdata2.obj
 0001:00010b64       ??_C@_1O@PAHLKOAC@?$AAA?$AAu?$AAg?$AAu?$AAs?$AAt?$AA?$AA@ 10011b64     LIBCMT:nlsdata2.obj
 0001:00010b74       ??_C@_19BIFMLPCD@?$AAJ?$AAu?$AAl?$AAy?$AA?$AA@ 10011b74     LIBCMT:nlsdata2.obj
 0001:00010b80       ??_C@_19EPFLPGAP@?$AAJ?$AAu?$AAn?$AAe?$AA?$AA@ 10011b80     LIBCMT:nlsdata2.obj
 0001:00010b8c       ??_C@_1M@GJNLMHFD@?$AAA?$AAp?$AAr?$AAi?$AAl?$AA?$AA@ 10011b8c     LIBCMT:nlsdata2.obj
 0001:00010b98       ??_C@_1M@IKEENEDF@?$AAM?$AAa?$AAr?$AAc?$AAh?$AA?$AA@ 10011b98     LIBCMT:nlsdata2.obj
 0001:00010ba4       ??_C@_1BC@JGDDFFAM@?$AAF?$AAe?$AAb?$AAr?$AAu?$AAa?$AAr?$AAy?$AA?$AA@ 10011ba4     LIBCMT:nlsdata2.obj
 0001:00010bb8       ??_C@_1BA@EFMEIEBA@?$AAJ?$AAa?$AAn?$AAu?$AAa?$AAr?$AAy?$AA?$AA@ 10011bb8     LIBCMT:nlsdata2.obj
 0001:00010bc8       ??_C@_17EGKACKIF@?$AAD?$AAe?$AAc?$AA?$AA@ 10011bc8     LIBCMT:nlsdata2.obj
 0001:00010bd0       ??_C@_17BBDMLCIG@?$AAN?$AAo?$AAv?$AA?$AA@ 10011bd0     LIBCMT:nlsdata2.obj
 0001:00010bd8       ??_C@_17FNLKOI@?$AAO?$AAc?$AAt?$AA?$AA@ 10011bd8     LIBCMT:nlsdata2.obj
 0001:00010be0       ??_C@_17HCHCOKMG@?$AAS?$AAe?$AAp?$AA?$AA@ 10011be0     LIBCMT:nlsdata2.obj
 0001:00010be8       ??_C@_17ICPELBCN@?$AAA?$AAu?$AAg?$AA?$AA@ 10011be8     LIBCMT:nlsdata2.obj
 0001:00010bf0       ??_C@_17IJPCKHK@?$AAJ?$AAu?$AAl?$AA?$AA@ 10011bf0     LIBCMT:nlsdata2.obj
 0001:00010bf8       ??_C@_17KCJGOCPB@?$AAJ?$AAu?$AAn?$AA?$AA@ 10011bf8     LIBCMT:nlsdata2.obj
 0001:00010c00       ??_C@_17PNNKMEED@?$AAM?$AAa?$AAy?$AA?$AA@ 10011c00     LIBCMT:nlsdata2.obj
 0001:00010c08       ??_C@_17LFPOIHDD@?$AAA?$AAp?$AAr?$AA?$AA@ 10011c08     LIBCMT:nlsdata2.obj
 0001:00010c10       ??_C@_17CKNLEDEC@?$AAM?$AAa?$AAr?$AA?$AA@ 10011c10     LIBCMT:nlsdata2.obj
 0001:00010c18       ??_C@_17LMDJEKJN@?$AAF?$AAe?$AAb?$AA?$AA@ 10011c18     LIBCMT:nlsdata2.obj
 0001:00010c20       ??_C@_17DKNBKCHM@?$AAJ?$AAa?$AAn?$AA?$AA@ 10011c20     LIBCMT:nlsdata2.obj
 0001:00010c28       ??_C@_1BC@ENMNNPAJ@?$AAS?$AAa?$AAt?$AAu?$AAr?$AAd?$AAa?$AAy?$AA?$AA@ 10011c28     LIBCMT:nlsdata2.obj
 0001:00010c3c       ??_C@_1O@PDICJHAG@?$AAF?$AAr?$AAi?$AAd?$AAa?$AAy?$AA?$AA@ 10011c3c     LIBCMT:nlsdata2.obj
 0001:00010c4c       ??_C@_1BC@HHMNLIHE@?$AAT?$AAh?$AAu?$AAr?$AAs?$AAd?$AAa?$AAy?$AA?$AA@ 10011c4c     LIBCMT:nlsdata2.obj
 0001:00010c60       ??_C@_1BE@EBOGMDOH@?$AAW?$AAe?$AAd?$AAn?$AAe?$AAs?$AAd?$AAa?$AAy?$AA?$AA@ 10011c60     LIBCMT:nlsdata2.obj
 0001:00010c74       ??_C@_1BA@ENFBFFEK@?$AAT?$AAu?$AAe?$AAs?$AAd?$AAa?$AAy?$AA?$AA@ 10011c74     LIBCMT:nlsdata2.obj
 0001:00010c84       ??_C@_1O@MMNBFLIA@?$AAM?$AAo?$AAn?$AAd?$AAa?$AAy?$AA?$AA@ 10011c84     LIBCMT:nlsdata2.obj
 0001:00010c94       ??_C@_1O@IHNHDHPB@?$AAS?$AAu?$AAn?$AAd?$AAa?$AAy?$AA?$AA@ 10011c94     LIBCMT:nlsdata2.obj
 0001:00010ca4       ??_C@_17GGIBDPIH@?$AAS?$AAa?$AAt?$AA?$AA@ 10011ca4     LIBCMT:nlsdata2.obj
 0001:00010cac       ??_C@_17HFOLPPLP@?$AAF?$AAr?$AAi?$AA?$AA@ 10011cac     LIBCMT:nlsdata2.obj
 0001:00010cb4       ??_C@_17PDPHAADD@?$AAT?$AAh?$AAu?$AA?$AA@ 10011cb4     LIBCMT:nlsdata2.obj
 0001:00010cbc       ??_C@_17CJEDCEPE@?$AAW?$AAe?$AAd?$AA?$AA@ 10011cbc     LIBCMT:nlsdata2.obj
 0001:00010cc4       ??_C@_17BMKGEGOJ@?$AAT?$AAu?$AAe?$AA?$AA@ 10011cc4     LIBCMT:nlsdata2.obj
 0001:00010ccc       ??_C@_17KBOMKBF@?$AAM?$AAo?$AAn?$AA?$AA@ 10011ccc     LIBCMT:nlsdata2.obj
 0001:00010cd4       ??_C@_17MBGCMIPB@?$AAS?$AAu?$AAn?$AA?$AA@ 10011cd4     LIBCMT:nlsdata2.obj
 0001:00010cdc       ??_C@_08JCCMCCIL@HH?3mm?3ss?$AA@ 10011cdc     LIBCMT:nlsdata2.obj
 0001:00010ce8       ??_C@_0BE@CKGJFCPC@dddd?0?5MMMM?5dd?0?5yyyy?$AA@ 10011ce8     LIBCMT:nlsdata2.obj
 0001:00010cfc       ??_C@_08BPBNCDIB@MM?1dd?1yy?$AA@ 10011cfc     LIBCMT:nlsdata2.obj
 0001:00010d08       ??_C@_02CJNFDJBF@PM?$AA@   10011d08     LIBCMT:nlsdata2.obj
 0001:00010d0c       ??_C@_02DEDBPAFC@AM?$AA@   10011d0c     LIBCMT:nlsdata2.obj
 0001:00010d10       ??_C@_08EDHMEBNP@December?$AA@ 10011d10     LIBCMT:nlsdata2.obj
 0001:00010d1c       ??_C@_08HCHEGEOA@November?$AA@ 10011d1c     LIBCMT:nlsdata2.obj
 0001:00010d28       ??_C@_07JJNFCEND@October?$AA@ 10011d28     LIBCMT:nlsdata2.obj
 0001:00010d30       ??_C@_09BHHEALKD@September?$AA@ 10011d30     LIBCMT:nlsdata2.obj
 0001:00010d3c       ??_C@_06LBBHFDDG@August?$AA@ 10011d3c     LIBCMT:nlsdata2.obj
 0001:00010d44       ??_C@_04MIEPOIFP@July?$AA@ 10011d44     LIBCMT:nlsdata2.obj
 0001:00010d4c       ??_C@_04CNLMGBGM@June?$AA@ 10011d4c     LIBCMT:nlsdata2.obj
 0001:00010d54       ??_C@_05DMJDNLEJ@April?$AA@ 10011d54     LIBCMT:nlsdata2.obj
 0001:00010d5c       ??_C@_05HPCKOFNC@March?$AA@ 10011d5c     LIBCMT:nlsdata2.obj
 0001:00010d64       ??_C@_08GNJGEPFN@February?$AA@ 10011d64     LIBCMT:nlsdata2.obj
 0001:00010d70       ??_C@_07CGJPFGJA@January?$AA@ 10011d70     LIBCMT:nlsdata2.obj
 0001:00010d78       ??_C@_03MKABNOCG@Dec?$AA@  10011d78     LIBCMT:nlsdata2.obj
 0001:00010d7c       ??_C@_03JPJOFNIA@Nov?$AA@  10011d7c     LIBCMT:nlsdata2.obj
 0001:00010d80       ??_C@_03BMAOKBAD@Oct?$AA@  10011d80     LIBCMT:nlsdata2.obj
 0001:00010d84       ??_C@_03GGCAPAJC@Sep?$AA@  10011d84     LIBCMT:nlsdata2.obj
 0001:00010d88       ??_C@_03IFJFEIGA@Aug?$AA@  10011d88     LIBCMT:nlsdata2.obj
 0001:00010d8c       ??_C@_03LBGABGKK@Jul?$AA@  10011d8c     LIBCMT:nlsdata2.obj
 0001:00010d90       ??_C@_03IDFGHECI@Jun?$AA@  10011d90     LIBCMT:nlsdata2.obj
 0001:00010d94       ??_C@_03CNMDKL@May?$AA@    10011d94     LIBCMT:nlsdata2.obj
 0001:00010d98       ??_C@_03LEOLGMJP@Apr?$AA@  10011d98     LIBCMT:nlsdata2.obj
 0001:00010d9c       ??_C@_03ODNJBKGA@Mar?$AA@  10011d9c     LIBCMT:nlsdata2.obj
 0001:00010da0       ??_C@_03HJBDCHOM@Feb?$AA@  10011da0     LIBCMT:nlsdata2.obj
 0001:00010da4       ??_C@_03JIHJHPIE@Jan?$AA@  10011da4     LIBCMT:nlsdata2.obj
 0001:00010da8       ??_C@_08INBOOONO@Saturday?$AA@ 10011da8     LIBCMT:nlsdata2.obj
 0001:00010db4       ??_C@_06JECMNKMI@Friday?$AA@ 10011db4     LIBCMT:nlsdata2.obj
 0001:00010dbc       ??_C@_08HACCIKIA@Thursday?$AA@ 10011dbc     LIBCMT:nlsdata2.obj
 0001:00010dc8       ??_C@_09DLIGFAKA@Wednesday?$AA@ 10011dc8     LIBCMT:nlsdata2.obj
 0001:00010dd4       ??_C@_07BAAGCFCM@Tuesday?$AA@ 10011dd4     LIBCMT:nlsdata2.obj
 0001:00010ddc       ??_C@_06JLEDEDGH@Monday?$AA@ 10011ddc     LIBCMT:nlsdata2.obj
 0001:00010de4       ??_C@_06OOPIFAJ@Sunday?$AA@ 10011de4     LIBCMT:nlsdata2.obj
 0001:00010dec       ??_C@_03FEFJNEK@Sat?$AA@   10011dec     LIBCMT:nlsdata2.obj
 0001:00010df0       ??_C@_03IDIOELNC@Fri?$AA@  10011df0     LIBCMT:nlsdata2.obj
 0001:00010df4       ??_C@_03IOFIKPDN@Thu?$AA@  10011df4     LIBCMT:nlsdata2.obj
 0001:00010df8       ??_C@_03MHOMLAJA@Wed?$AA@  10011df8     LIBCMT:nlsdata2.obj
 0001:00010dfc       ??_C@_03NAGEINEP@Tue?$AA@  10011dfc     LIBCMT:nlsdata2.obj
 0001:00010e00       ??_C@_03PDAGKDH@Mon?$AA@   10011e00     LIBCMT:nlsdata2.obj
 0001:00010e04       ??_C@_03KOEHGMDN@Sun?$AA@  10011e04     LIBCMT:nlsdata2.obj
 0001:00010e88       ??_C@_19CDGLJBOD@?$AA?4?$AAc?$AAo?$AAm?$AA?$AA@ 10011e88     LIBCMT:wspawnve.obj
 0001:00010e94       ??_C@_19DOGDICKI@?$AA?4?$AAe?$AAx?$AAe?$AA?$AA@ 10011e94     LIBCMT:wspawnve.obj
 0001:00010ea0       ??_C@_19PINKOIBI@?$AA?4?$AAb?$AAa?$AAt?$AA?$AA@ 10011ea0     LIBCMT:wspawnve.obj
 0001:00010eac       ??_C@_19BDKLHPGC@?$AA?4?$AAc?$AAm?$AAd?$AA?$AA@ 10011eac     LIBCMT:wspawnve.obj
 0001:00010eb8       ??_C@_15PCEAIKAA@?$AA?4?$AA?2?$AA?$AA@ 10011eb8     LIBCMT:wspawnve.obj
 0001:00010ec0       __XcptActTab               10011ec0     LIBCMT:winxfltr.obj
 0001:00010f50       __First_FPE_Indx           10011f50     LIBCMT:winxfltr.obj
 0001:00010f54       __Num_FPE                  10011f54     LIBCMT:winxfltr.obj
 0001:00010f58       __XcptActTabSize           10011f58     LIBCMT:winxfltr.obj
 0001:00010f5c       __XcptActTabCount          10011f5c     LIBCMT:winxfltr.obj
 0001:00010f60       ___lookuptable_s           10011f60     LIBCMT:outputs.obj
 0001:00010fbc       ??_C@_0BI@DFKBFLJE@GetProcessWindowStation?$AA@ 10011fbc     LIBCMT:crtmboxw.obj
 0001:00010fd4       ??_C@_0BK@DEKFELLI@GetUserObjectInformationW?$AA@ 10011fd4     LIBCMT:crtmboxw.obj
 0001:00010ff0       ??_C@_0BD@HHGDFDBJ@GetLastActivePopup?$AA@ 10011ff0     LIBCMT:crtmboxw.obj
 0001:00011004       ??_C@_0BA@HNOPNCHB@GetActiveWindow?$AA@ 10012004     LIBCMT:crtmboxw.obj
 0001:00011014       ??_C@_0M@DLDCCGNP@MessageBoxW?$AA@ 10012014     LIBCMT:crtmboxw.obj
 0001:00011020       ??_C@_1BG@GOEBHBDC@?$AAU?$AAS?$AAE?$AAR?$AA3?$AA2?$AA?4?$AAD?$AAL?$AAL?$AA?$AA@ 10012020     LIBCMT:crtmboxw.obj
 0001:00011040       ??_C@_13NMPKAAJP@?$AA?$DN?$AA?$AA@ 10012040     LIBCMT:wcenvarg.obj
 0001:00011044       ??_C@_1BG@FIGGICF@?$AAS?$AAy?$AAs?$AAt?$AAe?$AAm?$AAR?$AAo?$AAo?$AAt?$AA?$AA@ 10012044     LIBCMT:wcenvarg.obj
 0001:0001105c       ??_C@_06IMKFLFPG@1?$CDQNAN?$AA@ 1001205c     LIBCMT:_x10fout_.obj
 0001:00011064       ??_C@_05DNEBIAHO@1?$CDINF?$AA@ 10012064     LIBCMT:_x10fout_.obj
 0001:0001106c       ??_C@_05PHHOCPM@1?$CDIND?$AA@ 1001206c     LIBCMT:_x10fout_.obj
 0001:00011074       ??_C@_06PGGFOGJG@1?$CDSNAN?$AA@ 10012074     LIBCMT:_x10fout_.obj
 0001:0001107c       ??_C@_1BA@BALFACEM@?$AAC?$AAO?$AAN?$AAO?$AAU?$AAT?$AA$?$AA?$AA@ 1001207c     LIBCMT:initcon.obj
 0001:00011090       __load_config_used         10012090     LIBCMT:loadcfg.obj
 0001:000110e0       ___safe_se_handler_table   100120e0     <linker-defined>
 0001:000110ec       ___rtc_iaa                 100120ec     LIBCMT:_initsect_.obj
 0001:000110f0       ___rtc_izz                 100120f0     LIBCMT:_initsect_.obj
 0001:000110f4       ___rtc_taa                 100120f4     LIBCMT:_initsect_.obj
 0001:000110f8       ___rtc_tzz                 100120f8     LIBCMT:_initsect_.obj
 0001:00011100       __alloca_probe             10012100     chkstk.obj
 0001:00011100       __chkstk                   10012100 f   chkstk.obj
 0001:00011130       _bit64_pushuserdata        10012130 f   bit64.obj
 0001:00011170       _bit64_push                10012170 f   bit64.obj
 0001:00011200       _bit64_getvalue            10012200 f   bit64.obj
 0001:00012b40       _luaopen_bit64             10013b40 f   bit64.obj
 0001:00012b80       _traceback                 10013b80 f   exported.obj
 0001:00012c10       _GetExportFunction         10013c10 f   exported.obj
 0001:00012ca0       _pcall_msg                 10013ca0 f   exported.obj
 0001:00012d50       _ReplacePluginInfoCollector 10013d50 f   exported.obj
 0001:00012d80       _DestroyCollector          10013d80 f   exported.obj
 0001:00012dc0       _AddStringToCollectorField 10013dc0 f   exported.obj
 0001:00012e20       _AddBufToCollector         10013e20 f   exported.obj
 0001:00012e70       _CreateStringsArray        10013e70 f   exported.obj
 0001:00012fa0       _FarPanelItemFreeCallback@8 10013fa0 f   exported.obj
 0001:00012fd0       _FillPluginPanelItem       10013fd0 f   exported.obj
 0001:000131c0       _FillFindData              100141c0 f   exported.obj
 0001:00013500       _LF_GetFindData            10014500 f   exported.obj
 0001:000135d0       _LF_FreeFindData           100145d0 f   exported.obj
 0001:00013620       _UpdateFileSelection       10014620 f   exported.obj
 0001:000136f0       _LF_GetFiles               100146f0 f   exported.obj
 0001:00013a00       _LF_RunDefaultScript       10014a00 f   exported.obj
 0001:00013b30       _LF_Analyse                10014b30 f   exported.obj
 0001:00013bd0       _LF_CloseAnalyse           10014bd0 f   exported.obj
 0001:00013bf0       _LF_GetOpenPanelInfo       10014bf0 f   exported.obj
 0001:00014250       _PushFarMacroValue         10015250 f   exported.obj
 0001:00014350       _PackMacroValues           10015350 f   exported.obj
 0001:000146f0       _LF_Open                   100156f0 f   exported.obj
 0001:00014a70       _LF_ClosePanel             10015a70 f   exported.obj
 0001:00014b10       _LF_Compare                10015b10 f   exported.obj
 0001:00014bc0       _LF_Configure              10015bc0 f   exported.obj
 0001:00014c20       _LF_DeleteFiles            10015c20 f   exported.obj
 0001:00014cd0       _LF_MakeDirectory          10015cd0 f   exported.obj
 0001:00014de0       _LF_ProcessPanelEvent      10015de0 f   exported.obj
 0001:00014ea0       _LF_ProcessHostFile        10015ea0 f   exported.obj
 0001:00014f80       _LF_ProcessPanelInput      10015f80 f   exported.obj
 0001:00015010       _LF_PutFiles               10016010 f   exported.obj
 0001:00015100       _LF_SetDirectory           10016100 f   exported.obj
 0001:000151a0       _LF_SetFindList            100161a0 f   exported.obj
 0001:00015230       _LF_ExitFAR                10016230 f   exported.obj
 0001:00015260       _getPluginMenuItems        10016260 f   exported.obj
 0001:000152f0       _LF_GetPluginInfo          100162f0 f   exported.obj
 0001:000153f0       _LF_ProcessEditorInput     100163f0 f   exported.obj
 0001:00015450       _LF_ProcessEditorEvent     10016450 f   exported.obj
 0001:00015570       _LF_ProcessViewerEvent     10016570 f   exported.obj
 0001:000155f0       _LF_ProcessDialogEvent     100165f0 f   exported.obj
 0001:000157e0       _LF_ProcessSynchroEvent    100167e0 f   exported.obj
 0001:00015990       _LF_GetContentFields       10016990 f   exported.obj
 0001:00015a20       _LF_GetContentData         10016a20 f   exported.obj
 0001:00015b30       _LF_FreeContentData        10016b30 f   exported.obj
 0001:00015b60       _LF_GetGlobalInfo          10016b60 f   exported.obj
 0001:00015f00       _LF_ProcessConsoleInput    10016f00 f   exported.obj
 0001:00015ff0       _push_flags_table          10016ff0 f   flags.obj
 0001:00016040       _SetFarColors              10017040 f   keysandcolors.obj
 0001:00016180       _LF_LoadFile               10017180 f   lflua.obj
 0001:000163c0       _luaB_loadfileW            100173c0 f   lflua.obj
 0001:00016400       _luaB_dofileW              10017400 f   lflua.obj
 0001:00016450       _LF_Gsub                   10017450 f   lflua.obj
 0001:00016560       _method_gc                 10017560 f   lregex.obj
 0001:000165c0       _method_tostring           100175c0 f   lregex.obj
 0001:00016610       _check_regex_pattern       10017610 f   lregex.obj
 0001:000166b0       _push_far_regex            100176b0 f   lregex.obj
 0001:00016730       __regex_gmatch_closure     10017730 f   lregex.obj
 0001:00016820       _regex_gmatch_closure      10017820 f   lregex.obj
 0001:00016830       _regex_gmatch_closureW     10017830 f   lregex.obj
 0001:00016840       __Gmatch                   10017840 f   lregex.obj
 0001:00016920       _func_Gmatch               10017920 f   lregex.obj
 0001:00016930       _func_GmatchW              10017930 f   lregex.obj
 0001:00016940       _rx_find_match             10017940 f   lregex.obj
 0001:00016b80       _method_bracketscount      10017b80 f   lregex.obj
 0001:00016be0       _rx_gsub                   10017be0 f   lregex.obj
 0001:00017300       _func_New                  10018300 f   lregex.obj
 0001:00017330       _method_find               10018330 f   lregex.obj
 0001:00017350       _func_find                 10018350 f   lregex.obj
 0001:00017370       _method_findW              10018370 f   lregex.obj
 0001:00017390       _func_findW                10018390 f   lregex.obj
 0001:000173b0       _method_match              100183b0 f   lregex.obj
 0001:000173d0       _func_match                100183d0 f   lregex.obj
 0001:000173f0       _method_matchW             100183f0 f   lregex.obj
 0001:00017410       _func_matchW               10018410 f   lregex.obj
 0001:00017430       _method_gsub               10018430 f   lregex.obj
 0001:00017450       _func_gsub                 10018450 f   lregex.obj
 0001:00017470       _method_gsubW              10018470 f   lregex.obj
 0001:00017490       _func_gsubW                10018490 f   lregex.obj
 0001:000174b0       _luaopen_regex             100184b0 f   lregex.obj
 0001:00017590       _Open_Luamacro             10018590 f   luamacro.obj
 0001:00017980       _far_MacroCallFar          10018980 f   luamacro.obj
 0001:00017b20       _far_FarMacroCallToLua     10018b20 f   luamacro.obj
 0001:00017b90       _CheckFarUserControl       10018b90 f   lusercontrol.obj
 0001:00017be0       _uc_len                    10018be0 f   lusercontrol.obj
 0001:00017de0       _luaopen_usercontrol       10018de0 f   lusercontrol.obj
 0001:00017e20       _CreateRegKey              10018e20 f   reg.obj
 0001:00017e60       _OpenRegKey                10018e60 f   reg.obj
 0001:00017e90       _SetRegKeyStr              10018e90 f   reg.obj
 0001:00017f10       _SetRegKeyDword            10018f10 f   reg.obj
 0001:00017f70       _SetRegKeyArr              10018f70 f   reg.obj
 0001:00017fd0       _IsLuaJIT                  10018fd0 f   service.obj
 0001:00017fe0       _DllMain@12                10018fe0 f   service.obj
 0001:00018070       _OptHandle                 10019070 f   service.obj
 0001:00018280       _GetFlagCombination        10019280 f   service.obj
 0001:00018520       _GetFlagsFromTable         10019520 f   service.obj
 0001:00018560       _PutFlagsToTable           10019560 f   service.obj
 0001:00018590       _GetPluginData             10019590 f   service.obj
 0001:000185b0       _ConvertLuaValue           100195b0 f   service.obj
 0001:00018840       _PutMouseEvent             10019840 f   service.obj
 0001:000189f0       _PushPanelItem             100199f0 f   service.obj
 0001:00018c30       _PushPanelItems            10019c30 f   service.obj
 0001:0001aae0       _GetFarColor               1001bae0 f   service.obj
 0001:0001ac30       _PushFarColor              1001bc30 f   service.obj
 0001:0001b100       _PushInputRecord           1001c100 f   service.obj
 0001:0001b320       _FillInputRecord           1001c320 f   service.obj
 0001:0001be10       _LF_Message                1001ce10 f   service.obj
 0001:0001c280       _LF_Error                  1001d280 f   service.obj
 0001:0001db60       _CreateList                1001eb60 f   service.obj
 0001:0001e220       _NewDialogData             1001f220 f   service.obj
 0001:0001e290       _DialogHandleEqual         1001f290 f   service.obj
 0001:0001e2d0       _PushDMParams              1001f2d0 f   service.obj
 0001:0001f4b0       _PushDNParams              100204b0 f   service.obj
 0001:0001f700       _ProcessDNResult           10020700 f   service.obj
 0001:0001f960       _LF_DlgProc                10020960 f   service.obj
 0001:00022590       _MacroAddCallback@12       10023590 f   service.obj
 0001:00022a10       _pushFileTime              10023a10 f   service.obj
 0001:00022d90       _NewVirtualKeyTable        10023d90 f   service.obj
 0001:00023ac0       _TimerThreadFunc@4         10024ac0 f   service.obj
 0001:000240e0       _dir_exist                 100250e0 f   service.obj
 0001:00024d20       _LF_RunLuafarInit          10025d20 f   service.obj
 0001:00024de0       _LF_ProcessEnvVars         10025de0 f   service.obj
 0001:00024df0       _LF_InitLuaState1          10025df0 f   service.obj
 0001:00024f50       _LF_MacroCallback          10025f50 f   service.obj
 0001:00024f60       _LF_DoFile                 10025f60 f   service.obj
 0001:00024ff0       _LF_GetLuafarAPI           10025ff0 f   service.obj
 0001:000252c0       _LF_InitLuaState2          100262c0 f   service.obj
 0001:00027b30       _luaopen_unicode           10028b30 f   slnunico.obj
 0001:00028bd0       _luaopen_uio               10029bd0 f   uliolib51.obj
 0001:00029a80       _luaopen_upackage          1002aa80 f   uloadlib51.obj
 0001:00029bc0       _PutIntToArray             1002abc0 f   ustring.obj
 0001:00029bf0       _PutIntToTable             1002abf0 f   ustring.obj
 0001:00029c20       _PutNumToTable             1002ac20 f   ustring.obj
 0001:00029c50       _PutBoolToTable            1002ac50 f   ustring.obj
 0001:00029c80       _PutStrToTable             1002ac80 f   ustring.obj
 0001:00029cb0       _PutStrToArray             1002acb0 f   ustring.obj
 0001:00029ce0       _PutLStrToTable            1002ace0 f   ustring.obj
 0001:00029d10       _GetOptNumFromTable        1002ad10 f   ustring.obj
 0001:00029d60       _GetOptIntFromTable        1002ad60 f   ustring.obj
 0001:00029db0       _GetOptIntFromArray        1002adb0 f   ustring.obj
 0001:00029e00       _GetBoolFromTable          1002ae00 f   ustring.obj
 0001:00029e30       _GetOptBoolFromTable       1002ae30 f   ustring.obj
 0001:00029e90       _convert_multibyte_string  1002ae90 f   ustring.obj
 0001:00029f80       _check_utf8_string         1002af80 f   ustring.obj
 0001:00029fb0       _utf8_to_utf16             1002afb0 f   ustring.obj
 0001:0002a080       _opt_utf8_string           1002b080 f   ustring.obj
 0001:0002a150       _oem_to_utf16              1002b150 f   ustring.obj
 0001:0002a220       _push_multibyte_string     1002b220 f   ustring.obj
 0001:0002a2d0       _push_utf8_string          1002b2d0 f   ustring.obj
 0001:0002a2f0       _ustring_WideCharToMultiByte 1002b2f0 f   ustring.obj
 0001:0002a420       _ustring_OemToUtf8         1002b420 f   ustring.obj
 0001:0002a460       _ustring_Utf8ToOem         1002b460 f   ustring.obj
 0001:0002a510       _ustring_Utf16ToUtf8       1002b510 f   ustring.obj
 0001:0002a550       _ustring_Utf8ToUtf16       1002b550 f   ustring.obj
 0001:0002a600       _ustring_GetACP            1002b600 f   ustring.obj
 0001:0002a620       _ustring_GetOEMCP          1002b620 f   ustring.obj
 0001:0002a640       _ustring_GetDriveType      1002b640 f   ustring.obj
 0001:0002a720       _ustring_Uuid              1002b720 f   ustring.obj
 0001:0002a800       _ustring_SearchPath        1002b800 f   ustring.obj
 0001:0002aa00       _ustring_Sleep             1002ba00 f   ustring.obj
 0001:0002aa50       _PushAttrString            1002ba50 f   ustring.obj
 0001:0002aae0       _PutAttrToTable            1002bae0 f   ustring.obj
 0001:0002ab10       _DecodeAttributes          1002bb10 f   ustring.obj
 0001:0002abe0       _ustring_SHGetFolderPath   1002bbe0 f   ustring.obj
 0001:0002ace0       _push_utf16_string         1002bce0 f   ustring.obj
 0001:0002ad20       _ustring_sub               1002bd20 f   ustring.obj
 0001:0002adb0       _ustring_len               1002bdb0 f   ustring.obj
 0001:0002ade0       _check_utf16_string        1002bde0 f   ustring.obj
 0001:0002ae10       _opt_utf16_string          1002be10 f   ustring.obj
 0001:0002b020       _luaopen_ustring           1002c020 f   ustring.obj
 0001:0002b070       _pusherrorcode             1002c070 f   ustring.obj
 0001:0002b0f0       _pusherror                 1002c0f0 f   ustring.obj
 0001:0002b110       _SysErrorReturn            1002c110 f   ustring.obj
 0001:0002b140       _PutWStrToTable            1002c140 f   ustring.obj
 0001:0002b170       _PutWStrToArray            1002c170 f   ustring.obj
 0001:0002b1b0       _ustring_MultiByteToWideChar 1002c1b0 f   ustring.obj
 0001:0002b300       _EnumCodePagesProc@4       1002c300 f   ustring.obj
 0001:0002b3c0       _ustring_EnumSystemCodePages 1002c3c0 f   ustring.obj
 0001:0002b430       _ustring_GetCPInfo         1002c430 f   ustring.obj
 0001:0002b620       _ustring_GetLogicalDriveStrings 1002c620 f   ustring.obj
 0001:0002b760       _ustring_GlobalMemoryStatus 1002c760 f   ustring.obj
 0001:0002ba10       _ustring_SetFileAttr       1002ca10 f   ustring.obj
 0001:0002bb00       _ustring_GetFileAttr       1002cb00 f   ustring.obj
 0001:0002bbe0       _ustring_GetCurrentDir     1002cbe0 f   ustring.obj
 0001:0002bd70       _ustring_SetCurrentDir     1002cd70 f   ustring.obj
 0001:0002be50       _luaLF_SlotError           1002ce50 f   util.obj
 0001:0002be90       _luaLF_FieldError          1002ce90 f   util.obj
 0001:0002bed0       _GetIntFromArray           1002ced0 f   util.obj
 0001:0002bf50       _GetFileSizeFromTable      1002cf50 f   util.obj
 0001:0002bfc0       _GetFileTimeFromTable      1002cfc0 f   util.obj
 0001:0002c040       _PutFileTimeToTable        1002d040 f   util.obj
 0001:0002c080       _GetAttrFromTable          1002d080 f   util.obj
 0001:0002d640       _luaopen_win               1002e640 f   win.obj
 0001:0002d6ac       _lua_setmetatable          1002e6ac f   lua51:lua51.dll
 0001:0002d6b2       _lua_getfield              1002e6b2 f   lua51:lua51.dll
 0001:0002d6b8       _lua_newuserdata           1002e6b8 f   lua51:lua51.dll
 0001:0002d6be       _lua_pushnumber            1002e6be f   lua51:lua51.dll
 0001:0002d6c4       _lua_touserdata            1002e6c4 f   lua51:lua51.dll
 0001:0002d6ca       _lua_settop                1002e6ca f   lua51:lua51.dll
 0001:0002d6d0       _lua_rawequal              1002e6d0 f   lua51:lua51.dll
 0001:0002d6d6       _lua_getmetatable          1002e6d6 f   lua51:lua51.dll
 0001:0002d6dc       _lua_type                  1002e6dc f   lua51:lua51.dll
 0001:0002d6e2       _luaL_argerror             1002e6e2 f   lua51:lua51.dll
 0001:0002d6e8       _lua_tonumber              1002e6e8 f   lua51:lua51.dll
 0001:0002d6ee       _lua_gettop                1002e6ee f   lua51:lua51.dll
 0001:0002d6f4       _luaL_checkinteger         1002e6f4 f   lua51:lua51.dll
 0001:0002d6fa       _lua_pushnil               1002e6fa f   lua51:lua51.dll
 0001:0002d700       _lua_tolstring             1002e700 f   lua51:lua51.dll
 0001:0002d706       _lua_pushstring            1002e706 f   lua51:lua51.dll
 0001:0002d70c       _lua_pushboolean           1002e70c f   lua51:lua51.dll
 0001:0002d712       _luaL_register             1002e712 f   lua51:lua51.dll
 0001:0002d718       _luaL_newmetatable         1002e718 f   lua51:lua51.dll
 0001:0002d71e       _lua_call                  1002e71e f   lua51:lua51.dll
 0001:0002d724       _lua_pushinteger           1002e724 f   lua51:lua51.dll
 0001:0002d72a       _lua_pushvalue             1002e72a f   lua51:lua51.dll
 0001:0002d730       _lua_gc                    1002e730 f   lua51:lua51.dll
 0001:0002d736       _lua_remove                1002e736 f   lua51:lua51.dll
 0001:0002d73c       _lua_pcall                 1002e73c f   lua51:lua51.dll
 0001:0002d742       _lua_insert                1002e742 f   lua51:lua51.dll
 0001:0002d748       _lua_pushcclosure          1002e748 f   lua51:lua51.dll
 0001:0002d74e       _lua_rawgeti               1002e74e f   lua51:lua51.dll
 0001:0002d754       _lua_setfield              1002e754 f   lua51:lua51.dll
 0001:0002d75a       _lua_createtable           1002e75a f   lua51:lua51.dll
 0001:0002d760       _lua_rawseti               1002e760 f   lua51:lua51.dll
 0001:0002d766       _lua_objlen                1002e766 f   lua51:lua51.dll
 0001:0002d76c       _lua_isstring              1002e76c f   lua51:lua51.dll
 0001:0002d772       _lua_gettable              1002e772 f   lua51:lua51.dll
 0001:0002d778       _luaL_unref                1002e778 f   lua51:lua51.dll
 0001:0002d77e       _luaL_ref                  1002e77e f   lua51:lua51.dll
 0001:0002d784       _lua_toboolean             1002e784 f   lua51:lua51.dll
 0001:0002d78a       _lua_tointeger             1002e78a f   lua51:lua51.dll
 0001:0002d790       _lua_isnumber              1002e790 f   lua51:lua51.dll
 0001:0002d796       _lua_pushlightuserdata     1002e796 f   lua51:lua51.dll
 0001:0002d79c       _lua_pushlstring           1002e79c f   lua51:lua51.dll
 0001:0002d7a2       _luaL_loadstring           1002e7a2 f   lua51:lua51.dll
 0001:0002d7a8       _lua_pushfstring           1002e7a8 f   lua51:lua51.dll
 0001:0002d7ae       _lua_load                  1002e7ae f   lua51:lua51.dll
 0001:0002d7b4       _lua_concat                1002e7b4 f   lua51:lua51.dll
 0001:0002d7ba       _lua_error                 1002e7ba f   lua51:lua51.dll
 0001:0002d7c0       _luaL_pushresult           1002e7c0 f   lua51:lua51.dll
 0001:0002d7c6       _luaL_addlstring           1002e7c6 f   lua51:lua51.dll
 0001:0002d7cc       _luaL_buffinit             1002e7cc f   lua51:lua51.dll
 0001:0002d7d2       _luaL_checkudata           1002e7d2 f   lua51:lua51.dll
 0001:0002d7d8       _lua_replace               1002e7d8 f   lua51:lua51.dll
 0001:0002d7de       _luaL_optlstring           1002e7de f   lua51:lua51.dll
 0001:0002d7e4       _luaL_checklstring         1002e7e4 f   lua51:lua51.dll
 0001:0002d7ea       _luaL_error                1002e7ea f   lua51:lua51.dll
 0001:0002d7f0       _lua_checkstack            1002e7f0 f   lua51:lua51.dll
 0001:0002d7f6       _luaL_optinteger           1002e7f6 f   lua51:lua51.dll
 0001:0002d7fc       _luaL_addvalue             1002e7fc f   lua51:lua51.dll
 0001:0002d802       _lua_getinfo               1002e802 f   lua51:lua51.dll
 0001:0002d808       _lua_getstack              1002e808 f   lua51:lua51.dll
 0001:0002d80e       _luaL_checktype            1002e80e f   lua51:lua51.dll
 0001:0002d814       _luaopen_debug             1002e814 f   lua51:lua51.dll
 0001:0002d81a       _luaopen_math              1002e81a f   lua51:lua51.dll
 0001:0002d820       _luaopen_string            1002e820 f   lua51:lua51.dll
 0001:0002d826       _luaopen_os                1002e826 f   lua51:lua51.dll
 0001:0002d82c       _luaopen_table             1002e82c f   lua51:lua51.dll
 0001:0002d832       _luaopen_base              1002e832 f   lua51:lua51.dll
 0001:0002d838       _luaL_typerror             1002e838 f   lua51:lua51.dll
 0001:0002d83e       _lua_next                  1002e83e f   lua51:lua51.dll
 0001:0002d844       _lua_getallocf             1002e844 f   lua51:lua51.dll
 0001:0002d84a       _lua_rawset                1002e84a f   lua51:lua51.dll
 0001:0002d850       _luaL_optnumber            1002e850 f   lua51:lua51.dll
 0001:0002d856       _lua_rawget                1002e856 f   lua51:lua51.dll
 0001:0002d85c       _luaL_checkany             1002e85c f   lua51:lua51.dll
 0001:0002d862       _lua_settable              1002e862 f   lua51:lua51.dll
 0001:0002d868       _lua_setfenv               1002e868 f   lua51:lua51.dll
 0001:0002d86e       _lua_getfenv               1002e86e f   lua51:lua51.dll
 0001:0002d874       _luaL_checknumber          1002e874 f   lua51:lua51.dll
 0001:0002d87a       _lua_setallocf             1002e87a f   lua51:lua51.dll
 0001:0002d880       _luaL_prepbuffer           1002e880 f   lua51:lua51.dll
 0001:0002d886       _luaL_checkstack           1002e886 f   lua51:lua51.dll
 0001:0002d88c       _lua_dump                  1002e88c f   lua51:lua51.dll
 0001:0002d892       _lua_typename              1002e892 f   lua51:lua51.dll
 0001:0002d898       _lua_tocfunction           1002e898 f   lua51:lua51.dll
 0001:0002d89e       _luaL_checkoption          1002e89e f   lua51:lua51.dll
 0001:0002d8a4       _luaL_gsub                 1002e8a4 f   lua51:lua51.dll
 0001:0002d8aa       _lua_iscfunction           1002e8aa f   lua51:lua51.dll
 0001:0002d8b0       _luaL_findtable            1002e8b0 f   lua51:lua51.dll
 0001:0002d8b6       _lua_isuserdata            1002e8b6 f   lua51:lua51.dll
 0001:0002d8bc       __cfltcvt_init             1002e8bc f   LIBCMT:_fpinit_.obj
 0001:0002d91c       __fpmath                   1002e91c f   LIBCMT:_fpinit_.obj
 0001:0002d940       __ftol2_sse                1002e940 f   LIBCMT:ftol2.obj
 0001:0002d949       __ftol2_pentium4           1002e949 f   LIBCMT:ftol2.obj
 0001:0002d95c       __ftol2_sse_excpt          1002e95c f   LIBCMT:ftol2.obj
 0001:0002d976       __ftol2                    1002e976 f   LIBCMT:ftol2.obj
 0001:0002d9f0       __allshl                   1002e9f0 f   LIBCMT:llshl.obj
 0001:0002da10       __aullshr                  1002ea10 f   LIBCMT:ullshr.obj
 0001:0002da30       __allshr                   1002ea30 f   LIBCMT:llshr.obj
 0001:0002da51       _sprintf                   1002ea51 f   LIBCMT:sprintf.obj
 0001:0002dae0       __allmul                   1002eae0 f   LIBCMT:llmul.obj
 0001:0002db20       __alldiv                   1002eb20 f   LIBCMT:lldiv.obj
 0001:0002dbd0       __allrem                   1002ebd0 f   LIBCMT:llrem.obj
 0001:0002ddb0       __control87                1002edb0 f i LIBCMT:_ieee87_.obj
 0001:0002e0d0       _memset                    1002f0d0 f   LIBCMT:memset.obj
 0001:0002e14a       _free                      1002f14a f   LIBCMT:free.obj
 0001:0002e184       _malloc                    1002f184 f   LIBCMT:malloc.obj
 0001:0002e218       __fclose_nolock            1002f218 f   LIBCMT:fclose.obj
 0001:0002e285       _fclose                    1002f285 f   LIBCMT:fclose.obj
 0001:0002e2f9       __wfsopen                  1002f2f9 f   LIBCMT:wfopen.obj
 0001:0002e3b7       __wfopen                   1002f3b7 f   LIBCMT:wfopen.obj
 0001:0002e3ce       _wcsrchr                   1002f3ce f   LIBCMT:wcsrchr.obj
 0001:0002e400       _memcpy                    1002f400 f   LIBCMT:memcpy.obj
 0001:0002e761       __wcsdup                   1002f761 f   LIBCMT:wcsdup.obj
 0001:0002e761       _wcsdup                    1002f761 f   LIBCMT:wcsdup.obj
 0001:0002e7b6       __fread_nolock_s           1002f7b6 f   LIBCMT:fread.obj
 0001:0002e972       _fread_s                   1002f972 f   LIBCMT:fread.obj
 0001:0002ea00       _fread                     1002fa00 f   LIBCMT:fread.obj
 0001:0002ea1d       _feof                      1002fa1d f   LIBCMT:feoferr.obj
 0001:0002ea45       _ferror                    1002fa45 f   LIBCMT:feoferr.obj
 0001:0002ea6d       __get_sys_err_msg          1002fa6d f i LIBCMT:strerror.obj
 0001:0002ea95       _strerror                  1002fa95 f   LIBCMT:strerror.obj
 0001:0002eaff       __get_errno_from_oserr     1002faff f   LIBCMT:dosmap.obj
 0001:0002eb41       __errno                    1002fb41 f   LIBCMT:dosmap.obj
 0001:0002eb54       ___doserrno                1002fb54 f   LIBCMT:dosmap.obj
 0001:0002eb67       __dosmaperr                1002fb67 f   LIBCMT:dosmap.obj
 0001:0002eb8a       _rewind                    1002fb8a f   LIBCMT:rewind.obj
 0001:0002ec48       _getc                      1002fc48 f   LIBCMT:fgetc.obj
 0001:0002ed3c       __ungetc_nolock            1002fd3c f   LIBCMT:ungetc.obj
 0001:0002ee1f       _ungetc                    1002fe1f f   LIBCMT:ungetc.obj
 0001:0002ee88       __wfreopen_helper          1002fe88 f   LIBCMT:wfreopen.obj
 0001:0002ef5a       __wfreopen                 1002ff5a f   LIBCMT:wfreopen.obj
 0001:0002ef80       ___iob_func                1002ff80 f   LIBCMT:_file.obj
 0001:0002ef86       ___initstdio               1002ff86 f   LIBCMT:_file.obj
 0001:0002f037       ___endstdio                10030037 f   LIBCMT:_file.obj
 0001:0002f057       __lock_file                10030057 f   LIBCMT:_file.obj
 0001:0002f098       __lock_file2               10030098 f   LIBCMT:_file.obj
 0001:0002f0ca       __unlock_file              100300ca f   LIBCMT:_file.obj
 0001:0002f106       __unlock_file2             10030106 f   LIBCMT:_file.obj
 0001:0002f135       _wcsstr                    10030135 f   LIBCMT:wcsstr.obj
 0001:0002f1b0       _strchr                    100301b0 f   LIBCMT:strchr.obj
 0001:0002f1b6       ___from_strstr_to_strchr   100301b6     LIBCMT:strchr.obj
 0001:0002f26e       _wcsncpy                   1003026e f   LIBCMT:wcsncpy.obj
 0001:0002f2ba       _iswctype                  100302ba f   LIBCMT:iswctype.obj
 0001:0002f30f       _wcschr                    1003030f f   LIBCMT:wcschr.obj
 0001:0002f336       ??0_LocaleUpdate@@QAE@PAUlocaleinfo_struct@@@Z 10030336 f i LIBCMT:wcsicmp.obj
 0001:0002f3bd       __wcsicmp_l                100303bd f   LIBCMT:wcsicmp.obj
 0001:0002f4c0       __wcsicmp                  100304c0 f   LIBCMT:wcsicmp.obj
 0001:0002f54b       _strncmp                   1003054b f   LIBCMT:strncmp.obj
 0001:0002f610       __aulldiv                  10030610 f   LIBCMT:ulldiv.obj
 0001:0002f678       _fprintf                   10030678 f   LIBCMT:fprintf.obj
 0001:0002f784       __isdigit_l                10030784 f i LIBCMT:_ctype.obj
 0001:0002f7d5       _isdigit                   100307d5 f i LIBCMT:_ctype.obj
 0001:0002f803       __isxdigit_l               10030803 f i LIBCMT:_ctype.obj
 0001:0002f859       _isxdigit                  10030859 f i LIBCMT:_ctype.obj
 0001:0002f889       __isspace_l                10030889 f i LIBCMT:_ctype.obj
 0001:0002f8da       _isspace                   100308da f i LIBCMT:_ctype.obj
 0001:0002f910       _memchr                    10030910 f   LIBCMT:memchr.obj
 0001:0002f9c0       _strpbrk                   100309c0 f   LIBCMT:strpbrk.obj
 0001:0002fa00       _strncpy                   10030a00 f   LIBCMT:strncpy.obj
 0001:0002fb24       __snwprintf                10030b24 f   LIBCMT:snwprint.obj
 0001:0002fbf4       __pclose                   10030bf4 f   LIBCMT:popen.obj
 0001:0002fd1d       __wpopen                   10030d1d f   LIBCMT:wpopen.obj
 0001:00030289       __tmpfile_helper           10031289 f   LIBCMT:tmpfile.obj
 0001:0003047c       _tmpfile                   1003147c f   LIBCMT:tmpfile.obj
 0001:00030498       _vfscanf                   10031498 f   LIBCMT:fscanf.obj
 0001:00030592       _fscanf                    10031592 f   LIBCMT:fscanf.obj
 0001:000305b2       _fgets                     100315b2 f   LIBCMT:fgets.obj
 0001:000306ea       _clearerr_s                100316ea f   LIBCMT:clearerr.obj
 0001:0003078e       _clearerr                  1003178e f   LIBCMT:clearerr.obj
 0001:00030799       __fwrite_nolock            10031799 f   LIBCMT:fwrite.obj
 0001:000308f0       _fwrite                    100318f0 f   LIBCMT:fwrite.obj
 0001:0003096a       __ftell_nolock             1003196a f   LIBCMT:ftell.obj
 0001:00030afe       _ftell                     10031afe f   LIBCMT:ftell.obj
 0001:00030b63       __fseek_nolock             10031b63 f   LIBCMT:fseek.obj
 0001:00030bed       _fseek                     10031bed f   LIBCMT:fseek.obj
 0001:00030c69       _setvbuf                   10031c69 f   LIBCMT:setvbuf.obj
 0001:00030d5f       __flush                    10031d5f f   LIBCMT:fflush.obj
 0001:00030dc7       __fflush_nolock            10031dc7 f   LIBCMT:fflush.obj
 0001:00030ee9       _fflush                    10031ee9 f   LIBCMT:fflush.obj
 0001:00030f3c       __flushall                 10031f3c f   LIBCMT:fflush.obj
 0001:00030f50       _strrchr                   10031f50 f   LIBCMT:strrchr.obj
 0001:00030f7d       __wgetenv_helper_nolock    10031f7d f   LIBCMT:wgetenv.obj
 0001:00031018       __wgetenv                  10032018 f   LIBCMT:wgetenv.obj
 0001:00031092       __wdupenv_s                10032092 f   LIBCMT:wgetenv.obj
 0001:00031169       __wsystem                  10032169 f   LIBCMT:wsystem.obj
 0001:00031250       __alldvrm                  10032250 f   LIBCMT:lldvrm.obj
 0001:0003132f       _wcscmp                    1003232f f   LIBCMT:wcscmp.obj
 0001:0003136d       __CRT_INIT@12              1003236d f   LIBCMT:dllcrt0.obj
 0001:000315c7       __DllMainCRTStartup@12     100325c7 f   LIBCMT:dllcrt0.obj
 0001:000315ea       __forcdecpt_l              100325ea f   LIBCMT:cvt.obj
 0001:0003165e       __cropzeros_l              1003265e f   LIBCMT:cvt.obj
 0001:000316e0       __positive                 100326e0 f   LIBCMT:cvt.obj
 0001:000316fc       __fassign_l                100326fc f   LIBCMT:cvt.obj
 0001:0003173e       __fassign                  1003273e f   LIBCMT:cvt.obj
 0001:00031777       __forcdecpt                10032777 f   LIBCMT:cvt.obj
 0001:0003178a       __cropzeros                1003278a f   LIBCMT:cvt.obj
 0001:000318fe       __cftoe_l                  100328fe f   LIBCMT:cvt.obj
 0001:000319c5       __cftoe                    100329c5 f   LIBCMT:cvt.obj
 0001:000319e5       __cftoa_l                  100329e5 f   LIBCMT:cvt.obj
 0001:00031e5e       __cftof_l                  10032e5e f   LIBCMT:cvt.obj
 0001:00031f1f       __cftog_l                  10032f1f f   LIBCMT:cvt.obj
 0001:0003200c       __cfltcvt_l                1003300c f   LIBCMT:cvt.obj
 0001:00032094       __cfltcvt                  10033094 f   LIBCMT:cvt.obj
 0001:000320b7       __initp_misc_cfltcvt_tab   100330b7 f   LIBCMT:cmiscdat.obj
 0001:000320da       __setdefaultprecision      100330da f   LIBCMT:fp8.obj
 0001:00032102       ___sse2_available_init     10033102 f   LIBCMT:cpu_disp.obj
 0001:00032112       __flsbuf                   10033112 f   LIBCMT:_flsbuf.obj
 0001:0003231d       __output_l                 1003331d f   LIBCMT:output.obj
 0001:00032ec9       __initp_misc_invarg        10033ec9 f   LIBCMT:invarg.obj
 0001:00032ed8       __call_reportfault         10033ed8 f   LIBCMT:invarg.obj
 0001:00033001       __invoke_watson            10034001 f   LIBCMT:invarg.obj
 0001:00033026       __invalid_parameter        10034026 f   LIBCMT:invarg.obj
 0001:00033053       __invalid_parameter_noinfo 10034053 f   LIBCMT:invarg.obj
 0001:00033063       __controlfp_s              10034063 f   LIBCMT:_contrlfp_.obj
 0001:000330c2       ___set_fpsr_sse2           100340c2 f   LIBCMT:_fpctrl_.obj
 0001:00033134       __initp_misc_winsig        10034134 f   LIBCMT:winsig.obj
 0001:00033189       ___get_sigabrt             10034189 f   LIBCMT:winsig.obj
 0001:00033196       _raise                     10034196 f   LIBCMT:winsig.obj
 0001:00033339       __VEC_memzero              10034339 f   LIBCMT:p4_memset.obj
 0001:000333f3       __heap_init                100343f3 f   LIBCMT:heapinit.obj
 0001:00033411       __heap_term                10034411 f   LIBCMT:heapinit.obj
 0001:00033425       ___crtCorExitProcess       10034425 f   LIBCMT:crt0dat.obj
 0001:00033450       ___crtExitProcess          10034450 f   LIBCMT:crt0dat.obj
 0001:00033468       __lockexit                 10034468 f   LIBCMT:crt0dat.obj
 0001:00033471       __unlockexit               10034471 f   LIBCMT:crt0dat.obj
 0001:0003347a       __init_pointers            1003447a f   LIBCMT:crt0dat.obj
 0001:000334ad       __initterm_e               100344ad f   LIBCMT:crt0dat.obj
 0001:000334d1       __cinit                    100344d1 f   LIBCMT:crt0dat.obj
 0001:000336a8       __exit                     100346a8 f   LIBCMT:crt0dat.obj
 0001:000336be       __cexit                    100346be f   LIBCMT:crt0dat.obj
 0001:000336cd       __amsg_exit                100346cd f   LIBCMT:crt0dat.obj
 0001:000336eb       __GET_RTERRMSG             100346eb f   LIBCMT:crt0msg.obj
 0001:00033711       __NMSG_WRITE               10034711 f   LIBCMT:crt0msg.obj
 0001:000338c0       __FF_MSGBANNER             100348c0 f   LIBCMT:crt0msg.obj
 0001:000338f9       __initp_heap_handler       100348f9 f   LIBCMT:handler.obj
 0001:00033908       __callnewh                 10034908 f   LIBCMT:handler.obj
 0001:00033930       __close_nolock             10034930 f   LIBCMT:close.obj
 0001:000339cc       __close                    100349cc f   LIBCMT:close.obj
 0001:00033a90       __fileno                   10034a90 f   LIBCMT:fileno.obj
 0001:00033ab6       __freebuf                  10034ab6 f   LIBCMT:_freebuf.obj
 0001:00033af0       __SEH_prolog4              10034af0 f   LIBCMT:sehprolg4.obj
 0001:00033b35       __SEH_epilog4              10034b35 f   LIBCMT:sehprolg4.obj
 0001:00033b50       __except_handler4          10034b50 f   LIBCMT:chandler4.obj
 0001:00033cdf       __wopenfile                10034cdf f   LIBCMT:_wopen.obj
 0001:00033f9a       __getstream                10034f9a f   LIBCMT:stream.obj
 0001:000340d0       __local_unwind4            100350d0 f   LIBCMT:exsup4.obj
 0001:000341a6       __seh_longjmp_unwind4@4    100351a6 f   LIBCMT:exsup4.obj
 0001:000341c2       @_EH4_CallFilterFunc@8     100351c2 f   LIBCMT:exsup4.obj
 0001:000341d9       @_EH4_TransferToHandler@8  100351d9 f   LIBCMT:exsup4.obj
 0001:000341f2       @_EH4_GlobalUnwind2@8      100351f2 f   LIBCMT:exsup4.obj
 0001:0003420b       @_EH4_LocalUnwind@16       1003520b f   LIBCMT:exsup4.obj
 0001:00034222       __VEC_memcpy               10035222 f   LIBCMT:p4_memcpy.obj
 0001:00034325       _wcscpy_s                  10035325 f   LIBCMT:wcscpy_s.obj
 0001:00034388       _calloc                    10035388 f   LIBCMT:calloc.obj
 0001:000343c8       _wcslen                    100353c8 f   LIBCMT:wcslen.obj
 0001:000343e3       __filbuf                   100353e3 f   LIBCMT:_filbuf.obj
 0001:00034505       __read_nolock              10035505 f   LIBCMT:read.obj
 0001:00034abc       __read                     10035abc f   LIBCMT:read.obj
 0001:00034bb2       _memcpy_s                  10035bb2 f   LIBCMT:memcpy_s.obj
 0001:00034c27       ___sys_nerr                10035c27 f   LIBCMT:syserr.obj
 0001:00034c2d       ___sys_errlist             10035c2d f   LIBCMT:syserr.obj
 0001:00034c33       _strcpy_s                  10035c33 f   LIBCMT:strcpy_s.obj
 0001:00034c92       __malloc_crt               10035c92 f   LIBCMT:crtheap.obj
 0001:00034cd7       __calloc_crt               10035cd7 f   LIBCMT:crtheap.obj
 0001:00034d23       __realloc_crt              10035d23 f   LIBCMT:crtheap.obj
 0001:00034d71       __recalloc_crt             10035d71 f   LIBCMT:crtheap.obj
 0001:00034dc3       __encoded_null             10035dc3 f   LIBCMT:tidtable.obj
 0001:00034dcc       ___crtTlsAlloc@4           10035dcc f   LIBCMT:tidtable.obj
 0001:00034dd5       ___set_flsgetvalue         10035dd5 f   LIBCMT:tidtable.obj
 0001:00034e09       __mtterm                   10035e09 f   LIBCMT:tidtable.obj
 0001:00034e46       __initptd                  10035e46 f   LIBCMT:tidtable.obj
 0001:00034efa       __getptd_noexit            10035efa f   LIBCMT:tidtable.obj
 0001:00034f73       __getptd                   10035f73 f   LIBCMT:tidtable.obj
 0001:00034f8d       __freefls@4                10035f8d f   LIBCMT:tidtable.obj
 0001:000350bc       __freeptd                  100360bc f   LIBCMT:tidtable.obj
 0001:0003512a       __mtinit                   1003612a f   LIBCMT:tidtable.obj
 0001:000352a5       __lseek_nolock             100362a5 f   LIBCMT:lseek.obj
 0001:0003531a       __lseek                    1003631a f   LIBCMT:lseek.obj
 0001:000353ee       __ioinit                   100363ee f   LIBCMT:ioinit.obj
 0001:00035633       __ioterm                   10036633 f   LIBCMT:ioinit.obj
 0001:00035686       __getbuf                   10036686 f   LIBCMT:_getbuf.obj
 0001:000356cf       __fcloseall                100366cf f   LIBCMT:closeall.obj
 0001:0003576b       __mtinitlocks              1003676b f   LIBCMT:mlock.obj
 0001:000357b5       __mtdeletelocks            100367b5 f   LIBCMT:mlock.obj
 0001:0003580c       __unlock                   1003680c f   LIBCMT:mlock.obj
 0001:00035823       __mtinitlocknum            10036823 f   LIBCMT:mlock.obj
 0001:000358e5       __lock                     100368e5 f   LIBCMT:mlock.obj
 0001:00035b3b       ___updatetmbcinfo          10036b3b f   LIBCMT:mbctype.obj
 0001:00035c5b       __setmbcp_nolock           10036c5b f   LIBCMT:mbctype.obj
 0001:00035e44       __setmbcp                  10036e44 f   LIBCMT:mbctype.obj
 0001:00035fde       ___initmbctable            10036fde f   LIBCMT:mbctype.obj
 0001:00035ffc       ___addlocaleref            10036ffc f   LIBCMT:localref.obj
 0001:0003608b       ___removelocaleref         1003708b f   LIBCMT:localref.obj
 0001:00036124       ___freetlocinfo            10037124 f   LIBCMT:localref.obj
 0001:0003626f       __updatetlocinfoEx_nolock  1003726f f   LIBCMT:localref.obj
 0001:000362bc       ___updatetlocinfo          100372bc f   LIBCMT:localref.obj
 0001:00036335       __towlower_l               10037335 f   LIBCMT:towlower.obj
 0001:000363d5       __stbuf                    100373d5 f   LIBCMT:_sftbuf.obj
 0001:00036471       __ftbuf                    10037471 f   LIBCMT:_sftbuf.obj
 0001:000364a5       __isctype_l                100374a5 f   LIBCMT:isctype.obj
 0001:00036605       __woutput_l                10037605 f   LIBCMT:woutput.obj
 0001:000371c9       __mbsrchr_l                100381c9 f   LIBCMT:mbsrchr.obj
 0001:00037273       __mbsrchr                  10038273 f   LIBCMT:mbsrchr.obj
 0001:0003728a       _strcat_s                  1003828a f   LIBCMT:strcat_s.obj
 0001:00037300       _strlen                    10038300 f   LIBCMT:strlen.obj
 0001:0003738b       __pipe                     1003838b f   LIBCMT:pipe.obj
 0001:00037631       __cwait                    10038631 f   LIBCMT:wait.obj
 0001:000376c2       __wgetpath                 100386c2 f   LIBCMT:wgetpath.obj
 0001:00037773       __waccess_s                10038773 f   LIBCMT:waccess.obj
 0001:000377f2       _wcscat_s                  100387f2 f   LIBCMT:wcscat_s.obj
 0001:00037867       __wfdopen                  10038867 f   LIBCMT:wfdopen.obj
 0001:000379f0       __SEH_prolog4_GS           100389f0 f   LIBCMT:sehprolg4gs.obj
 0001:00037a38       __SEH_epilog4_GS           10038a38 f   LIBCMT:sehprolg4gs.obj
 0001:00037b01       __ultoa_s                  10038b01 f   LIBCMT:xtoas.obj
 0001:00037b1b       __getpid                   10038b1b f   LIBCMT:getpid.obj
 0001:00037d4c       _strtoul                   10038d4c f   LIBCMT:strtol.obj
 0001:00037d78       @__security_check_cookie@4 10038d78 f   LIBCMT:secchk.obj
 0001:00037d87       __rmtmp                    10038d87 f   LIBCMT:rmtmp.obj
 0001:00037e30       __strdup                   10038e30 f   LIBCMT:strdup.obj
 0001:000385b6       __sopen_helper             100395b6 f   LIBCMT:open.obj
 0001:0003867a       __sopen_s                  1003967a f   LIBCMT:open.obj
 0001:00038751       __input_l                  10039751 f   LIBCMT:input.obj
 0001:00039755       __write_nolock             1003a755 f   LIBCMT:write.obj
 0001:00039e52       __write                    1003ae52 f   LIBCMT:write.obj
 0001:00039f26       __commit                   1003af26 f   LIBCMT:commit.obj
 0001:00039fff       __wcsnicoll_l              1003afff f   LIBCMT:wcsnicol.obj
 0001:0003a11f       __wcsnicoll                1003b11f f   LIBCMT:wcsnicol.obj
 0001:0003a1d9       ___mbtow_environ           1003b1d9 f   LIBCMT:mbtowenv.obj
 0001:0003a260       __wsetenvp                 1003b260 f   LIBCMT:wstdenvp.obj
 0001:0003a33c       ___crtGetEnvironmentStringsW 1003b33c f   LIBCMT:w_env.obj
 0001:0003a394       _wcsnlen                   1003b394 f   LIBCMT:wcslen_s.obj
 0001:0003a3b4       __wspawnvpe                1003b3b4 f   LIBCMT:wspwnvpe.obj
 0001:0003a63e       __wspawnve                 1003b63e f   LIBCMT:wspawnve.obj
 0001:0003a82c       __setenvp                  1003b82c f   LIBCMT:stdenvp.obj
 0001:0003aaa2       __setargv                  1003baa2 f   LIBCMT:stdargv.obj
 0001:0003ab5d       ___crtGetEnvironmentStringsA 1003bb5d f   LIBCMT:a_env.obj
 0001:0003abf4       __RTC_Initialize           1003bbf4 f   LIBCMT:_initsect_.obj
 0001:0003ac1a       __RTC_Terminate            1003bc1a f   LIBCMT:_initsect_.obj
 0001:0003ac40       __XcptFilter               1003bc40 f   LIBCMT:winxfltr.obj
 0001:0003ad8a       ___CppXcptFilter           1003bd8a f   LIBCMT:winxfltr.obj
 0001:0003adaa       ___security_init_cookie    1003bdaa f   LIBCMT:gs_support.obj
 0001:0003ae45       __tolower_l                1003be45 f   LIBCMT:tolower.obj
 0001:0003af5a       _tolower                   1003bf5a f   LIBCMT:tolower.obj
 0001:0003af86       __atodbl_l                 1003bf86 f   LIBCMT:atodbl.obj
 0001:0003b02e       __atoflt_l                 1003c02e f   LIBCMT:atodbl.obj
 0001:0003b0e0       _memmove                   1003c0e0 f   LIBCMT:memmove.obj
 0001:0003b441       __fptostr                  1003c441 f   LIBCMT:_fptostr.obj
 0001:0003b4f4       ___dtold                   1003c4f4 f   LIBCMT:_cfout_.obj
 0001:0003b5a7       __fltout2                  1003c5a7 f   LIBCMT:_cfout_.obj
 0001:0003b635       __fptrap                   1003c635 f   LIBCMT:crt0fp.obj
 0001:0003b63e       __lseeki64_nolock          1003c63e f   LIBCMT:lseeki64.obj
 0001:0003b6c3       __lseeki64                 1003c6c3 f   LIBCMT:lseeki64.obj
 0001:0003b7ad       __isatty                   1003c7ad f   LIBCMT:isatty.obj
 0001:0003b803       __get_printf_count_output  1003c803 f   LIBCMT:printf.obj
 0001:0003b819       __wctomb_s_l               1003c819 f   LIBCMT:wctomb.obj
 0001:0003b96e       _wctomb_s                  1003c96e f   LIBCMT:wctomb.obj
 0001:0003b98b       __isleadbyte_l             1003c98b f i LIBCMT:_wctype.obj
 0001:0003b9c3       _isleadbyte                1003c9c3 f i LIBCMT:_wctype.obj
 0001:0003b9e0       __aulldvrm                 1003c9e0 f   LIBCMT:ulldvrm.obj
 0001:0003ba75       __crt_debugger_hook        1003ca75 f   LIBCMT:dbghook.obj
 0001:0003ba7d       ?terminate@@YAXXZ          1003ca7d f   LIBCMT:hooks.obj
 0001:0003bab6       __initp_eh_hooks           1003cab6 f   LIBCMT:hooks.obj
 0001:0003bac7       __initp_misc_rand_s        1003cac7 f   LIBCMT:rand_s.obj
 0001:0003bad6       __initp_misc_purevirt      1003cad6 f   LIBCMT:inithelp.obj
 0001:0003bb9b       ___onexitinit              1003cb9b f   LIBCMT:onexit.obj
 0001:0003bbcc       __onexit                   1003cbcc f   LIBCMT:onexit.obj
 0001:0003bc08       _atexit                    1003cc08 f   LIBCMT:onexit.obj
 0001:0003bc20       __ValidateImageBase        1003cc20 f   LIBCMT:pesect.obj
 0001:0003bc60       __FindPESection            1003cc60 f   LIBCMT:pesect.obj
 0001:0003bcb0       __IsNonwritableInCurrentImage 1003ccb0 f   LIBCMT:pesect.obj
 0001:0003bd6c       ___crtMessageBoxW          1003cd6c f   LIBCMT:crtmboxw.obj
 0001:0003bed8       _wcsncpy_s                 1003ced8 f   LIBCMT:wcsncpy_s.obj
 0001:0003bfa5       __set_error_mode           1003cfa5 f   LIBCMT:errmode.obj
 0001:0003bfe4       __set_osfhnd               1003cfe4 f   LIBCMT:osfinfo.obj
 0001:0003c065       __free_osfhnd              1003d065 f   LIBCMT:osfinfo.obj
 0001:0003c0eb       __get_osfhandle            1003d0eb f   LIBCMT:osfinfo.obj
 0001:0003c154       ___lock_fhandle            1003d154 f   LIBCMT:osfinfo.obj
 0001:0003c1f3       __unlock_fhandle           1003d1f3 f   LIBCMT:osfinfo.obj
 0001:0003c21a       __alloc_osfhnd             1003d21a f   LIBCMT:osfinfo.obj
 0001:0003cae8       __wsopen_helper            1003dae8 f   LIBCMT:wopen.obj
 0001:0003cbac       __wsopen_s                 1003dbac f   LIBCMT:wopen.obj
 0001:0003cbcc       __wcsnicmp_l               1003dbcc f   LIBCMT:wcsnicmp.obj
 0001:0003ccb1       __wcsnicmp                 1003dcb1 f   LIBCMT:wcsnicmp.obj
 0001:0003cd4f       _wcsncmp                   1003dd4f f   LIBCMT:wcsncmp.obj
 0001:0003cd90       __global_unwind2           1003dd90 f   LIBCMT:exsup.obj
 0001:0003cdf5       __local_unwind2            1003ddf5 f   LIBCMT:exsup.obj
 0001:0003ce79       __abnormal_termination     1003de79 f   LIBCMT:exsup.obj
 0001:0003ce9c       __NLG_Notify1              1003de9c f   LIBCMT:exsup.obj
 0001:0003cea5       __NLG_Notify               1003dea5 f   LIBCMT:exsup.obj
 0001:0003cebc       __NLG_Dispatch2            1003debc     LIBCMT:exsup.obj
 0001:0003cebc       __NLG_Dispatch             1003debc     LIBCMT:exsup.obj
 0001:0003cec4       __NLG_Call                 1003dec4 f   LIBCMT:exsup.obj
 0001:0003cec6       __NLG_Return2              1003dec6     LIBCMT:exsup.obj
 0001:0003cec7       __calloc_impl              1003dec7 f   LIBCMT:calloc_impl.obj
 0001:0003cf49       _realloc                   1003df49 f   LIBCMT:realloc.obj
 0001:0003cff6       __recalloc                 1003dff6 f   LIBCMT:recalloc.obj
 0001:0003d064       __freea                    1003e064 f i LIBCMT:a_map.obj
 0001:0003d26b       ___crtLCMapStringA         1003e26b f   LIBCMT:a_map.obj
 0001:0003d398       ___crtGetStringTypeA       1003e398 f   LIBCMT:a_str.obj
 0001:0003d3d8       ___free_lc_time            1003e3d8 f   LIBCMT:inittime.obj
 0001:0003d74f       ___free_lconv_num          1003e74f f   LIBCMT:initnum.obj
 0001:0003d7b8       ___free_lconv_mon          1003e7b8 f   LIBCMT:initmon.obj
 0001:0003d8b6       ___crtLCMapStringW         1003e8b6 f   LIBCMT:w_map.obj
 0001:0003d8f0       _strcspn                   1003e8f0 f   LIBCMT:strcspn.obj
 0001:0003d940       _strcmp                    1003e940 f   LIBCMT:strcmp.obj
 0001:0003d9c8       __fputwc_nolock            1003e9c8 f   LIBCMT:fputwc.obj
 0001:0003db4f       __mbtowc_l                 1003eb4f f   LIBCMT:mbtowc.obj
 0001:0003dc65       _mbtowc                    1003ec65 f   LIBCMT:mbtowc.obj
 0001:0003dc7f       _strnlen                   1003ec7f f   LIBCMT:strlen_s.obj
 0001:0003dc9c       __setmode_nolock           1003ec9c f   LIBCMT:setmode.obj
 0001:0003dd57       __get_fmode                1003ed57 f   LIBCMT:setmode.obj
 0001:0003dd84       ___report_gsfailure        1003ed84 f   LIBCMT:gs_report.obj
 0001:0003de8a       __chsize_nolock            1003ee8a f   LIBCMT:chsize.obj
 0001:0003e040       __putwch_nolock            1003f040 f   LIBCMT:putwch.obj
 0001:0003e082       ___crtCompareStringW       1003f082 f   LIBCMT:w_cmp.obj
 0001:0003e19a       ___crtwsetenv              1003f19a f   LIBCMT:wsetenv.obj
 0001:0003e41a       __wdospawn                 1003f41a f   LIBCMT:wdospawn.obj
 0001:0003e629       __wcenvarg                 1003f629 f   LIBCMT:wcenvarg.obj
 0001:0003ea5a       __ismbblead                1003fa5a f   LIBCMT:ismbbyte.obj
 0001:0003ea72       __ld12tod                  1003fa72 f   LIBCMT:_intrncvt_.obj
 0001:0003efc3       __ld12tof                  1003ffc3 f   LIBCMT:_intrncvt_.obj
 0001:0003f514       ___strgtold12_l            10040514 f   LIBCMT:_strgtold_.obj
 0001:0003fbf0       _$I10_OUTPUT               10040bf0 f   LIBCMT:_x10fout_.obj
 0001:000404e8       _abort                     100414e8 f   LIBCMT:abort.obj
 0001:0004051b       __msize                    1004151b f   LIBCMT:msize.obj
 0001:00040550       __alloca_probe_16          10041550 f   LIBCMT:alloca16.obj
 0001:00040566       __alloca_probe_8           10041566     LIBCMT:alloca16.obj
 0001:0004057c       __flswbuf                  1004157c f   LIBCMT:_flswbuf.obj
 0001:000406f0       ___initconout              100416f0 f   LIBCMT:initcon.obj
 0001:0004070f       ___termconout              1004170f f   LIBCMT:initcon.obj
 0001:00040726       ___mtold12                 10041726 f   LIBCMT:_mantold_.obj
 0001:00040910       ___ascii_strnicmp          10041910 f   LIBCMT:_strnicm.obj
 0001:00040972       _RtlUnwind@16              10041972 f   kernel32:KERNEL32.dll
 0001:00040aec       __strupr_s_l               10041aec f   LIBCMT:strupr.obj
 0001:00040b21       _strupr                    10041b21 f   LIBCMT:strupr.obj
 0001:00040b21       __strupr                   10041b21 f   LIBCMT:strupr.obj
 0001:0004120c       __IMPORT_DESCRIPTOR_KERNEL32 1004220c     kernel32:KERNEL32.dll
 0001:00041220       __IMPORT_DESCRIPTOR_ADVAPI32 10042220     advapi32:ADVAPI32.dll
 0001:00041234       __IMPORT_DESCRIPTOR_SHELL32 10042234     shell32:SHELL32.dll
 0001:00041248       __IMPORT_DESCRIPTOR_lua51  10042248     lua51:lua51.dll
 0001:0004125c       __IMPORT_DESCRIPTOR_RPCRT4 1004225c     rpcrt4:RPCRT4.dll
 0001:00041270       __NULL_IMPORT_DESCRIPTOR   10042270     kernel32:KERNEL32.dll
 0002:00000000       _Keys                      10044000     flags.obj
 0002:00000ac8       _VirtualKeyStrings         10044ac8     service.obj
 0002:00007c34       __fltused                  1004bc34     LIBCMT:_fpinit_.obj
 0002:00007c38       __ldused                   1004bc38     LIBCMT:_fpinit_.obj
 0002:00007db0       __iob                      1004bdb0     LIBCMT:_file.obj
 0002:00008030       __cfltcvt_tab              1004c030     LIBCMT:cmiscdat.obj
 0002:00008058       ___nullstring              1004c058     LIBCMT:output.obj
 0002:0000805c       ___wnullstring             1004c05c     LIBCMT:output.obj
 0002:00008080       ___security_cookie         1004c080     LIBCMT:gs_cookie.obj
 0002:00008084       ___security_cookie_complement 1004c084     LIBCMT:gs_cookie.obj
 0002:00008090       __lookuptrailbytes         1004c090     LIBCMT:read.obj
 0002:00008190       __sys_errlist              1004c190     LIBCMT:syserr.obj
 0002:00008240       __sys_nerr                 1004c240     LIBCMT:syserr.obj
 0002:00008244       ___flsindex                1004c244     LIBCMT:tidtable.obj
 0002:00008248       ___getvalueindex           1004c248     LIBCMT:tidtable.obj
 0002:00008250       ___badioinfo               1004c250     LIBCMT:ioinit.obj
 0002:000083b0       __pctype                   1004c3b0     LIBCMT:ctype.obj
 0002:000083b4       __pwctype                  1004c3b4     LIBCMT:ctype.obj
 0002:000083b8       ___initialmbcinfo          1004c3b8     LIBCMT:mbctype.obj
 0002:000085d8       __mbctype                  1004c5d8     LIBCMT:mbctype.obj
 0002:000086e0       __mbcasemap                1004c6e0     LIBCMT:mbctype.obj
 0002:000087e0       ___ptmbcinfo               1004c7e0     LIBCMT:mbctype.obj
 0002:000088d8       ___globallocalestatus      1004c8d8     LIBCMT:glstatus.obj
 0002:000088dc       ___clocalestr              1004c8dc     LIBCMT:nlsdata2.obj
 0002:000088e0       ___lc_time_c               1004c8e0     LIBCMT:nlsdata2.obj
 0002:00008a48       ___initiallocinfo          1004ca48     LIBCMT:nlsdata2.obj
 0002:00008b20       ___ptlocinfo               1004cb20     LIBCMT:nlsdata2.obj
 0002:00008b24       ___initiallocalestructinfo 1004cb24     LIBCMT:nlsdata2.obj
 0002:00008b30       __tmpoff                   1004cb30     LIBCMT:rmtmp.obj
 0002:00008b34       __tempoff                  1004cb34     LIBCMT:rmtmp.obj
 0002:00008b50       __NLG_Destination          1004cb50     LIBCMT:exsup.obj
 0002:00008b60       ___lconv_static_decimal    1004cb60     LIBCMT:lconv.obj
 0002:00008b64       ___lconv_static_W_decimal  1004cb64     LIBCMT:lconv.obj
 0002:00008b68       ___lconv_c                 1004cb68     LIBCMT:lconv.obj
 0002:00008bb8       ___lconv                   1004cbb8     LIBCMT:lconv.obj
 0002:00008bbc       ___mb_cur_max              1004cbbc     LIBCMT:nlsdata1.obj
 0002:00008bc0       ___decimal_point           1004cbc0     LIBCMT:nlsdata1.obj
 0002:00008bc4       ___decimal_point_length    1004cbc4     LIBCMT:nlsdata1.obj
 0002:00008c00       ___abort_behavior          1004cc00     LIBCMT:abort.obj
 0002:00008c10       __confh                    1004cc10     LIBCMT:initcon.obj
 0002:00008c18       __pow10pos                 1004cc18     LIBCMT:_constpow_.obj
 0002:00008d78       __pow10neg                 1004cd78     LIBCMT:_constpow_.obj
 0002:00008eec       ___fastflag                1004ceec     LIBCMT:_fpinit_.obj
 0002:00008ef0       __cflush                   1004cef0     LIBCMT:_file.obj
 0002:00008ef4       ___idtabsiz                1004cef4     LIBCMT:popen.obj
 0002:00008ef8       ___idpairs                 1004cef8     LIBCMT:popen.obj
 0002:00008f38       __aenvptr                  1004cf38     LIBCMT:dllcrt0.obj
 0002:00008f3c       __wenvptr                  1004cf3c     LIBCMT:dllcrt0.obj
 0002:00008f40       ___error_mode              1004cf40     LIBCMT:dllcrt0.obj
 0002:00008f44       ___app_type                1004cf44     LIBCMT:dllcrt0.obj
 0002:00008f48       ___pInvalidArgHandler      1004cf48     LIBCMT:invarg.obj
 0002:00008f60       __crtheap                  1004cf60     LIBCMT:heapinit.obj
 0002:00008f64       __umaskval                 1004cf64     LIBCMT:crt0dat.obj
 0002:00008f68       ___argc                    1004cf68     LIBCMT:crt0dat.obj
 0002:00008f6c       ___argv                    1004cf6c     LIBCMT:crt0dat.obj
 0002:00008f70       ___wargv                   1004cf70     LIBCMT:crt0dat.obj
 0002:00008f74       __environ                  1004cf74     LIBCMT:crt0dat.obj
 0002:00008f78       ___initenv                 1004cf78     LIBCMT:crt0dat.obj
 0002:00008f7c       __wenviron                 1004cf7c     LIBCMT:crt0dat.obj
 0002:00008f80       ___winitenv                1004cf80     LIBCMT:crt0dat.obj
 0002:00008f84       __pgmptr                   1004cf84     LIBCMT:crt0dat.obj
 0002:00008f88       __wpgmptr                  1004cf88     LIBCMT:crt0dat.obj
 0002:00008f8c       __exitflag                 1004cf8c     LIBCMT:crt0dat.obj
 0002:00008f90       __C_Termination_Done       1004cf90     LIBCMT:crt0dat.obj
 0002:00008f94       __C_Exit_Done              1004cf94     LIBCMT:crt0dat.obj
 0002:000095c0       ?_pnhHeap@@3P6AHI@ZA       1004d5c0     LIBCMT:handler.obj
 0002:000095c4       __newmode                  1004d5c4     LIBCMT:_newmode.obj
 0002:000095c8       __maxwait                  1004d5c8     LIBCMT:crtheap.obj
 0002:000095cc       _gpFlsAlloc                1004d5cc     LIBCMT:tidtable.obj
 0002:000095d0       _gpFlsGetValue             1004d5d0     LIBCMT:tidtable.obj
 0002:000095d4       _gpFlsSetValue             1004d5d4     LIBCMT:tidtable.obj
 0002:000095d8       _gpFlsFree                 1004d5d8     LIBCMT:tidtable.obj
 0002:00009734       ___mbulinfo                1004d734     LIBCMT:mbctype.obj
 0002:00009740       ___mbcodepage              1004d740     LIBCMT:mbctype.obj
 0002:00009744       ___ismbcodepage            1004d744     LIBCMT:mbctype.obj
 0002:00009748       ___mblcid                  1004d748     LIBCMT:mbctype.obj
 0002:0000974c       ___locale_changed          1004d74c     LIBCMT:setlocal.obj
 0002:00009750       __stdbuf                   1004d750     LIBCMT:_sftbuf.obj
 0002:00009758       __old_pfxlen               1004d758     LIBCMT:rmtmp.obj
 0002:0000975c       __commode                  1004d75c     LIBCMT:ncommode.obj
 0002:00009868       __outputformat             1004d868     LIBCMT:outputformat.obj
 0002:00009870       ?__pInconsistency@@3P6AXXZA 1004d870     LIBCMT:hooks.obj
 0002:00009878       ___pPurecall               1004d878     LIBCMT:inithelp.obj
 0002:00009890       ___lconv_static_null       1004d890     LIBCMT:lconv.obj
 0002:00009894       ___lconv_static_W_null     1004d894     LIBCMT:lconv.obj
 0002:00009bbc       __fmode                    1004dbbc     LIBCMT:txtmode.obj
 0002:00009bc0       _EnumCP                    1004dbc0     <common>
 0002:00009bc8       __debugger_hook_dummy      1004dbc8     <common>
 0002:00009bcc       __nhandle                  1004dbcc     <common>
 0002:00009be0       ___pioinfo                 1004dbe0     <common>
 0002:00009ce0       __pDestructExceptionObject 1004dce0     <common>
 0002:00009ce4       ___env_initialized         1004dce4     <common>
 0002:00009ce8       ___onexitend               1004dce8     <common>
 0002:00009cec       ___onexitbegin             1004dcec     <common>
 0002:00009cf0       ___mbctype_initialized     1004dcf0     <common>
 0002:00009cf4       ___dyn_tls_init_callback   1004dcf4     <common>
 0002:00009cf8       ___sse2_available          1004dcf8     <common>
 0002:00009cfc       __acmdln                   1004dcfc     <common>
 0002:00009d00       ___piob                    1004dd00     <common>
 0002:00009d20       __bufin                    1004dd20     <common>
 0002:0000ad20       __nstream                  1004ed20     <common>

 entry point at        0001:000315c7

 Static symbols

 0001:00011280       _band                      10012280 f   bit64.obj
 0001:00011400       _bor                       10012400 f   bit64.obj
 0001:00011580       _bxor                      10012580 f   bit64.obj
 0001:00011700       _bnot                      10012700 f   bit64.obj
 0001:000117f0       _lshift                    100127f0 f   bit64.obj
 0001:000118e0       _rshift                    100128e0 f   bit64.obj
 0001:000119d0       _arshift                   100129d0 f   bit64.obj
 0001:00011ac0       _f_new                     10012ac0 f   bit64.obj
 0001:00011cf0       _f_tostring                10012cf0 f   bit64.obj
 0001:00011dc0       _f_type                    10012dc0 f   bit64.obj
 0001:00011e30       _f_add                     10012e30 f   bit64.obj
 0001:00011fb0       _f_sub                     10012fb0 f   bit64.obj
 0001:00012110       _f_mul                     10013110 f   bit64.obj
 0001:000122a0       _f_div                     100132a0 f   bit64.obj
 0001:000124c0       _f_mod                     100134c0 f   bit64.obj
 0001:00012630       _f_unm                     10013630 f   bit64.obj
 0001:000126f0       _f_eq                      100136f0 f   bit64.obj
 0001:00012860       _f_lt                      10013860 f   bit64.obj
 0001:000129d0       _f_le                      100139d0 f   bit64.obj
 0001:00013820       _RunDefaultScript          10014820 f   exported.obj
 0001:00013a20       _CheckReloadDefaultScript  10014a20 f   exported.obj
 0001:00013a90       _RegisterObject            10014a90 f   exported.obj
 0001:00013ad0       _PushAnalyseInfo           10014ad0 f   exported.obj
 0001:000144a0       _FillFarMacroCall_Callback@12 100154a0 f   exported.obj
 0001:00014500       _FillFarMacroCall          10015500 f   exported.obj
 0001:00016090       _getF                      10017090 f   lflua.obj
 0001:000160f0       _errfile                   100170f0 f   lflua.obj
 0001:00016130       _skipBOM                   10017130 f   lflua.obj
 0001:00017520       _FL_PushParams             10018520 f   luamacro.obj
 0001:00017950       _MacroCallFarCallback@12   10018950 f   luamacro.obj
 0001:00017bb0       _uc_tostring               10018bb0 f   lusercontrol.obj
 0001:00017c10       _uc_index                  10018c10 f   lusercontrol.obj
 0001:00017c90       _uc_newindex               10018c90 f   lusercontrol.obj
 0001:00017d50       _uc_New                    10018d50 f   lusercontrol.obj
 0001:00018050       _CreateSynchroData         10019050 f   service.obj
 0001:00018100       _get_env_flag              10019100 f   service.obj
 0001:00018230       _check_env_flag            10019230 f   service.obj
 0001:00018490       _CheckFlags                10019490 f   service.obj
 0001:000184d0       _CheckFlagsFromTable       100194d0 f   service.obj
 0001:00018700       _far_GetFileOwner          10019700 f   service.obj
 0001:00018790       _far_GetNumberOfLinks      10019790 f   service.obj
 0001:000187e0       _GetMouseEvent             100197e0 f   service.obj
 0001:00018910       _PushEditorSetPosition     10019910 f   service.obj
 0001:00018980       _FillEditorSetPosition     10019980 f   service.obj
 0001:00018ea0       _far_PluginStartupInfo     10019ea0 f   service.obj
 0001:00018f40       _far_GetCurrentDirectory   10019f40 f   service.obj
 0001:00018fa0       _editor_GetFileName        10019fa0 f   service.obj
 0001:00019050       _editor_GetInfo            1001a050 f   service.obj
 0001:00019350       _FastGetString             1001a350 f   service.obj
 0001:000193b0       __EditorGetString          1001a3b0 f   service.obj
 0001:000195c0       _editor_GetString          1001a5c0 f   service.obj
 0001:000195d0       _editor_GetStringW         1001a5d0 f   service.obj
 0001:000195e0       __EditorSetString          1001a5e0 f   service.obj
 0001:000196d0       _editor_SetString          1001a6d0 f   service.obj
 0001:000196f0       _editor_SetStringW         1001a6f0 f   service.obj
 0001:00019710       _editor_InsertString       1001a710 f   service.obj
 0001:00019780       _editor_DeleteString       1001a780 f   service.obj
 0001:000197d0       __EditorInsertText         1001a7d0 f   service.obj
 0001:000198a0       _editor_InsertText         1001a8a0 f   service.obj
 0001:00019900       _editor_InsertTextW        1001a900 f   service.obj
 0001:00019920       _editor_DeleteChar         1001a920 f   service.obj
 0001:00019970       _editor_DeleteBlock        1001a970 f   service.obj
 0001:000199c0       _editor_UndoRedo           1001a9c0 f   service.obj
 0001:00019a60       _FillKeyBarTitles          1001aa60 f   service.obj
 0001:00019bf0       _SetKeyBar                 1001abf0 f   service.obj
 0001:00019d40       _editor_SetKeyBar          1001ad40 f   service.obj
 0001:00019d50       _viewer_SetKeyBar          1001ad50 f   service.obj
 0001:00019d60       _editor_SetParam           1001ad60 f   service.obj
 0001:00019ed0       _editor_SetPosition        1001aed0 f   service.obj
 0001:00019fb0       _editor_Redraw             1001afb0 f   service.obj
 0001:0001a000       _editor_ExpandTabs         1001b000 f   service.obj
 0001:0001a060       _PushBookmarks             1001b060 f   service.obj
 0001:0001a1d0       _editor_GetBookmarks       1001b1d0 f   service.obj
 0001:0001a1f0       _editor_GetSessionBookmarks 1001b1f0 f   service.obj
 0001:0001a210       _editor_AddSessionBookmark 1001b210 f   service.obj
 0001:0001a260       _editor_ClearSessionBookmarks 1001b260 f   service.obj
 0001:0001a2b0       _editor_DeleteSessionBookmark 1001b2b0 f   service.obj
 0001:0001a310       _editor_NextSessionBookmark 1001b310 f   service.obj
 0001:0001a360       _editor_PrevSessionBookmark 1001b360 f   service.obj
 0001:0001a3b0       _editor_SetTitle           1001b3b0 f   service.obj
 0001:0001a410       _editor_GetTitle           1001b410 f   service.obj
 0001:0001a4a0       _editor_Quit               1001b4a0 f   service.obj
 0001:0001a4f0       _FillEditorSelect          1001b4f0 f   service.obj
 0001:0001a590       _editor_Select             1001b590 f   service.obj
 0001:0001a690       _editor_GetSelection       1001b690 f   service.obj
 0001:0001aa10       __EditorTabConvert         1001ba10 f   service.obj
 0001:0001aaa0       _editor_TabToReal          1001baa0 f   service.obj
 0001:0001aac0       _editor_RealToTab          1001bac0 f   service.obj
 0001:0001acb0       _GetOptGuid                1001bcb0 f   service.obj
 0001:0001ad30       _editor_AddColor           1001bd30 f   service.obj
 0001:0001ae80       _editor_DelColor           1001be80 f   service.obj
 0001:0001af20       _editor_GetColor           1001bf20 f   service.obj
 0001:0001b070       _editor_SaveFile           1001c070 f   service.obj
 0001:0001b2b0       _editor_ReadInput          1001c2b0 f   service.obj
 0001:0001b540       _OptInputRecord            1001c540 f   service.obj
 0001:0001b5c0       _editor_ProcessInput       1001c5c0 f   service.obj
 0001:0001b630       _editor_SubscribeChangeEvent 1001c630 f   service.obj
 0001:0001b6c0       _far_Menu                  1001c6c0 f   service.obj
 0001:0001c340       _far_Message               1001d340 f   service.obj
 0001:0001c480       _panel_CheckPanelsExist    1001d480 f   service.obj
 0001:0001c4c0       _panel_ClosePanel          1001d4c0 f   service.obj
 0001:0001c510       _panel_GetPanelInfo        1001d510 f   service.obj
 0001:0001c700       _get_panel_item            1001d700 f   service.obj
 0001:0001c7f0       _panel_GetPanelItem        1001d7f0 f   service.obj
 0001:0001c810       _panel_GetSelectedPanelItem 1001d810 f   service.obj
 0001:0001c830       _panel_GetCurrentPanelItem 1001d830 f   service.obj
 0001:0001c850       _get_string_info           1001d850 f   service.obj
 0001:0001c910       _panel_GetPanelFormat      1001d910 f   service.obj
 0001:0001c930       _panel_GetPanelHostFile    1001d930 f   service.obj
 0001:0001c950       _panel_GetColumnTypes      1001d950 f   service.obj
 0001:0001c970       _panel_GetColumnWidths     1001d970 f   service.obj
 0001:0001c990       _panel_GetPanelPrefix      1001d990 f   service.obj
 0001:0001c9b0       _panel_RedrawPanel         1001d9b0 f   service.obj
 0001:0001ca90       _SetPanelBooleanProperty   1001da90 f   service.obj
 0001:0001cb20       _SetPanelIntegerProperty   1001db20 f   service.obj
 0001:0001cbe0       _panel_SetCaseSensitiveSort 1001dbe0 f   service.obj
 0001:0001cc00       _panel_SetNumericSort      1001dc00 f   service.obj
 0001:0001cc20       _panel_SetSortOrder        1001dc20 f   service.obj
 0001:0001cc40       _panel_SetDirectoriesFirst 1001dc40 f   service.obj
 0001:0001cc60       _panel_UpdatePanel         1001dc60 f   service.obj
 0001:0001cc80       _panel_SetSortMode         1001dc80 f   service.obj
 0001:0001cc90       _panel_SetViewMode         1001dc90 f   service.obj
 0001:0001cca0       _panel_GetPanelDirectory   1001dca0 f   service.obj
 0001:0001cdb0       _panel_SetPanelDirectory   1001ddb0 f   service.obj
 0001:0001cf70       _panel_GetCmdLine          1001df70 f   service.obj
 0001:0001cff0       _panel_SetCmdLine          1001dff0 f   service.obj
 0001:0001d050       _panel_GetCmdLinePos       1001e050 f   service.obj
 0001:0001d0c0       _panel_SetCmdLinePos       1001e0c0 f   service.obj
 0001:0001d120       _panel_InsertCmdLine       1001e120 f   service.obj
 0001:0001d180       _panel_GetCmdLineSelection 1001e180 f   service.obj
 0001:0001d210       _panel_SetCmdLineSelection 1001e210 f   service.obj
 0001:0001d2a0       _ChangePanelSelection      1001e2a0 f   service.obj
 0001:0001d4a0       _panel_SetSelection        1001e4a0 f   service.obj
 0001:0001d4c0       _panel_ClearSelection      1001e4c0 f   service.obj
 0001:0001d4d0       _panel_SetUserScreen       1001e4d0 f   service.obj
 0001:0001d520       _panel_GetUserScreen       1001e520 f   service.obj
 0001:0001d570       _panel_IsActivePanel       1001e570 f   service.obj
 0001:0001d5c0       _panel_SetActivePanel      1001e5c0 f   service.obj
 0001:0001d640       _far_GetDirList            1001e640 f   service.obj
 0001:0001d940       _far_GetPluginDirList      1001e940 f   service.obj
 0001:0001d9d0       _far_RestoreScreen         1001e9d0 f   service.obj
 0001:0001da50       _far_SaveScreen            1001ea50 f   service.obj
 0001:0001daf0       _GetDialogItemType         1001eaf0 f   service.obj
 0001:0001dd00       _PushList                  1001ed00 f   service.obj
 0001:0001dda0       _SetFarDialogItem          1001eda0 f   service.obj
 0001:0001e000       _PushDlgItem               1001f000 f   service.obj
 0001:0001e0f0       _PushDlgItemNum            1001f0f0 f   service.obj
 0001:0001e1a0       _SetDlgItem                1001f1a0 f   service.obj
 0001:0001e3c0       _far_SendDlgMessage        1001f3c0 f   service.obj
 0001:0001fac0       _far_DialogInit            10020ac0 f   service.obj
 0001:0001fd90       _far_DialogRun             10020d90 f   service.obj
 0001:0001fe40       _far_DialogFree            10020e40 f   service.obj
 0001:0001fea0       _dialog_tostring           10020ea0 f   service.obj
 0001:0001ff00       _dialog_rawhandle          10020f00 f   service.obj
 0001:0001ff40       _far_GetDlgItem            10020f40 f   service.obj
 0001:0001ffb0       _far_SetDlgItem            10020fb0 f   service.obj
 0001:00020020       _far_SubscribeDialogDrawEvents 10021020 f   service.obj
 0001:00020040       _editor_Editor             10021040 f   service.obj
 0001:00020160       _viewer_Viewer             10021160 f   service.obj
 0001:00020260       _viewer_GetFileName        10021260 f   service.obj
 0001:00020310       _viewer_GetInfo            10021310 f   service.obj
 0001:00020570       _viewer_Quit               10021570 f   service.obj
 0001:000205b0       _viewer_Redraw             100215b0 f   service.obj
 0001:000205f0       _viewer_Select             100215f0 f   service.obj
 0001:00020680       _viewer_SetPosition        10021680 f   service.obj
 0001:00020830       _viewer_SetMode            10021830 f   service.obj
 0001:00020930       _far_ShowHelp              10021930 f   service.obj
 0001:000209c0       _far_InputBox              100219c0 f   service.obj
 0001:00020b40       _far_GetMsg                10021b40 f   service.obj
 0001:00020bb0       _far_Text                  10021bb0 f   service.obj
 0001:00020c40       _far_CopyToClipboard       10021c40 f   service.obj
 0001:00020d20       _far_PasteFromClipboard    10021d20 f   service.obj
 0001:00020df0       _far_InputRecordToName     10021df0 f   service.obj
 0001:00020fc0       _far_NameToInputRecord     10021fc0 f   service.obj
 0001:00021030       _far_LStricmp              10022030 f   service.obj
 0001:00021080       _far_LStrnicmp             10022080 f   service.obj
 0001:000210f0       _far_ProcessName           100220f0 f   service.obj
 0001:00021310       _far_GetReparsePointInfo   10022310 f   service.obj
 0001:000213a0       _far_LIsAlpha              100223a0 f   service.obj
 0001:000213f0       _far_LIsAlphanum           100223f0 f   service.obj
 0001:00021440       _far_LIsLower              10022440 f   service.obj
 0001:00021490       _far_LIsUpper              10022490 f   service.obj
 0001:000214e0       _far_LLowerBuf             100224e0 f   service.obj
 0001:00021540       _far_LUpperBuf             10022540 f   service.obj
 0001:000215a0       _far_MkTemp                100225a0 f   service.obj
 0001:00021620       _far_MkLink                10022620 f   service.obj
 0001:000216f0       _far_GetPathRoot           100226f0 f   service.obj
 0001:00021770       _truncstring               10022770 f   service.obj
 0001:00021830       _far_TruncPathStr          10022830 f   service.obj
 0001:00021850       _far_TruncStr              10022850 f   service.obj
 0001:00021870       _FrsUserFunc@12            10022870 f   service.obj
 0001:00021930       _far_RecursiveSearch       10022930 f   service.obj
 0001:00021a40       _far_ConvertPath           10022a40 f   service.obj
 0001:00021b00       _far_AdvControl            10022b00 f   service.obj
 0001:00022240       _far_MacroLoadAll          10023240 f   service.obj
 0001:00022300       _far_MacroSaveAll          10023300 f   service.obj
 0001:00022350       _far_MacroGetState         10023350 f   service.obj
 0001:00022390       _far_MacroGetArea          10023390 f   service.obj
 0001:000223d0       _MacroSendString           100233d0 f   service.obj
 0001:000224b0       _far_MacroPost             100234b0 f   service.obj
 0001:000224c0       _far_MacroCheck            100234c0 f   service.obj
 0001:000224d0       _far_MacroGetLastError     100234d0 f   service.obj
 0001:00022630       _far_MacroAdd              10023630 f   service.obj
 0001:00022810       _far_MacroDelete           10023810 f   service.obj
 0001:000228a0       _AddMacroData_gc           100238a0 f   service.obj
 0001:000228b0       _far_MacroExecute          100238b0 f   service.obj
 0001:000229e0       _far_CPluginStartupInfo    100239e0 f   service.obj
 0001:00022a60       _far_MakeMenuItems         10023a60 f   service.obj
 0001:00022d10       _far_Show                  10023d10 f   service.obj
 0001:00022e10       _far_CreateFileFilter      10023e10 f   service.obj
 0001:00022ee0       _filefilter_Free           10023ee0 f   service.obj
 0001:00022f60       _filefilter_gc             10023f60 f   service.obj
 0001:00022f70       _filefilter_tostring       10023f70 f   service.obj
 0001:00022fc0       _filefilter_OpenMenu       10023fc0 f   service.obj
 0001:00023030       _filefilter_Starting       10024030 f   service.obj
 0001:000230a0       _filefilter_IsFileInFilter 100240a0 f   service.obj
 0001:00023140       _plugin_load               10024140 f   service.obj
 0001:00023200       _far_LoadPlugin            10024200 f   service.obj
 0001:00023210       _far_ForcedLoadPlugin      10024210 f   service.obj
 0001:00023220       _far_UnloadPlugin          10024220 f   service.obj
 0001:00023270       _far_FindPlugin            10024270 f   service.obj
 0001:00023350       _PutPluginMenuItemToTable  10024350 f   service.obj
 0001:00023410       _PutVersionInfoToTable     10024410 f   service.obj
 0001:00023470       _far_GetPluginInformation  10024470 f   service.obj
 0001:00023680       _far_GetPlugins            10024680 f   service.obj
 0001:00023760       _far_IsPluginLoaded        10024760 f   service.obj
 0001:00023870       _far_XLat                  10024870 f   service.obj
 0001:00023960       _far_FormatFileSize        10024960 f   service.obj
 0001:00023a50       _far_FarClock              10024a50 f   service.obj
 0001:00023bc0       _far_Timer                 10024bc0 f   service.obj
 0001:00023d20       _timer_Close               10024d20 f   service.obj
 0001:00023d40       _timer_tostring            10024d40 f   service.obj
 0001:00023d90       _timer_index               10024d90 f   service.obj
 0001:00023f60       _timer_newindex            10024f60 f   service.obj
 0001:00024100       _far_CreateSettings        10025100 f   service.obj
 0001:00024310       _Settings_set              10025310 f   service.obj
 0001:00024440       _Settings_get              10025440 f   service.obj
 0001:00024590       _Settings_delete           10025590 f   service.obj
 0001:00024630       _Settings_createsubkey     10025630 f   service.obj
 0001:00024740       _Settings_opensubkey       10025740 f   service.obj
 0001:000247f0       _Settings_enum             100257f0 f   service.obj
 0001:00024ab0       _Settings_free             10025ab0 f   service.obj
 0001:00024b30       _far_FreeSettings          10025b30 f   service.obj
 0001:00024bb0       _Settings_tostring         10025bb0 f   service.obj
 0001:00024c10       _far_ColorDialog           10025c10 f   service.obj
 0001:00024f40       _CustomAllocator           10025f40 f   service.obj
 0001:00025020       _luaopen_far               10026020 f   service.obj
 0001:00025360       _grab_one_utf8             10026360 f   slnunico.obj
 0001:000253e0       _utf8_enco                 100263e0 f   slnunico.obj
 0001:000254d0       _utf8_deco                 100264d0 f   slnunico.obj
 0001:000255b0       _utf8_oced                 100265b0 f   slnunico.obj
 0001:00025680       _utf8_graphext             10026680 f   slnunico.obj
 0001:000257a0       _utf8_count                100267a0 f   slnunico.obj
 0001:00025830       _unic_len                  10026830 f   slnunico.obj
 0001:000258b0       _unic_sub                  100268b0 f   slnunico.obj
 0001:00025a00       _str_reverse               10026a00 f   slnunico.obj
 0001:00025b60       _unic_lower                10026b60 f   slnunico.obj
 0001:00025cb0       _unic_upper                10026cb0 f   slnunico.obj
 0001:00025e00       _str_rep                   10026e00 f   slnunico.obj
 0001:00025e80       _unic_byte                 10026e80 f   slnunico.obj
 0001:00026010       _unic_char                 10027010 f   slnunico.obj
 0001:00026110       _writer                    10027110 f   slnunico.obj
 0001:00026130       _str_dump                  10027130 f   slnunico.obj
 0001:000261a0       _classend                  100271a0 f   slnunico.obj
 0001:00026240       _match_class               10027240 f   slnunico.obj
 0001:00026390       _singlematch               10027390 f   slnunico.obj
 0001:00026650       _matchbalance              10027650 f   slnunico.obj
 0001:000266c0       _max_expand                100276c0 f   slnunico.obj
 0001:000267c0       _start_capture             100277c0 f   slnunico.obj
 0001:00026810       _end_capture               10027810 f   slnunico.obj
 0001:00026870       _match_capture             10027870 f   slnunico.obj
 0001:00026900       _match                     10027900 f   slnunico.obj
 0001:00026b10       _lmemfind                  10027b10 f   slnunico.obj
 0001:00026bc0       _push_onecapture           10027bc0 f   slnunico.obj
 0001:00026c40       _push_captures             10027c40 f   slnunico.obj
 0001:00026d00       _unic_find_aux             10027d00 f   slnunico.obj
 0001:00026f00       _unic_find                 10027f00 f   slnunico.obj
 0001:00026f10       _unic_match                10027f10 f   slnunico.obj
 0001:00026f20       _gmatch_aux                10027f20 f   slnunico.obj
 0001:00027000       _gmatch                    10028000 f   slnunico.obj
 0001:000270b0       _gfind_nodef               100280b0 f   slnunico.obj
 0001:000270d0       _add_s                     100280d0 f   slnunico.obj
 0001:000271b0       _add_value                 100281b0 f   slnunico.obj
 0001:000272d0       _unic_gsub                 100282d0 f   slnunico.obj
 0001:00027470       _addquoted                 10028470 f   slnunico.obj
 0001:000275d0       _scanformat                100285d0 f   slnunico.obj
 0001:000276d0       _str_format                100286d0 f   slnunico.obj
 0001:00027a30       _utf8_valid                10028a30 f   slnunico.obj
 0001:00027c60       _pushresult                10028c60 f   uliolib51.obj
 0001:00027d00       _fileerror                 10028d00 f   uliolib51.obj
 0001:00027d50       _io_type                   10028d50 f   uliolib51.obj
 0001:00027df0       _io_noclose                10028df0 f   uliolib51.obj
 0001:00027e20       _io_pclose                 10028e20 f   uliolib51.obj
 0001:00027ea0       _io_fclose                 10028ea0 f   uliolib51.obj
 0001:00027f20       _io_close                  10028f20 f   uliolib51.obj
 0001:00027fa0       _io_gc                     10028fa0 f   uliolib51.obj
 0001:00027ff0       _io_tostring               10028ff0 f   uliolib51.obj
 0001:00028040       _io_open                   10029040 f   uliolib51.obj
 0001:00028120       _io_popen                  10029120 f   uliolib51.obj
 0001:000281a0       _io_tmpfile                100291a0 f   uliolib51.obj
 0001:00028220       _g_iofile                  10029220 f   uliolib51.obj
 0001:00028310       _io_input                  10029310 f   uliolib51.obj
 0001:00028330       _io_output                 10029330 f   uliolib51.obj
 0001:00028350       _read_number               10029350 f   uliolib51.obj
 0001:00028390       _read_line                 10029390 f   uliolib51.obj
 0001:00028460       _read_chars                10029460 f   uliolib51.obj
 0001:000284f0       _g_read                    100294f0 f   uliolib51.obj
 0001:00028680       _io_read                   10029680 f   uliolib51.obj
 0001:000286d0       _f_read                    100296d0 f   uliolib51.obj
 0001:00028710       _io_readline               10029710 f   uliolib51.obj
 0001:000287d0       _g_write                   100297d0 f   uliolib51.obj
 0001:000288c0       _io_write                  100298c0 f   uliolib51.obj
 0001:00028910       _f_write                   10029910 f   uliolib51.obj
 0001:00028950       _f_seek                    10029950 f   uliolib51.obj
 0001:00028a00       _f_setvbuf                 10029a00 f   uliolib51.obj
 0001:00028ab0       _io_flush                  10029ab0 f   uliolib51.obj
 0001:00028b40       _f_flush                   10029b40 f   uliolib51.obj
 0001:00028df0       _f_lines                   10029df0 f   uliolib51.obj
 0001:00028e40       _io_lines                  10029e40 f   uliolib51.obj
 0001:00028f20       _setprogdir                10029f20 f   uloadlib51.obj
 0001:00028fa0       _ll_register               10029fa0 f   uloadlib51.obj
 0001:00029050       _gctm                      1002a050 f   uloadlib51.obj
 0001:00029080       _ll_loadfunc               1002a080 f   uloadlib51.obj
 0001:000290f0       _ll_loadlib                1002a0f0 f   uloadlib51.obj
 0001:00029160       _pushnexttemplate          1002a160 f   uloadlib51.obj
 0001:000291e0       _findfile                  1002a1e0 f   uloadlib51.obj
 0001:00029310       _loaderror                 1002a310 f   uloadlib51.obj
 0001:00029350       _loader_Lua                1002a350 f   uloadlib51.obj
 0001:000293d0       _mkfuncname                1002a3d0 f   uloadlib51.obj
 0001:00029420       _loader_C                  1002a420 f   uloadlib51.obj
 0001:000294e0       _loader_Croot              1002a4e0 f   uloadlib51.obj
 0001:00029570       _loader_preload            1002a570 f   uloadlib51.obj
 0001:000295e0       _ll_require                1002a5e0 f   uloadlib51.obj
 0001:00029790       _setfenv                   1002a790 f   uloadlib51.obj
 0001:00029800       _dooptions                 1002a800 f   uloadlib51.obj
 0001:00029840       _modinit                   1002a840 f   uloadlib51.obj
 0001:000298a0       _ll_module                 1002a8a0 f   uloadlib51.obj
 0001:00029980       _ll_seeall                 1002a980 f   uloadlib51.obj
 0001:000299e0       _setpath                   1002a9e0 f   uloadlib51.obj
 0001:0002ae30       _ustring_OutputDebugString 1002be30 f   ustring.obj
 0001:0002aff0       _ustring_system            1002bff0 f   ustring.obj
 0001:0002c0d0       _win_GetEnv                1002d0d0 f   win.obj
 0001:0002c180       _win_SetEnv                1002d180 f   win.obj
 0001:0002c1c0       _CheckHKey                 1002d1c0 f   win.obj
 0001:0002c300       _win_SetRegKey             1002d300 f   win.obj
 0001:0002c550       _win_GetRegKey             1002d550 f   win.obj
 0001:0002c6f0       _win_DeleteRegKey          1002d6f0 f   win.obj
 0001:0002c730       _win_DeleteRegValue        1002d730 f   win.obj
 0001:0002c7c0       _win_EnumRegKey            1002d7c0 f   win.obj
 0001:0002c8b0       _win_EnumRegValue          1002d8b0 f   win.obj
 0001:0002c9a0       _ExtractKey                1002d9a0 f   win.obj
 0001:0002ca20       _win_ExtractKey            1002da20 f   win.obj
 0001:0002ca70       _PushWinFindData           1002da70 f   win.obj
 0001:0002cb30       _win_GetFileInfo           1002db30 f   win.obj
 0001:0002cba0       _pushSystemTime            1002dba0 f   win.obj
 0001:0002cc30       _win_GetSystemTimeAsFileTime 1002dc30 f   win.obj
 0001:0002cc60       _win_FileTimeToSystemTime  1002dc60 f   win.obj
 0001:0002ccd0       _win_SystemTimeToFileTime  1002dcd0 f   win.obj
 0001:0002cdd0       _win_FileTimeToLocalFileTime 1002ddd0 f   win.obj
 0001:0002ce40       _win_CompareString         1002de40 f   win.obj
 0001:0002cfe0       _win_wcscmp                1002dfe0 f   win.obj
 0001:0002d030       _win_GetVirtualKeys        1002e030 f   win.obj
 0001:0002d050       _win_GetConsoleScreenBufferInfo 1002e050 f   win.obj
 0001:0002d160       _win_CopyFile              1002e160 f   win.obj
 0001:0002d1d0       _win_MoveFile              1002e1d0 f   win.obj
 0001:0002d2a0       _win_DeleteFile            1002e2a0 f   win.obj
 0001:0002d2e0       _mkdir                     1002e2e0 f   win.obj
 0001:0002d480       _win_CreateDir             1002e480 f   win.obj
 0001:0002d560       _win_RemoveDir             1002e560 f   win.obj
 0001:0002d5a0       _win_ShellExecute          1002e5a0 f   win.obj
 0001:0002dc82       __hw_cw                    1002ec82 f   LIBCMT:_ieee87_.obj
 0001:0002dd10       ___hw_cw_sse2              1002ed10 f   LIBCMT:_ieee87_.obj
 0001:0002fcbf       _idtab                     10030cbf f   LIBCMT:wpopen.obj
 0001:0002fcbf       _idtab                     10030cbf f   LIBCMT:wpopen.obj
 0001:000301f1       _genfname                  100311f1 f   LIBCMT:tmpfile.obj
 0001:00030e0f       _flsall                    10031e0f f   LIBCMT:fflush.obj
 0001:000314d1       ___DllMainCRTStartup       100324d1 f   LIBCMT:dllcrt0.obj
 0001:00031758       __shift                    10032758 f   LIBCMT:cvt.obj
 0001:0003179d       __cftoe2_l                 1003279d f   LIBCMT:cvt.obj
 0001:00031d5b       __cftof2_l                 10032d5b f   LIBCMT:cvt.obj
 0001:00032276       _write_char                10033276 f   LIBCMT:output.obj
 0001:000322a9       _write_string              100332a9 f   LIBCMT:output.obj
 0001:00033152       _siglookup                 10034152 f   LIBCMT:winsig.obj
 0001:00033568       _doexit                    10034568 f   LIBCMT:crt0dat.obj
 0001:00034160       __unwind_handler4          10035160 f   LIBCMT:exsup4.obj
 0001:00035918       ?CPtoLCID@@YAHH@Z          10036918 f   LIBCMT:mbctype.obj
 0001:00035947       ?setSBCS@@YAXPAUthreadmbcinfostruct@@@Z 10036947 f   LIBCMT:mbctype.obj
 0001:000359ab       ?setSBUpLow@@YAXPAUthreadmbcinfostruct@@@Z 100369ab f   LIBCMT:mbctype.obj
 0001:00035bdf       ?getSystemCP@@YAHH@Z       10036bdf f   LIBCMT:mbctype.obj
 0001:0003655d       _write_char                1003755d f   LIBCMT:woutput.obj
 0001:0003658c       _write_string              1003758c f   LIBCMT:woutput.obj
 0001:00037a47       _xtoa_s@20                 10038a47 f   LIBCMT:xtoas.obj
 0001:00037b21       ?strtoxl@@YAKPAUlocaleinfo_struct@@PBDPAPBDHH@Z 10038b21 f   LIBCMT:strtol.obj
 0001:00037e82       __tsopen_nolock            10038e82 f   LIBCMT:open.obj
 0001:0003869a       ___check_float_string      1003969a f   LIBCMT:input.obj
 0001:000386f1       __hextodec                 100396f1 f   LIBCMT:input.obj
 0001:00038711       __inc                      10039711 f   LIBCMT:input.obj
 0001:00038727       __whiteout                 10039727 f   LIBCMT:input.obj
 0001:0003a5cc       _wcomexecmd                1003b5cc f   LIBCMT:wspawnve.obj
 0001:0003a908       _parse_cmdline             1003b908 f   LIBCMT:stdargv.obj
 0001:0003bae5       __onexit_nolock            1003cae5 f   LIBCMT:onexit.obj
 0001:0003c3b3       __tsopen_nolock            1003d3b3 f   LIBCMT:wopen.obj
 0001:0003cdb0       __unwind_handler           1003ddb0 f   LIBCMT:exsup.obj
 0001:0003d084       ?__crtLCMapStringA_stat@@YAHPAUlocaleinfo_struct@@KKPBDHPADHHH@Z 1003e084 f   LIBCMT:a_map.obj
 0001:0003d2b1       ?__crtGetStringTypeA_stat@@YAHPAUlocaleinfo_struct@@KPBDHPAGHHH@Z 1003e2b1 f   LIBCMT:a_str.obj
 0001:0003e0e5       _wfindenv                  1003f0e5 f   LIBCMT:wsetenv.obj
 0001:0003e13a       _copy_environ              1003f13a f   LIBCMT:wsetenv.obj
 0001:0003ea07       ?x_ismbbtype_l@@YAHPAUlocaleinfo_struct@@IHH@Z 1003fa07 f   LIBCMT:ismbbyte.obj
 0001:00040978       ?_strupr_s_l_stat@@YAHPADIPAUlocaleinfo_struct@@@Z 10041978 f   LIBCMT:strupr.obj
